Component: ARM Compiler 5.06 update 6 (build 750) Tool: armlink [4d35ed]

==============================================================================

Section Cross References

    main.o(i.CSC_Init) refers to mg32x02z__common_drv.o(i.UnProtectModuleReg) for UnProtectModuleReg
    main.o(i.CSC_Init) refers to mg32x02z_mem_drv.o(i.MEM_SetFlashWaitState) for MEM_SetFlashWaitState
    main.o(i.CSC_Init) refers to mg32x02z__common_drv.o(i.ProtectModuleReg) for ProtectModuleReg
    main.o(i.CSC_Init) refers to mg32x02z_csc_drv.o(i.CSC_CK_APB_Divider_Select) for CSC_CK_APB_Divider_Select
    main.o(i.CSC_Init) refers to mg32x02z_csc_drv.o(i.CSC_CK_AHB_Divider_Select) for CSC_CK_AHB_Divider_Select
    main.o(i.CSC_Init) refers to mg32x02z_csc_drv.o(i.CSC_IHRCO_Select) for CSC_IHRCO_Select
    main.o(i.CSC_Init) refers to mg32x02z_csc_drv.o(i.CSC_IHRCO_Cmd) for CSC_IHRCO_Cmd
    main.o(i.CSC_Init) refers to mg32x02z_csc_drv.o(i.CSC_GetSingleFlagStatus) for CSC_GetSingleFlagStatus
    main.o(i.CSC_Init) refers to mg32x02z_csc_drv.o(i.CSC_ClearFlag) for CSC_ClearFlag
    main.o(i.CSC_Init) refers to mg32x02z_csc_drv.o(i.CSC_CK_HS_Select) for CSC_CK_HS_Select
    main.o(i.CSC_Init) refers to mg32x02z_csc_drv.o(i.CSC_PLL_Config) for CSC_PLL_Config
    main.o(i.CSC_Init) refers to mg32x02z_csc_drv.o(i.CSC_PLL_Cmd) for CSC_PLL_Cmd
    main.o(i.CSC_Init) refers to mg32x02z_csc_drv.o(i.CSC_CK_MAIN_Select) for CSC_CK_MAIN_Select
    main.o(i.DMA_Init) refers to mg32x02z__common_drv.o(i.UnProtectModuleReg) for UnProtectModuleReg
    main.o(i.DMA_Init) refers to mg32x02z_csc_drv.o(i.CSC_PeriphOnModeClock_Config) for CSC_PeriphOnModeClock_Config
    main.o(i.DMA_Init) refers to mg32x02z__common_drv.o(i.ProtectModuleReg) for ProtectModuleReg
    main.o(i.DMA_Init) refers to mg32x02z_dma_drv.o(i.DMA_Cmd) for DMA_Cmd
    main.o(i.DMA_Init) refers to mg32x02z_dma_drv.o(i.DMA_Channel_Cmd) for DMA_Channel_Cmd
    main.o(i.DMA_Init) refers to mg32x02z_dma_drv.o(i.DMA_BaseInitStructure_Init) for DMA_BaseInitStructure_Init
    main.o(i.DMA_Init) refers to mg32x02z_dma_drv.o(i.DMA_Base_Init) for DMA_Base_Init
    main.o(i.DMA_Init) refers to main.o(.data) for DataPattern
    main.o(i.GPL_CRC_Check) refers to mg32x02z__common_drv.o(i.UnProtectModuleReg) for UnProtectModuleReg
    main.o(i.GPL_CRC_Check) refers to mg32x02z_csc_drv.o(i.CSC_PeriphOnModeClock_Config) for CSC_PeriphOnModeClock_Config
    main.o(i.GPL_CRC_Check) refers to mg32x02z__common_drv.o(i.ProtectModuleReg) for ProtectModuleReg
    main.o(i.GPL_CRC_Check) refers to main.o(i.GPL_CRC_Config) for GPL_CRC_Config
    main.o(i.GPL_CRC_Check) refers to mg32x02z_gpl_drv.o(i.GPL_DMA_Cmd) for GPL_DMA_Cmd
    main.o(i.GPL_CRC_Check) refers to mg32x02z_dma_drv.o(i.DMA_GetSingleFlagStatus) for DMA_GetSingleFlagStatus
    main.o(i.GPL_CRC_Check) refers to mg32x02z_dma_drv.o(i.DMA_ClearFlag) for DMA_ClearFlag
    main.o(i.GPL_CRC_Check) refers to printf8.o(i.__0printf$8) for __2printf
    main.o(i.GPL_CRC_Check) refers to main.o(.conststring) for .conststring
    main.o(i.Sample_URT0_Init) refers to mg32x02z__common_drv.o(i.UnProtectModuleReg) for UnProtectModuleReg
    main.o(i.Sample_URT0_Init) refers to mg32x02z_csc_drv.o(i.CSC_PeriphProcessClockSource_Config) for CSC_PeriphProcessClockSource_Config
    main.o(i.Sample_URT0_Init) refers to mg32x02z_csc_drv.o(i.CSC_PeriphOnModeClock_Config) for CSC_PeriphOnModeClock_Config
    main.o(i.Sample_URT0_Init) refers to mg32x02z__common_drv.o(i.ProtectModuleReg) for ProtectModuleReg
    main.o(i.Sample_URT0_Init) refers to mg32x02z_gpio_drv.o(i.GPIO_PinMode_Config) for GPIO_PinMode_Config
    main.o(i.Sample_URT0_Init) refers to mg32x02z_urt_drv.o(i.URT_BaudRateGenerator_Config) for URT_BaudRateGenerator_Config
    main.o(i.Sample_URT0_Init) refers to mg32x02z_urt_drv.o(i.URT_BaudRateGenerator_Cmd) for URT_BaudRateGenerator_Cmd
    main.o(i.Sample_URT0_Init) refers to mg32x02z_urt_drv.o(i.URT_TXClockSource_Select) for URT_TXClockSource_Select
    main.o(i.Sample_URT0_Init) refers to mg32x02z_urt_drv.o(i.URT_RXClockSource_Select) for URT_RXClockSource_Select
    main.o(i.Sample_URT0_Init) refers to mg32x02z_urt_drv.o(i.URT_TXOverSamplingSampleNumber_Select) for URT_TXOverSamplingSampleNumber_Select
    main.o(i.Sample_URT0_Init) refers to mg32x02z_urt_drv.o(i.URT_RXOverSamplingSampleNumber_Select) for URT_RXOverSamplingSampleNumber_Select
    main.o(i.Sample_URT0_Init) refers to mg32x02z_urt_drv.o(i.URT_RXOverSamplingMode_Select) for URT_RXOverSamplingMode_Select
    main.o(i.Sample_URT0_Init) refers to mg32x02z_urt_drv.o(i.URT_TX_Cmd) for URT_TX_Cmd
    main.o(i.Sample_URT0_Init) refers to mg32x02z_urt_drv.o(i.URT_RX_Cmd) for URT_RX_Cmd
    main.o(i.Sample_URT0_Init) refers to mg32x02z_urt_drv.o(i.URT_DataCharacter_Config) for URT_DataCharacter_Config
    main.o(i.Sample_URT0_Init) refers to mg32x02z_urt_drv.o(i.URT_Mode_Select) for URT_Mode_Select
    main.o(i.Sample_URT0_Init) refers to mg32x02z_urt_drv.o(i.URT_DataLine_Select) for URT_DataLine_Select
    main.o(i.Sample_URT0_Init) refers to mg32x02z_urt_drv.o(i.URT_RXShadowBufferThreshold_Select) for URT_RXShadowBufferThreshold_Select
    main.o(i.Sample_URT0_Init) refers to mg32x02z_urt_drv.o(i.URT_IdlehandleMode_Select) for URT_IdlehandleMode_Select
    main.o(i.Sample_URT0_Init) refers to mg32x02z_urt_drv.o(i.URT_TXGaudTime_Select) for URT_TXGaudTime_Select
    main.o(i.Sample_URT0_Init) refers to mg32x02z_urt_drv.o(i.URT_IT_Cmd) for URT_IT_Cmd
    main.o(i.Sample_URT0_Init) refers to mg32x02z_urt_drv.o(i.URT_ITEA_Cmd) for URT_ITEA_Cmd
    main.o(i.Sample_URT0_Init) refers to mg32x02z_urt_drv.o(i.URT_Cmd) for URT_Cmd
    main.o(i.UartSendByte) refers to mg32x02z_urt_drv.o(i.URT_SetTXData) for URT_SetTXData
    main.o(i.UartSendByte) refers to mg32x02z_urt_drv.o(i.URT_GetITSingleFlagStatus) for URT_GetITSingleFlagStatus
    main.o(i.UartSendByte) refers to mg32x02z_urt_drv.o(i.URT_ClearITFlag) for URT_ClearITFlag
    main.o(i.fputc) refers to mg32x02z_urt_drv.o(i.URT_SetTXData) for URT_SetTXData
    main.o(i.fputc) refers to mg32x02z_urt_drv.o(i.URT_GetITSingleFlagStatus) for URT_GetITSingleFlagStatus
    main.o(i.fputc) refers to mg32x02z_urt_drv.o(i.URT_ClearITFlag) for URT_ClearITFlag
    main.o(i.main) refers to main.o(i.CSC_Init) for CSC_Init
    main.o(i.main) refers to main.o(i.Sample_URT0_Init) for Sample_URT0_Init
    main.o(i.main) refers to printf8.o(i.__0printf$8) for __2printf
    main.o(i.main) refers to main.o(i.DMA_Init) for DMA_Init
    main.o(i.main) refers to mg32x02z_dma_drv.o(i.DMA_ClearFlag) for DMA_ClearFlag
    main.o(i.main) refers to mg32x02z_dma_drv.o(i.DMA_StartRequest) for DMA_StartRequest
    main.o(i.main) refers to main.o(i.GPL_CRC_Check) for GPL_CRC_Check
    mg32x02z__common_drv.o(i.Delay) refers to mg32x02z__common_drv.o(i.GetTick) for GetTick
    mg32x02z__common_drv.o(i.GetTick) refers to mg32x02z__common_drv.o(.data) for uwTick
    mg32x02z__common_drv.o(i.IncTick) refers to mg32x02z__common_drv.o(.data) for uwTick
    mg32x02z__common_drv.o(i.InitTick) refers to uidiv.o(.text) for __aeabi_uidivmod
    mg32x02z__common_drv.o(i.InitTick) refers to mg32x02z__common_drv.o(i.__NVIC_SetPriority) for __NVIC_SetPriority
    mg32x02z_csc_drv.o(i.CSC_XOSC_Cmd) refers to mg32x02z_gpio_drv.o(i.GPIO_PinFunction_Select) for GPIO_PinFunction_Select
    mg32x02z_mem_drv.o(i.MEM_Access_Cmd) refers to mg32x02z__common_drv.o(i.UnProtectModuleReg) for UnProtectModuleReg
    mg32x02z_mem_drv.o(i.MEM_Access_Cmd) refers to mg32x02z__common_drv.o(i.ProtectModuleReg) for ProtectModuleReg
    mg32x02z_mem_drv.o(i.MEM_Cmd) refers to mg32x02z__common_drv.o(i.UnProtectModuleReg) for UnProtectModuleReg
    mg32x02z_mem_drv.o(i.MEM_Cmd) refers to mg32x02z__common_drv.o(i.ProtectModuleReg) for ProtectModuleReg
    mg32x02z_mem_drv.o(i.MEM_ErrorHardFault_Cmd) refers to mg32x02z__common_drv.o(i.UnProtectModuleReg) for UnProtectModuleReg
    mg32x02z_mem_drv.o(i.MEM_ErrorHardFault_Cmd) refers to mg32x02z__common_drv.o(i.ProtectModuleReg) for ProtectModuleReg
    mg32x02z_mem_drv.o(i.MEM_ErrorReset_Cmd) refers to mg32x02z__common_drv.o(i.UnProtectModuleReg) for UnProtectModuleReg
    mg32x02z_mem_drv.o(i.MEM_ErrorReset_Cmd) refers to mg32x02z__common_drv.o(i.ProtectModuleReg) for ProtectModuleReg
    mg32x02z_mem_drv.o(i.MEM_ITEA_Cmd) refers to mg32x02z__common_drv.o(i.UnProtectModuleReg) for UnProtectModuleReg
    mg32x02z_mem_drv.o(i.MEM_ITEA_Cmd) refers to mg32x02z__common_drv.o(i.ProtectModuleReg) for ProtectModuleReg
    mg32x02z_mem_drv.o(i.MEM_IT_Cmd) refers to mg32x02z__common_drv.o(i.UnProtectModuleReg) for UnProtectModuleReg
    mg32x02z_mem_drv.o(i.MEM_IT_Cmd) refers to mg32x02z__common_drv.o(i.ProtectModuleReg) for ProtectModuleReg
    mg32x02z_mem_drv.o(i.MEM_SetFlashWaitState) refers to mg32x02z__common_drv.o(i.UnProtectModuleReg) for UnProtectModuleReg
    mg32x02z_mem_drv.o(i.MEM_SetFlashWaitState) refers to mg32x02z__common_drv.o(i.ProtectModuleReg) for ProtectModuleReg
    mg32x02z_mem_drv.o(i.MEM_SetIAPSize) refers to mg32x02z_mem_drv.o(i.MEM_ClearFlag) for MEM_ClearFlag
    mg32x02z_mem_drv.o(i.MEM_SetIAPSize) refers to mg32x02z__common_drv.o(i.UnProtectModuleReg) for UnProtectModuleReg
    mg32x02z_mem_drv.o(i.MEM_SetIAPSize) refers to mg32x02z__common_drv.o(i.ProtectModuleReg) for ProtectModuleReg
    mg32x02z_mem_drv.o(i.MEM_SetIAPSize) refers to mg32x02z_mem_drv.o(i.MEM_GetFlagStatus) for MEM_GetFlagStatus
    mg32x02z_mem_drv.o(i.MEM_SetIAPSize) refers to mg32x02z_mem_drv.o(i.MEM_GetIAPSize) for MEM_GetIAPSize
    mg32x02z_mem_drv.o(i.MEM_SetIAPSizeLock) refers to mg32x02z__common_drv.o(i.UnProtectModuleReg) for UnProtectModuleReg
    mg32x02z_mem_drv.o(i.MEM_SetIAPSizeLock) refers to mg32x02z__common_drv.o(i.ProtectModuleReg) for ProtectModuleReg
    mg32x02z_mem_drv.o(i.MEM_SetWriteMode) refers to mg32x02z__common_drv.o(i.UnProtectModuleReg) for UnProtectModuleReg
    mg32x02z_mem_drv.o(i.MEM_SetWriteMode) refers to mg32x02z__common_drv.o(i.ProtectModuleReg) for ProtectModuleReg
    mg32x02z_mem_drv.o(i.MEM_WriteFlashHold_Cmd) refers to mg32x02z__common_drv.o(i.UnProtectModuleReg) for UnProtectModuleReg
    mg32x02z_mem_drv.o(i.MEM_WriteFlashHold_Cmd) refers to mg32x02z__common_drv.o(i.ProtectModuleReg) for ProtectModuleReg
    mg32x02z_dma_drv.o(i.DMA_Base_Init) refers to mg32x02z_dma_drv.o(i.DMA_SetExtTriggerPin) for DMA_SetExtTriggerPin
    mg32x02z_dma_drv.o(i.DMA_Base_Init) refers to mg32x02z_dma_drv.o(i.DMA_SetExtTriggerMode) for DMA_SetExtTriggerMode
    mg32x02z_dma_drv.o(i.DMA_Base_Init) refers to mg32x02z_dma_drv.o(i.DMA_LoopMode_Cmd) for DMA_LoopMode_Cmd
    mg32x02z_dma_drv.o(i.DMA_Base_Init) refers to mg32x02z_dma_drv.o(i.DMA_AutoIncreaseSourceAddress) for DMA_AutoIncreaseSourceAddress
    mg32x02z_dma_drv.o(i.DMA_Base_Init) refers to mg32x02z_dma_drv.o(i.DMA_AutoIncreaseDestinationAddress) for DMA_AutoIncreaseDestinationAddress
    mg32x02z_dma_drv.o(i.DMA_Base_Init) refers to mg32x02z_dma_drv.o(i.DMA_Source_Select) for DMA_Source_Select
    mg32x02z_dma_drv.o(i.DMA_Base_Init) refers to mg32x02z_dma_drv.o(i.DMA_Destination_Select) for DMA_Destination_Select
    mg32x02z_dma_drv.o(i.DMA_Base_Init) refers to mg32x02z_dma_drv.o(i.DMA_SetBurstSize) for DMA_SetBurstSize
    mg32x02z_dma_drv.o(i.DMA_Base_Init) refers to mg32x02z_dma_drv.o(i.DMA_SetTransferDataNumber) for DMA_SetTransferDataNumber
    mg32x02z_dma_drv.o(i.DMA_Base_Init) refers to mg32x02z_dma_drv.o(i.DMA_SetSourceAddress) for DMA_SetSourceAddress
    mg32x02z_dma_drv.o(i.DMA_Base_Init) refers to mg32x02z_dma_drv.o(i.DMA_SetDestinationAddress) for DMA_SetDestinationAddress
    mg32x02z_adc_drv.o(i.ADC_Base_Init) refers to mg32x02z_adc_drv.o(i.ADC_ClockSource_Select) for ADC_ClockSource_Select
    mg32x02z_adc_drv.o(i.ADC_Base_Init) refers to mg32x02z_adc_drv.o(i.ADC_SetInternalClockDivider) for ADC_SetInternalClockDivider
    mg32x02z_adc_drv.o(i.ADC_Base_Init) refers to mg32x02z_adc_drv.o(i.ADC_SetPLLClockDivider) for ADC_SetPLLClockDivider
    mg32x02z_adc_drv.o(i.ADC_Base_Init) refers to mg32x02z_adc_drv.o(i.ADC_DataAlignment_Select) for ADC_DataAlignment_Select
    mg32x02z_adc_drv.o(i.ADC_Base_Init) refers to mg32x02z_adc_drv.o(i.ADC_DataResolution_Select) for ADC_DataResolution_Select
    mg32x02z_adc_drv.o(i.ADC_Base_Init) refers to mg32x02z_adc_drv.o(i.ADC_DataOverrunMode_Select) for ADC_DataOverrunMode_Select
    mg32x02z_adc_drv.o(i.ADC_ConversionMode_Select) refers to mg32x02z_adc_drv.o(i.__ARM_common_switch8) for __ARM_common_switch8
    mg32x02z_adc_drv.o(i.ADC_ConversionMode_Select) refers to mg32x02z_adc_drv.o(i.ADC_MainConversionMode_Select) for ADC_MainConversionMode_Select
    mg32x02z_adc_drv.o(i.ADC_ConversionMode_Select) refers to mg32x02z_adc_drv.o(i.ADC_ContinueMode_Cmd) for ADC_ContinueMode_Cmd
    mg32x02z_adc_drv.o(i.ADC_PGAOffsetCalibration_Cmd) refers to mg32x02z_adc_drv.o(i.ADC_SetPGAOffset) for ADC_SetPGAOffset
    mg32x02z_adc_drv.o(i.ADC_PGAOffsetCalibration_Cmd) refers to mg32x02z_adc_drv.o(i.ADC_PGA_Cmd) for ADC_PGA_Cmd
    mg32x02z_adc_drv.o(i.ADC_StartCalibration) refers to mg32x02z_adc_drv.o(i.ADC_ConversionMode_Select) for ADC_ConversionMode_Select
    mg32x02z_adc_drv.o(i.ADC_StartCalibration) refers to mg32x02z_adc_drv.o(i.ADC_TriggerSource_Select) for ADC_TriggerSource_Select
    mg32x02z_adc_drv.o(i.ADC_StartCalibration) refers to mg32x02z_adc_drv.o(i.ADC_SingleDifferentMode_Select) for ADC_SingleDifferentMode_Select
    mg32x02z_adc_drv.o(i.ADC_StartCalibration) refers to mg32x02z_adc_drv.o(i.ADC_SetOutputCodeFormat) for ADC_SetOutputCodeFormat
    mg32x02z_adc_drv.o(i.ADC_StartCalibration) refers to mg32x02z_adc_drv.o(i.ADC_DataResolution_Select) for ADC_DataResolution_Select
    mg32x02z_adc_drv.o(i.ADC_StartCalibration) refers to mg32x02z__common_drv.o(i.UnProtectModuleReg) for UnProtectModuleReg
    mg32x02z_adc_drv.o(i.ADC_StartCalibration) refers to mg32x02z_cfg_drv.o(i.CFG_SetADC0RefTop) for CFG_SetADC0RefTop
    mg32x02z_adc_drv.o(i.ADC_StartCalibration) refers to mg32x02z_cfg_drv.o(i.CFG_SetADC0RefMiddle) for CFG_SetADC0RefMiddle
    mg32x02z_adc_drv.o(i.ADC_StartCalibration) refers to mg32x02z_cfg_drv.o(i.CFG_SetADC0RefBottom) for CFG_SetADC0RefBottom
    mg32x02z_adc_drv.o(i.ADC_StartCalibration) refers to mg32x02z_adc_drv.o(i.ADC_ChannelMUX_Select) for ADC_ChannelMUX_Select
    mg32x02z_adc_drv.o(i.ADC_StartCalibration) refers to mg32x02z_adc_drv.o(i.ADC_InternalChannel_Select) for ADC_InternalChannel_Select
    mg32x02z_adc_drv.o(i.ADC_StartCalibration) refers to mg32x02z_adc_drv.o(i.ADC_SoftwareConversion_Cmd) for ADC_SoftwareConversion_Cmd
    mg32x02z_adc_drv.o(i.ADC_StartCalibration) refers to mg32x02z_adc_drv.o(i.ADC_GetSingleFlagStatus) for ADC_GetSingleFlagStatus
    mg32x02z_adc_drv.o(i.ADC_StartCalibration) refers to mg32x02z_adc_drv.o(i.ADC_ClearFlag) for ADC_ClearFlag
    mg32x02z_adc_drv.o(i.ADC_StartCalibration) refers to mg32x02z_adc_drv.o(i.ADC_GetDAT0Data) for ADC_GetDAT0Data
    mg32x02z_adc_drv.o(i.ADC_StartCalibration) refers to idiv.o(.text) for __aeabi_idivmod
    mg32x02z_adc_drv.o(i.ADC_StartCalibration) refers to mg32x02z_cfg_drv.o(i.CFG_GetADC0RefTop) for CFG_GetADC0RefTop
    mg32x02z_adc_drv.o(i.ADC_StartCalibration) refers to mg32x02z_cfg_drv.o(i.CFG_GetADC0RefBottom) for CFG_GetADC0RefBottom
    mg32x02z_adc_drv.o(i.ADC_StartCalibration) refers to mg32x02z_adc_drv.o(i.ADC_VRMCalibration) for ADC_VRMCalibration
    mg32x02z_adc_drv.o(i.ADC_StartCalibration) refers to mg32x02z__common_drv.o(i.ProtectModuleReg) for ProtectModuleReg
    mg32x02z_adc_drv.o(i.ADC_VRMCalibration) refers to mg32x02z__common_drv.o(i.UnProtectModuleReg) for UnProtectModuleReg
    mg32x02z_adc_drv.o(i.ADC_VRMCalibration) refers to mg32x02z_adc_drv.o(i.ADC_InternalChannel_Select) for ADC_InternalChannel_Select
    mg32x02z_adc_drv.o(i.ADC_VRMCalibration) refers to mg32x02z_adc_drv.o(i.ADC_SoftwareConversion_Cmd) for ADC_SoftwareConversion_Cmd
    mg32x02z_adc_drv.o(i.ADC_VRMCalibration) refers to mg32x02z_adc_drv.o(i.ADC_GetSingleFlagStatus) for ADC_GetSingleFlagStatus
    mg32x02z_adc_drv.o(i.ADC_VRMCalibration) refers to mg32x02z_adc_drv.o(i.ADC_ClearFlag) for ADC_ClearFlag
    mg32x02z_adc_drv.o(i.ADC_VRMCalibration) refers to mg32x02z_adc_drv.o(i.ADC_GetDAT0Data) for ADC_GetDAT0Data
    mg32x02z_adc_drv.o(i.ADC_VRMCalibration) refers to idiv.o(.text) for __aeabi_idivmod
    mg32x02z_adc_drv.o(i.ADC_VRMCalibration) refers to mg32x02z_cfg_drv.o(i.CFG_SetADC0RefMiddle) for CFG_SetADC0RefMiddle
    mg32x02z_tm_drv.o(i.TM_TimeBase_Init) refers to mg32x02z_tm_drv.o(i.TM_Prescaler_Config) for TM_Prescaler_Config
    mg32x02z_tm_drv.o(i.TM_TimeBase_Init) refers to mg32x02z_tm_drv.o(i.TM_Counter_Config) for TM_Counter_Config
    mg32x02z_tm_drv.o(i.TM_TimeBase_Init) refers to mg32x02z_tm_drv.o(i.TM_TimerMode_Select) for TM_TimerMode_Select
    mg32x02z_tm_drv.o(i.TM_TimeBase_Init) refers to mg32x02z_tm_drv.o(i.TM_CounterClock_Select) for TM_CounterClock_Select
    mg32x02z_tm_drv.o(i.TM_TimeBase_Init) refers to mg32x02z_tm_drv.o(i.TM_PrescalerClock_Select) for TM_PrescalerClock_Select
    mg32x02z_tm_drv.o(i.TM_TimeBase_Init) refers to mg32x02z_tm_drv.o(i.TM_SetInternalClockDivider) for TM_SetInternalClockDivider
    mg32x02z_tm_drv.o(i.TM_TimeBase_Init) refers to mg32x02z_tm_drv.o(i.TM_SetCounterDirection) for TM_SetCounterDirection
    mg32x02z_tm_drv.o(i.TM_TimeBase_Init) refers to mg32x02z_tm_drv.o(i.TM_SetPrescalerDirection) for TM_SetPrescalerDirection
    mg32x02z_wwdt_irq.o(i.WWDT_IRQ) refers to mg32x02z_wwdt_drv.o(i.WWDT_GetSingleFlagStatus) for WWDT_GetSingleFlagStatus
    mg32x02z_wwdt_irq.o(i.WWDT_IRQ) refers to mg32x02z_wwdt_drv.o(i.WWDT_ClearFlag) for WWDT_ClearFlag
    mg32x02z_iwdt_irq.o(i.IWDT_IRQ) refers to mg32x02z_iwdt_drv.o(i.IWDT_GetSingleFlagStatus) for IWDT_GetSingleFlagStatus
    mg32x02z_iwdt_irq.o(i.IWDT_IRQ) refers to mg32x02z_iwdt_drv.o(i.IWDT_ClearFlag) for IWDT_ClearFlag
    mg32x02z_iwdt_irq.o(i.IWDT_IRQ) refers to mg32x02z_iwdt_drv.o(i.IWDT_RefreshCounter) for IWDT_RefreshCounter
    mg32x02z_iwdt_irq.o(i.IWDT_IRQ) refers to mg32x02z_iwdt_drv.o(i.IWDT_GetAllFlagStatus) for IWDT_GetAllFlagStatus
    mg32x02z_pw_irq.o(i.PW_IRQ) refers to mg32x02z_pw_drv.o(i.PW_GetSingleFlagStatus) for PW_GetSingleFlagStatus
    mg32x02z_pw_irq.o(i.PW_IRQ) refers to mg32x02z_pw_drv.o(i.PW_ClearFlag) for PW_ClearFlag
    mg32x02z_pw_irq.o(i.PW_IRQ) refers to mg32x02z_pw_drv.o(i.PW_GetAllFlagStatus) for PW_GetAllFlagStatus
    mg32x02z_rtc_irq.o(i.RTC_IRQ) refers to mg32x02z_rtc_drv.o(i.RTC_GetSingleFlagStatus) for RTC_GetSingleFlagStatus
    mg32x02z_rtc_irq.o(i.RTC_IRQ) refers to mg32x02z_rtc_drv.o(i.RTC_ClearFlag) for RTC_ClearFlag
    mg32x02z_csc_irq.o(i.CSC_IRQ) refers to mg32x02z_csc_drv.o(i.CSC_GetSingleFlagStatus) for CSC_GetSingleFlagStatus
    mg32x02z_csc_irq.o(i.CSC_IRQ) refers to mg32x02z_csc_drv.o(i.CSC_ClearFlag) for CSC_ClearFlag
    mg32x02z_csc_irq.o(i.CSC_IRQ) refers to mg32x02z_csc_drv.o(i.CSC_GetAllFlagStatus) for CSC_GetAllFlagStatus
    mg32x02z_apb_irq.o(i.APB_IRQ) refers to mg32x02z_apb_drv.o(i.APB_GetSingleFlagStatus) for APB_GetSingleFlagStatus
    mg32x02z_apb_irq.o(i.APB_IRQ) refers to mg32x02z_apb_drv.o(i.APB_ClearFlag) for APB_ClearFlag
    mg32x02z_exic_irq.o(i.EXINT0_IRQ) refers to mg32x02z_exic_drv.o(i.EXIC_GetPxTriggerAndITFlagStatus) for EXIC_GetPxTriggerAndITFlagStatus
    mg32x02z_exic_irq.o(i.EXINT0_IRQ) refers to mg32x02z_exic_drv.o(i.EXIC_ClearPxTriggerITFlag) for EXIC_ClearPxTriggerITFlag
    mg32x02z_exic_irq.o(i.EXINT0_IRQ) refers to mg32x02z_exic_drv.o(i.EXIC_GetPxTriggerOrITFlagStatus) for EXIC_GetPxTriggerOrITFlagStatus
    mg32x02z_exic_irq.o(i.EXINT0_IRQ) refers to mg32x02z_exic_drv.o(i.EXIC_ClearPxTriggerEventFlag) for EXIC_ClearPxTriggerEventFlag
    mg32x02z_exic_irq.o(i.EXINT1_IRQ) refers to mg32x02z_exic_drv.o(i.EXIC_GetPxTriggerAndITFlagStatus) for EXIC_GetPxTriggerAndITFlagStatus
    mg32x02z_exic_irq.o(i.EXINT1_IRQ) refers to mg32x02z_exic_drv.o(i.EXIC_ClearPxTriggerITFlag) for EXIC_ClearPxTriggerITFlag
    mg32x02z_exic_irq.o(i.EXINT1_IRQ) refers to mg32x02z_exic_drv.o(i.EXIC_GetPxTriggerOrITFlagStatus) for EXIC_GetPxTriggerOrITFlagStatus
    mg32x02z_exic_irq.o(i.EXINT1_IRQ) refers to mg32x02z_exic_drv.o(i.EXIC_ClearPxTriggerEventFlag) for EXIC_ClearPxTriggerEventFlag
    mg32x02z_exic_irq.o(i.EXINT2_IRQ) refers to mg32x02z_exic_drv.o(i.EXIC_GetPxTriggerAndITFlagStatus) for EXIC_GetPxTriggerAndITFlagStatus
    mg32x02z_exic_irq.o(i.EXINT2_IRQ) refers to mg32x02z_exic_drv.o(i.EXIC_ClearPxTriggerITFlag) for EXIC_ClearPxTriggerITFlag
    mg32x02z_exic_irq.o(i.EXINT2_IRQ) refers to mg32x02z_exic_drv.o(i.EXIC_GetPxTriggerOrITFlagStatus) for EXIC_GetPxTriggerOrITFlagStatus
    mg32x02z_exic_irq.o(i.EXINT2_IRQ) refers to mg32x02z_exic_drv.o(i.EXIC_ClearPxTriggerEventFlag) for EXIC_ClearPxTriggerEventFlag
    mg32x02z_exic_irq.o(i.EXINT3_IRQ) refers to mg32x02z_exic_drv.o(i.EXIC_GetPxTriggerAndITFlagStatus) for EXIC_GetPxTriggerAndITFlagStatus
    mg32x02z_exic_irq.o(i.EXINT3_IRQ) refers to mg32x02z_exic_drv.o(i.EXIC_ClearPxTriggerITFlag) for EXIC_ClearPxTriggerITFlag
    mg32x02z_exic_irq.o(i.EXINT3_IRQ) refers to mg32x02z_exic_drv.o(i.EXIC_GetPxTriggerOrITFlagStatus) for EXIC_GetPxTriggerOrITFlagStatus
    mg32x02z_exic_irq.o(i.EXINT3_IRQ) refers to mg32x02z_exic_drv.o(i.EXIC_ClearPxTriggerEventFlag) for EXIC_ClearPxTriggerEventFlag
    mg32x02z_cmp_irq.o(i.CMP_IRQ) refers to mg32x02z_cmp_drv.o(i.CMP_GetSingleFlagStatus) for CMP_GetSingleFlagStatus
    mg32x02z_cmp_irq.o(i.CMP_IRQ) refers to mg32x02z_cmp_drv.o(i.CMP_ClearFlag) for CMP_ClearFlag
    mg32x02z_dma_irq.o(i.DMA_IRQ) refers to mg32x02z_dma_drv.o(i.DMA_GetSingleFlagStatus) for DMA_GetSingleFlagStatus
    mg32x02z_dma_irq.o(i.DMA_IRQ) refers to mg32x02z_dma_drv.o(i.DMA_ClearFlag) for DMA_ClearFlag
    mg32x02z_adc_irq.o(i.ADC_IRQ) refers to mg32x02z_adc_drv.o(i.ADC_GetSingleFlagStatus) for ADC_GetSingleFlagStatus
    mg32x02z_adc_irq.o(i.ADC_IRQ) refers to mg32x02z_adc_drv.o(i.ADC_ClearFlag) for ADC_ClearFlag
    mg32x02z_adc_irq.o(i.ADC_IRQ) refers to mg32x02z_adc_drv.o(i.ADC_ClearSum0Flags) for ADC_ClearSum0Flags
    mg32x02z_adc_irq.o(i.ADC_IRQ) refers to mg32x02z_adc_drv.o(i.ADC_ClearSum1Flags) for ADC_ClearSum1Flags
    mg32x02z_adc_irq.o(i.ADC_IRQ) refers to mg32x02z_adc_drv.o(i.ADC_ClearSum2Flags) for ADC_ClearSum2Flags
    mg32x02z_dac_irq.o(i.DAC_IRQ) refers to mg32x02z_dac_drv.o(i.DAC_GetAllFlagStatus) for DAC_GetAllFlagStatus
    mg32x02z_dac_irq.o(i.DAC_IRQ) refers to mg32x02z_dac_drv.o(i.DAC_ClearFlag) for DAC_ClearFlag
    mg32x02z_tm00_irq.o(i.TM00_IRQ) refers to mg32x02z_tm_drv.o(i.TM_GetSingleFlagStatus) for TM_GetSingleFlagStatus
    mg32x02z_tm00_irq.o(i.TM00_IRQ) refers to mg32x02z_tm_drv.o(i.TM_ClearFlag) for TM_ClearFlag
    mg32x02z_tm01_irq.o(i.TM01_IRQ) refers to mg32x02z_tm_drv.o(i.TM_GetSingleFlagStatus) for TM_GetSingleFlagStatus
    mg32x02z_tm01_irq.o(i.TM01_IRQ) refers to mg32x02z_tm_drv.o(i.TM_ClearFlag) for TM_ClearFlag
    mg32x02z_tm10_irq.o(i.TM10_IRQ) refers to mg32x02z_tm_drv.o(i.TM_GetSingleFlagStatus) for TM_GetSingleFlagStatus
    mg32x02z_tm10_irq.o(i.TM10_IRQ) refers to mg32x02z_tm_drv.o(i.TM_ClearFlag) for TM_ClearFlag
    mg32x02z_tm16_irq.o(i.TM16_IRQ) refers to mg32x02z_tm_drv.o(i.TM_GetSingleFlagStatus) for TM_GetSingleFlagStatus
    mg32x02z_tm16_irq.o(i.TM16_IRQ) refers to mg32x02z_tm_drv.o(i.TM_ClearFlag) for TM_ClearFlag
    mg32x02z_tm20_irq.o(i.TM20_IRQ) refers to mg32x02z_tm_drv.o(i.TM_GetSingleFlagStatus) for TM_GetSingleFlagStatus
    mg32x02z_tm20_irq.o(i.TM20_IRQ) refers to mg32x02z_tm_drv.o(i.TM_ClearFlag) for TM_ClearFlag
    mg32x02z_tm26_irq.o(i.TM26_IRQ) refers to mg32x02z_tm_drv.o(i.TM_GetSingleFlagStatus) for TM_GetSingleFlagStatus
    mg32x02z_tm26_irq.o(i.TM26_IRQ) refers to mg32x02z_tm_drv.o(i.TM_ClearFlag) for TM_ClearFlag
    mg32x02z_tm36_irq.o(i.TM36_IRQ) refers to mg32x02z_tm_drv.o(i.TM_GetSingleFlagStatus) for TM_GetSingleFlagStatus
    mg32x02z_tm36_irq.o(i.TM36_IRQ) refers to mg32x02z_tm_drv.o(i.TM_ClearFlag) for TM_ClearFlag
    mg32x02z_urt0_irq.o(i.URT0_IRQ) refers to mg32x02z_urt_drv.o(i.URT_GetITAllFlagStatus) for URT_GetITAllFlagStatus
    mg32x02z_urt0_irq.o(i.URT0_IRQ) refers to mg32x02z_urt_drv.o(i.URT_GetITStatus) for URT_GetITStatus
    mg32x02z_urt0_irq.o(i.URT0_IRQ) refers to mg32x02z_urt_drv.o(i.URT_ClearITFlag) for URT_ClearITFlag
    mg32x02z_urt0_irq.o(i.URT0_IRQ) refers to mg32x02z_urt_drv.o(i.URT_GetRXData) for URT_GetRXData
    mg32x02z_urt0_irq.o(i.URT0_IRQ) refers to mg32x02z_urt_drv.o(i.URT_SetTXData) for URT_SetTXData
    mg32x02z_urt1_irq.o(i.URT1_IRQ) refers to mg32x02z_urt_drv.o(i.URT_GetITAllFlagStatus) for URT_GetITAllFlagStatus
    mg32x02z_urt1_irq.o(i.URT1_IRQ) refers to mg32x02z_urt_drv.o(i.URT_GetITStatus) for URT_GetITStatus
    mg32x02z_urt1_irq.o(i.URT1_IRQ) refers to mg32x02z_urt_drv.o(i.URT_ClearITFlag) for URT_ClearITFlag
    mg32x02z_urt1_irq.o(i.URT1_IRQ) refers to mg32x02z_urt_drv.o(i.URT_GetRXData) for URT_GetRXData
    mg32x02z_urt1_irq.o(i.URT1_IRQ) refers to mg32x02z_urt_drv.o(i.URT_SetTXData) for URT_SetTXData
    mg32x02z_urt2_irq.o(i.URT2_IRQ) refers to mg32x02z_urt_drv.o(i.URT_GetITAllFlagStatus) for URT_GetITAllFlagStatus
    mg32x02z_urt2_irq.o(i.URT2_IRQ) refers to mg32x02z_urt_drv.o(i.URT_GetITStatus) for URT_GetITStatus
    mg32x02z_urt2_irq.o(i.URT2_IRQ) refers to mg32x02z_urt_drv.o(i.URT_ClearITFlag) for URT_ClearITFlag
    mg32x02z_urt2_irq.o(i.URT2_IRQ) refers to mg32x02z_urt_drv.o(i.URT_GetRXData) for URT_GetRXData
    mg32x02z_urt2_irq.o(i.URT2_IRQ) refers to mg32x02z_urt_drv.o(i.URT_SetTXData) for URT_SetTXData
    mg32x02z_urt3_irq.o(i.URT3_IRQ) refers to mg32x02z_urt_drv.o(i.URT_GetITAllFlagStatus) for URT_GetITAllFlagStatus
    mg32x02z_urt3_irq.o(i.URT3_IRQ) refers to mg32x02z_urt_drv.o(i.URT_GetITStatus) for URT_GetITStatus
    mg32x02z_urt3_irq.o(i.URT3_IRQ) refers to mg32x02z_urt_drv.o(i.URT_ClearITFlag) for URT_ClearITFlag
    mg32x02z_urt3_irq.o(i.URT3_IRQ) refers to mg32x02z_urt_drv.o(i.URT_GetRXData) for URT_GetRXData
    mg32x02z_urt3_irq.o(i.URT3_IRQ) refers to mg32x02z_urt_drv.o(i.URT_SetTXData) for URT_SetTXData
    mg32x02z_spi_irq.o(i.SPI0_IRQ) refers to mg32x02z_spi_drv.o(i.SPI_GetSingleFlagStatus) for SPI_GetSingleFlagStatus
    mg32x02z_spi_irq.o(i.SPI0_IRQ) refers to mg32x02z_spi_drv.o(i.SPI_ClearFlag) for SPI_ClearFlag
    mg32x02z_spi_irq.o(i.SPI0_IRQ) refers to mg32x02z_spi_drv.o(i.SPI_ClearRxData) for SPI_ClearRxData
    mg32x02z_spi_irq.o(i.SPI0_IRQ) refers to mg32x02z_spi_drv.o(i.SPI_SetTxData) for SPI_SetTxData
    mg32x02z_spi_irq.o(i.SPI0_IRQ) refers to mg32x02z_spi_drv.o(i.SPI_GetRxData) for SPI_GetRxData
    mg32x02z_spi_irq.o(i.SPI0_IRQ) refers to printf8.o(i.__0printf$8) for __2printf
    mg32x02z_i2c_irq.o(i.I2C0_IRQ) refers to mg32x02z_i2c_irq.o(i.I2C_WakeUp_Handler) for I2C_WakeUp_Handler
    mg32x02z_i2c_irq.o(i.I2C0_IRQ) refers to mg32x02z_i2c_irq.o(i.I2C_Timeout_Handler) for I2C_Timeout_Handler
    mg32x02z_i2c_irq.o(i.I2C0_IRQ) refers to mg32x02z_i2c_irq.o(i.I2C_ByteMode_Event_Handler) for I2C_ByteMode_Event_Handler
    mg32x02z_i2c_irq.o(i.I2C1_IRQ) refers to mg32x02z_i2c_irq.o(i.I2C_WakeUp_Handler) for I2C_WakeUp_Handler
    mg32x02z_i2c_irq.o(i.I2C1_IRQ) refers to mg32x02z_i2c_irq.o(i.I2C_Timeout_Handler) for I2C_Timeout_Handler
    mg32x02z_i2c_irq.o(i.I2C1_IRQ) refers to mg32x02z_i2c_irq.o(i.I2C_ByteMode_Event_Handler) for I2C_ByteMode_Event_Handler
    mg32x02z_i2c_irq.o(i.I2C_ByteMode_Event_Handler) refers to mg32x02z_i2c_drv.o(i.I2C_GetFlagStatus) for I2C_GetFlagStatus
    mg32x02z_i2c_irq.o(i.I2C_ByteMode_Event_Handler) refers to mg32x02z_i2c_drv.o(i.I2C_GetEventCode) for I2C_GetEventCode
    mg32x02z_i2c_irq.o(i.I2C_ByteMode_Event_Handler) refers to mg32x02z_adc_drv.o(i.__ARM_common_switch8) for __ARM_common_switch8
    mg32x02z_i2c_irq.o(i.I2C_ByteMode_Event_Handler) refers to mg32x02z_i2c_drv.o(i.I2C_ClearFlag) for I2C_ClearFlag
    mg32x02z_i2c_irq.o(i.I2C_Timeout_Handler) refers to mg32x02z_i2c_drv.o(i.I2C_GetFlagStatus) for I2C_GetFlagStatus
    mg32x02z_i2c_irq.o(i.I2C_Timeout_Handler) refers to mg32x02z_i2c_drv.o(i.I2C_ClearFlag) for I2C_ClearFlag
    startup_mg32x02z.o(RESET) refers to startup_mg32x02z.o(STACK) for __initial_sp
    startup_mg32x02z.o(RESET) refers to startup_mg32x02z.o(.text) for MG32x02z_IEC60730_MANAGER
    startup_mg32x02z.o(.text) refers to system_mg32x02z.o(i.SystemInit) for SystemInit
    startup_mg32x02z.o(.text) refers to entry.o(.ARM.Collect$$$$00000000) for __main
    system_mg32x02z.o(i.SystemCoreClockUpdate) refers to system_mg32x02z.o(.data) for SystemCoreClock
    system_mg32x02z.o(i.SystemInit) refers to system_mg32x02z.o(.data) for SystemCoreClock
    entry.o(.ARM.Collect$$$$00000000) refers (Special) to entry10a.o(.ARM.Collect$$$$0000000D) for __rt_final_cpp
    entry.o(.ARM.Collect$$$$00000000) refers (Special) to entry11a.o(.ARM.Collect$$$$0000000F) for __rt_final_exit
    entry.o(.ARM.Collect$$$$00000000) refers (Special) to entry7b.o(.ARM.Collect$$$$00000008) for _main_clock
    entry.o(.ARM.Collect$$$$00000000) refers (Special) to entry8b.o(.ARM.Collect$$$$0000000A) for _main_cpp_init
    entry.o(.ARM.Collect$$$$00000000) refers (Special) to entry9a.o(.ARM.Collect$$$$0000000B) for _main_init
    entry.o(.ARM.Collect$$$$00000000) refers (Special) to entry5.o(.ARM.Collect$$$$00000004) for _main_scatterload
    entry.o(.ARM.Collect$$$$00000000) refers (Special) to entry2.o(.ARM.Collect$$$$00000001) for _main_stk
    idiv.o(.text) refers to uidiv.o(.text) for __aeabi_uidivmod
    printfb.o(i.__0fprintf$bare) refers to printfb.o(i._printf_core) for _printf_core
    printfb.o(i.__0fprintf$bare) refers to main.o(i.fputc) for fputc
    printfb.o(i.__0printf$bare) refers to printfb.o(i._printf_core) for _printf_core
    printfb.o(i.__0printf$bare) refers to main.o(i.fputc) for fputc
    printfb.o(i.__0printf$bare) refers to stdout.o(.data) for __stdout
    printfb.o(i.__0snprintf$bare) refers to printfb.o(i._printf_core) for _printf_core
    printfb.o(i.__0snprintf$bare) refers to printfb.o(i._snputc) for _snputc
    printfb.o(i.__0sprintf$bare) refers to printfb.o(i._printf_core) for _printf_core
    printfb.o(i.__0sprintf$bare) refers to printfb.o(i._sputc) for _sputc
    printfb.o(i.__0vfprintf$bare) refers to printfb.o(i._printf_core) for _printf_core
    printfb.o(i.__0vfprintf$bare) refers to main.o(i.fputc) for fputc
    printfb.o(i.__0vprintf$bare) refers to printfb.o(i._printf_core) for _printf_core
    printfb.o(i.__0vprintf$bare) refers to main.o(i.fputc) for fputc
    printfb.o(i.__0vprintf$bare) refers to stdout.o(.data) for __stdout
    printfb.o(i.__0vsnprintf$bare) refers to printfb.o(i._printf_core) for _printf_core
    printfb.o(i.__0vsnprintf$bare) refers to printfb.o(i._snputc) for _snputc
    printfb.o(i.__0vsprintf$bare) refers to printfb.o(i._printf_core) for _printf_core
    printfb.o(i.__0vsprintf$bare) refers to printfb.o(i._sputc) for _sputc
    printf0.o(i.__0fprintf$0) refers to printf0.o(i._printf_core) for _printf_core
    printf0.o(i.__0fprintf$0) refers to main.o(i.fputc) for fputc
    printf0.o(i.__0printf$0) refers to printf0.o(i._printf_core) for _printf_core
    printf0.o(i.__0printf$0) refers to main.o(i.fputc) for fputc
    printf0.o(i.__0printf$0) refers to stdout.o(.data) for __stdout
    printf0.o(i.__0snprintf$0) refers to printf0.o(i._printf_core) for _printf_core
    printf0.o(i.__0snprintf$0) refers to printf0.o(i._snputc) for _snputc
    printf0.o(i.__0sprintf$0) refers to printf0.o(i._printf_core) for _printf_core
    printf0.o(i.__0sprintf$0) refers to printf0.o(i._sputc) for _sputc
    printf0.o(i.__0vfprintf$0) refers to printf0.o(i._printf_core) for _printf_core
    printf0.o(i.__0vfprintf$0) refers to main.o(i.fputc) for fputc
    printf0.o(i.__0vprintf$0) refers to printf0.o(i._printf_core) for _printf_core
    printf0.o(i.__0vprintf$0) refers to main.o(i.fputc) for fputc
    printf0.o(i.__0vprintf$0) refers to stdout.o(.data) for __stdout
    printf0.o(i.__0vsnprintf$0) refers to printf0.o(i._printf_core) for _printf_core
    printf0.o(i.__0vsnprintf$0) refers to printf0.o(i._snputc) for _snputc
    printf0.o(i.__0vsprintf$0) refers to printf0.o(i._printf_core) for _printf_core
    printf0.o(i.__0vsprintf$0) refers to printf0.o(i._sputc) for _sputc
    printf1.o(i.__0fprintf$1) refers to printf1.o(i._printf_core) for _printf_core
    printf1.o(i.__0fprintf$1) refers to main.o(i.fputc) for fputc
    printf1.o(i.__0printf$1) refers to printf1.o(i._printf_core) for _printf_core
    printf1.o(i.__0printf$1) refers to main.o(i.fputc) for fputc
    printf1.o(i.__0printf$1) refers to stdout.o(.data) for __stdout
    printf1.o(i.__0snprintf$1) refers to printf1.o(i._printf_core) for _printf_core
    printf1.o(i.__0snprintf$1) refers to printf1.o(i._snputc) for _snputc
    printf1.o(i.__0sprintf$1) refers to printf1.o(i._printf_core) for _printf_core
    printf1.o(i.__0sprintf$1) refers to printf1.o(i._sputc) for _sputc
    printf1.o(i.__0vfprintf$1) refers to printf1.o(i._printf_core) for _printf_core
    printf1.o(i.__0vfprintf$1) refers to main.o(i.fputc) for fputc
    printf1.o(i.__0vprintf$1) refers to printf1.o(i._printf_core) for _printf_core
    printf1.o(i.__0vprintf$1) refers to main.o(i.fputc) for fputc
    printf1.o(i.__0vprintf$1) refers to stdout.o(.data) for __stdout
    printf1.o(i.__0vsnprintf$1) refers to printf1.o(i._printf_core) for _printf_core
    printf1.o(i.__0vsnprintf$1) refers to printf1.o(i._snputc) for _snputc
    printf1.o(i.__0vsprintf$1) refers to printf1.o(i._printf_core) for _printf_core
    printf1.o(i.__0vsprintf$1) refers to printf1.o(i._sputc) for _sputc
    printf1.o(i._printf_core) refers to uidiv.o(.text) for __aeabi_uidivmod
    printf2.o(i.__0fprintf$2) refers to printf2.o(i._printf_core) for _printf_core
    printf2.o(i.__0fprintf$2) refers to main.o(i.fputc) for fputc
    printf2.o(i.__0printf$2) refers to printf2.o(i._printf_core) for _printf_core
    printf2.o(i.__0printf$2) refers to main.o(i.fputc) for fputc
    printf2.o(i.__0printf$2) refers to stdout.o(.data) for __stdout
    printf2.o(i.__0snprintf$2) refers to printf2.o(i._printf_core) for _printf_core
    printf2.o(i.__0snprintf$2) refers to printf2.o(i._snputc) for _snputc
    printf2.o(i.__0sprintf$2) refers to printf2.o(i._printf_core) for _printf_core
    printf2.o(i.__0sprintf$2) refers to printf2.o(i._sputc) for _sputc
    printf2.o(i.__0vfprintf$2) refers to printf2.o(i._printf_core) for _printf_core
    printf2.o(i.__0vfprintf$2) refers to main.o(i.fputc) for fputc
    printf2.o(i.__0vprintf$2) refers to printf2.o(i._printf_core) for _printf_core
    printf2.o(i.__0vprintf$2) refers to main.o(i.fputc) for fputc
    printf2.o(i.__0vprintf$2) refers to stdout.o(.data) for __stdout
    printf2.o(i.__0vsnprintf$2) refers to printf2.o(i._printf_core) for _printf_core
    printf2.o(i.__0vsnprintf$2) refers to printf2.o(i._snputc) for _snputc
    printf2.o(i.__0vsprintf$2) refers to printf2.o(i._printf_core) for _printf_core
    printf2.o(i.__0vsprintf$2) refers to printf2.o(i._sputc) for _sputc
    printf3.o(i.__0fprintf$3) refers to printf3.o(i._printf_core) for _printf_core
    printf3.o(i.__0fprintf$3) refers to main.o(i.fputc) for fputc
    printf3.o(i.__0printf$3) refers to printf3.o(i._printf_core) for _printf_core
    printf3.o(i.__0printf$3) refers to main.o(i.fputc) for fputc
    printf3.o(i.__0printf$3) refers to stdout.o(.data) for __stdout
    printf3.o(i.__0snprintf$3) refers to printf3.o(i._printf_core) for _printf_core
    printf3.o(i.__0snprintf$3) refers to printf3.o(i._snputc) for _snputc
    printf3.o(i.__0sprintf$3) refers to printf3.o(i._printf_core) for _printf_core
    printf3.o(i.__0sprintf$3) refers to printf3.o(i._sputc) for _sputc
    printf3.o(i.__0vfprintf$3) refers to printf3.o(i._printf_core) for _printf_core
    printf3.o(i.__0vfprintf$3) refers to main.o(i.fputc) for fputc
    printf3.o(i.__0vprintf$3) refers to printf3.o(i._printf_core) for _printf_core
    printf3.o(i.__0vprintf$3) refers to main.o(i.fputc) for fputc
    printf3.o(i.__0vprintf$3) refers to stdout.o(.data) for __stdout
    printf3.o(i.__0vsnprintf$3) refers to printf3.o(i._printf_core) for _printf_core
    printf3.o(i.__0vsnprintf$3) refers to printf3.o(i._snputc) for _snputc
    printf3.o(i.__0vsprintf$3) refers to printf3.o(i._printf_core) for _printf_core
    printf3.o(i.__0vsprintf$3) refers to printf3.o(i._sputc) for _sputc
    printf3.o(i._printf_core) refers to uidiv.o(.text) for __aeabi_uidivmod
    printf4.o(i.__0fprintf$4) refers to printf4.o(i._printf_core) for _printf_core
    printf4.o(i.__0fprintf$4) refers to main.o(i.fputc) for fputc
    printf4.o(i.__0printf$4) refers to printf4.o(i._printf_core) for _printf_core
    printf4.o(i.__0printf$4) refers to main.o(i.fputc) for fputc
    printf4.o(i.__0printf$4) refers to stdout.o(.data) for __stdout
    printf4.o(i.__0snprintf$4) refers to printf4.o(i._printf_core) for _printf_core
    printf4.o(i.__0snprintf$4) refers to printf4.o(i._snputc) for _snputc
    printf4.o(i.__0sprintf$4) refers to printf4.o(i._printf_core) for _printf_core
    printf4.o(i.__0sprintf$4) refers to printf4.o(i._sputc) for _sputc
    printf4.o(i.__0vfprintf$4) refers to printf4.o(i._printf_core) for _printf_core
    printf4.o(i.__0vfprintf$4) refers to main.o(i.fputc) for fputc
    printf4.o(i.__0vprintf$4) refers to printf4.o(i._printf_core) for _printf_core
    printf4.o(i.__0vprintf$4) refers to main.o(i.fputc) for fputc
    printf4.o(i.__0vprintf$4) refers to stdout.o(.data) for __stdout
    printf4.o(i.__0vsnprintf$4) refers to printf4.o(i._printf_core) for _printf_core
    printf4.o(i.__0vsnprintf$4) refers to printf4.o(i._snputc) for _snputc
    printf4.o(i.__0vsprintf$4) refers to printf4.o(i._printf_core) for _printf_core
    printf4.o(i.__0vsprintf$4) refers to printf4.o(i._sputc) for _sputc
    printf4.o(i._printf_core) refers to uldiv.o(.text) for __aeabi_uldivmod
    printf5.o(i.__0fprintf$5) refers to printf5.o(i._printf_core) for _printf_core
    printf5.o(i.__0fprintf$5) refers to main.o(i.fputc) for fputc
    printf5.o(i.__0printf$5) refers to printf5.o(i._printf_core) for _printf_core
    printf5.o(i.__0printf$5) refers to main.o(i.fputc) for fputc
    printf5.o(i.__0printf$5) refers to stdout.o(.data) for __stdout
    printf5.o(i.__0snprintf$5) refers to printf5.o(i._printf_core) for _printf_core
    printf5.o(i.__0snprintf$5) refers to printf5.o(i._snputc) for _snputc
    printf5.o(i.__0sprintf$5) refers to printf5.o(i._printf_core) for _printf_core
    printf5.o(i.__0sprintf$5) refers to printf5.o(i._sputc) for _sputc
    printf5.o(i.__0vfprintf$5) refers to printf5.o(i._printf_core) for _printf_core
    printf5.o(i.__0vfprintf$5) refers to main.o(i.fputc) for fputc
    printf5.o(i.__0vprintf$5) refers to printf5.o(i._printf_core) for _printf_core
    printf5.o(i.__0vprintf$5) refers to main.o(i.fputc) for fputc
    printf5.o(i.__0vprintf$5) refers to stdout.o(.data) for __stdout
    printf5.o(i.__0vsnprintf$5) refers to printf5.o(i._printf_core) for _printf_core
    printf5.o(i.__0vsnprintf$5) refers to printf5.o(i._snputc) for _snputc
    printf5.o(i.__0vsprintf$5) refers to printf5.o(i._printf_core) for _printf_core
    printf5.o(i.__0vsprintf$5) refers to printf5.o(i._sputc) for _sputc
    printf5.o(i._printf_core) refers to uldiv.o(.text) for __aeabi_uldivmod
    printf6.o(i.__0fprintf$6) refers to printf6.o(i._printf_core) for _printf_core
    printf6.o(i.__0fprintf$6) refers to main.o(i.fputc) for fputc
    printf6.o(i.__0printf$6) refers to printf6.o(i._printf_core) for _printf_core
    printf6.o(i.__0printf$6) refers to main.o(i.fputc) for fputc
    printf6.o(i.__0printf$6) refers to stdout.o(.data) for __stdout
    printf6.o(i.__0snprintf$6) refers to printf6.o(i._printf_core) for _printf_core
    printf6.o(i.__0snprintf$6) refers to printf6.o(i._snputc) for _snputc
    printf6.o(i.__0sprintf$6) refers to printf6.o(i._printf_core) for _printf_core
    printf6.o(i.__0sprintf$6) refers to printf6.o(i._sputc) for _sputc
    printf6.o(i.__0vfprintf$6) refers to printf6.o(i._printf_core) for _printf_core
    printf6.o(i.__0vfprintf$6) refers to main.o(i.fputc) for fputc
    printf6.o(i.__0vprintf$6) refers to printf6.o(i._printf_core) for _printf_core
    printf6.o(i.__0vprintf$6) refers to main.o(i.fputc) for fputc
    printf6.o(i.__0vprintf$6) refers to stdout.o(.data) for __stdout
    printf6.o(i.__0vsnprintf$6) refers to printf6.o(i._printf_core) for _printf_core
    printf6.o(i.__0vsnprintf$6) refers to printf6.o(i._snputc) for _snputc
    printf6.o(i.__0vsprintf$6) refers to printf6.o(i._printf_core) for _printf_core
    printf6.o(i.__0vsprintf$6) refers to printf6.o(i._sputc) for _sputc
    printf6.o(i._printf_core) refers to printf6.o(i._printf_pre_padding) for _printf_pre_padding
    printf6.o(i._printf_core) refers to printf6.o(i._printf_post_padding) for _printf_post_padding
    printf6.o(i._printf_core) refers to uidiv.o(.text) for __aeabi_uidivmod
    printf7.o(i.__0fprintf$7) refers to printf7.o(i._printf_core) for _printf_core
    printf7.o(i.__0fprintf$7) refers to main.o(i.fputc) for fputc
    printf7.o(i.__0printf$7) refers to printf7.o(i._printf_core) for _printf_core
    printf7.o(i.__0printf$7) refers to main.o(i.fputc) for fputc
    printf7.o(i.__0printf$7) refers to stdout.o(.data) for __stdout
    printf7.o(i.__0snprintf$7) refers to printf7.o(i._printf_core) for _printf_core
    printf7.o(i.__0snprintf$7) refers to printf7.o(i._snputc) for _snputc
    printf7.o(i.__0sprintf$7) refers to printf7.o(i._printf_core) for _printf_core
    printf7.o(i.__0sprintf$7) refers to printf7.o(i._sputc) for _sputc
    printf7.o(i.__0vfprintf$7) refers to printf7.o(i._printf_core) for _printf_core
    printf7.o(i.__0vfprintf$7) refers to main.o(i.fputc) for fputc
    printf7.o(i.__0vprintf$7) refers to printf7.o(i._printf_core) for _printf_core
    printf7.o(i.__0vprintf$7) refers to main.o(i.fputc) for fputc
    printf7.o(i.__0vprintf$7) refers to stdout.o(.data) for __stdout
    printf7.o(i.__0vsnprintf$7) refers to printf7.o(i._printf_core) for _printf_core
    printf7.o(i.__0vsnprintf$7) refers to printf7.o(i._snputc) for _snputc
    printf7.o(i.__0vsprintf$7) refers to printf7.o(i._printf_core) for _printf_core
    printf7.o(i.__0vsprintf$7) refers to printf7.o(i._sputc) for _sputc
    printf7.o(i._printf_core) refers to printf7.o(i._printf_pre_padding) for _printf_pre_padding
    printf7.o(i._printf_core) refers to printf7.o(i._printf_post_padding) for _printf_post_padding
    printf7.o(i._printf_core) refers to uldiv.o(.text) for __aeabi_uldivmod
    printf8.o(i.__0fprintf$8) refers to printf8.o(i._printf_core) for _printf_core
    printf8.o(i.__0fprintf$8) refers to main.o(i.fputc) for fputc
    printf8.o(i.__0printf$8) refers to printf8.o(i._printf_core) for _printf_core
    printf8.o(i.__0printf$8) refers to main.o(i.fputc) for fputc
    printf8.o(i.__0printf$8) refers to stdout.o(.data) for __stdout
    printf8.o(i.__0snprintf$8) refers to printf8.o(i._printf_core) for _printf_core
    printf8.o(i.__0snprintf$8) refers to printf8.o(i._snputc) for _snputc
    printf8.o(i.__0sprintf$8) refers to printf8.o(i._printf_core) for _printf_core
    printf8.o(i.__0sprintf$8) refers to printf8.o(i._sputc) for _sputc
    printf8.o(i.__0vfprintf$8) refers to printf8.o(i._printf_core) for _printf_core
    printf8.o(i.__0vfprintf$8) refers to main.o(i.fputc) for fputc
    printf8.o(i.__0vprintf$8) refers to printf8.o(i._printf_core) for _printf_core
    printf8.o(i.__0vprintf$8) refers to main.o(i.fputc) for fputc
    printf8.o(i.__0vprintf$8) refers to stdout.o(.data) for __stdout
    printf8.o(i.__0vsnprintf$8) refers to printf8.o(i._printf_core) for _printf_core
    printf8.o(i.__0vsnprintf$8) refers to printf8.o(i._snputc) for _snputc
    printf8.o(i.__0vsprintf$8) refers to printf8.o(i._printf_core) for _printf_core
    printf8.o(i.__0vsprintf$8) refers to printf8.o(i._sputc) for _sputc
    printf8.o(i._printf_core) refers to printf8.o(i._printf_pre_padding) for _printf_pre_padding
    printf8.o(i._printf_core) refers to printf8.o(i._printf_post_padding) for _printf_post_padding
    printf8.o(i._printf_core) refers to uldiv.o(.text) for __aeabi_uldivmod
    printfa.o(i.__0fprintf) refers (Special) to iusefp.o(.text) for __I$use$fp
    printfa.o(i.__0fprintf) refers to printfa.o(i._printf_core) for _printf_core
    printfa.o(i.__0fprintf) refers to main.o(i.fputc) for fputc
    printfa.o(i.__0printf) refers (Special) to iusefp.o(.text) for __I$use$fp
    printfa.o(i.__0printf) refers to printfa.o(i._printf_core) for _printf_core
    printfa.o(i.__0printf) refers to main.o(i.fputc) for fputc
    printfa.o(i.__0printf) refers to stdout.o(.data) for __stdout
    printfa.o(i.__0snprintf) refers (Special) to iusefp.o(.text) for __I$use$fp
    printfa.o(i.__0snprintf) refers to printfa.o(i._printf_core) for _printf_core
    printfa.o(i.__0snprintf) refers to printfa.o(i._snputc) for _snputc
    printfa.o(i.__0sprintf) refers (Special) to iusefp.o(.text) for __I$use$fp
    printfa.o(i.__0sprintf) refers to printfa.o(i._printf_core) for _printf_core
    printfa.o(i.__0sprintf) refers to printfa.o(i._sputc) for _sputc
    printfa.o(i.__0vfprintf) refers (Special) to iusefp.o(.text) for __I$use$fp
    printfa.o(i.__0vfprintf) refers to printfa.o(i._printf_core) for _printf_core
    printfa.o(i.__0vfprintf) refers to main.o(i.fputc) for fputc
    printfa.o(i.__0vprintf) refers (Special) to iusefp.o(.text) for __I$use$fp
    printfa.o(i.__0vprintf) refers to printfa.o(i._printf_core) for _printf_core
    printfa.o(i.__0vprintf) refers to main.o(i.fputc) for fputc
    printfa.o(i.__0vprintf) refers to stdout.o(.data) for __stdout
    printfa.o(i.__0vsnprintf) refers (Special) to iusefp.o(.text) for __I$use$fp
    printfa.o(i.__0vsnprintf) refers to printfa.o(i._printf_core) for _printf_core
    printfa.o(i.__0vsnprintf) refers to printfa.o(i._snputc) for _snputc
    printfa.o(i.__0vsprintf) refers (Special) to iusefp.o(.text) for __I$use$fp
    printfa.o(i.__0vsprintf) refers to printfa.o(i._printf_core) for _printf_core
    printfa.o(i.__0vsprintf) refers to printfa.o(i._sputc) for _sputc
    printfa.o(i._fp_digits) refers (Special) to iusefp.o(.text) for __I$use$fp
    printfa.o(i._fp_digits) refers to dmul.o(.text) for __aeabi_dmul
    printfa.o(i._fp_digits) refers to ddiv.o(.text) for __aeabi_ddiv
    printfa.o(i._fp_digits) refers to cdrcmple.o(.text) for __aeabi_cdrcmple
    printfa.o(i._fp_digits) refers to dadd.o(.text) for __aeabi_dadd
    printfa.o(i._fp_digits) refers to dfixul.o(.text) for __aeabi_d2ulz
    printfa.o(i._fp_digits) refers to uldiv.o(.text) for __aeabi_uldivmod
    printfa.o(i._printf_core) refers (Special) to iusefp.o(.text) for __I$use$fp
    printfa.o(i._printf_core) refers to printfa.o(i._printf_pre_padding) for _printf_pre_padding
    printfa.o(i._printf_core) refers to uldiv.o(.text) for __aeabi_uldivmod
    printfa.o(i._printf_core) refers to printfa.o(i._printf_post_padding) for _printf_post_padding
    printfa.o(i._printf_core) refers to printfa.o(i._fp_digits) for _fp_digits
    printfa.o(i._printf_core) refers to uidiv.o(.text) for __aeabi_uidivmod
    printfa.o(i._printf_post_padding) refers (Special) to iusefp.o(.text) for __I$use$fp
    printfa.o(i._printf_pre_padding) refers (Special) to iusefp.o(.text) for __I$use$fp
    printfa.o(i._snputc) refers (Special) to iusefp.o(.text) for __I$use$fp
    printfa.o(i._sputc) refers (Special) to iusefp.o(.text) for __I$use$fp
    entry2.o(.ARM.Collect$$$$00000001) refers to entry2.o(.ARM.Collect$$$$00002712) for __lit__00000000
    entry2.o(.ARM.Collect$$$$00002712) refers to startup_mg32x02z.o(STACK) for __initial_sp
    entry2.o(__vectab_stack_and_reset_area) refers to startup_mg32x02z.o(STACK) for __initial_sp
    entry2.o(__vectab_stack_and_reset_area) refers to entry.o(.ARM.Collect$$$$00000000) for __main
    entry5.o(.ARM.Collect$$$$00000004) refers to init.o(.text) for __scatterload
    entry9a.o(.ARM.Collect$$$$0000000B) refers to main.o(i.main) for main
    entry9b.o(.ARM.Collect$$$$0000000C) refers to main.o(i.main) for main
    uldiv.o(.text) refers to llushr.o(.text) for __aeabi_llsr
    uldiv.o(.text) refers to llshl.o(.text) for __aeabi_llsl
    dadd.o(.text) refers to llshl.o(.text) for __aeabi_llsl
    dadd.o(.text) refers to llsshr.o(.text) for __aeabi_lasr
    dadd.o(.text) refers to depilogue.o(.text) for _double_epilogue
    dmul.o(.text) refers to depilogue.o(.text) for _double_epilogue
    ddiv.o(.text) refers to depilogue.o(.text) for _double_round
    dfixul.o(.text) refers to llushr.o(.text) for __aeabi_llsr
    dfixul.o(.text) refers to llshl.o(.text) for __aeabi_llsl
    init.o(.text) refers to entry5.o(.ARM.Collect$$$$00000004) for __main_after_scatterload
    depilogue.o(.text) refers to depilogue.o(i.__ARM_clz) for __ARM_clz
    depilogue.o(.text) refers to llshl.o(.text) for __aeabi_llsl
    depilogue.o(.text) refers to llushr.o(.text) for __aeabi_llsr


==============================================================================

Removing Unused input sections from the image.

    Removing main.o(.rev16_text), (4 bytes).
    Removing main.o(.revsh_text), (4 bytes).
    Removing main.o(i.UartSendByte), (44 bytes).
    Removing mg32x02z__common_drv.o(.rev16_text), (4 bytes).
    Removing mg32x02z__common_drv.o(.revsh_text), (4 bytes).
    Removing mg32x02z__common_drv.o(i.Delay), (32 bytes).
    Removing mg32x02z__common_drv.o(i.GetTick), (12 bytes).
    Removing mg32x02z__common_drv.o(i.IncTick), (16 bytes).
    Removing mg32x02z__common_drv.o(i.InitTick), (76 bytes).
    Removing mg32x02z__common_drv.o(i.LockModuleReg), (24 bytes).
    Removing mg32x02z__common_drv.o(i.ResumeTick), (20 bytes).
    Removing mg32x02z__common_drv.o(i.SuspendTick), (20 bytes).
    Removing mg32x02z__common_drv.o(i.__NVIC_SetPriority), (120 bytes).
    Removing mg32x02z__common_drv.o(.data), (4 bytes).
    Removing mg32x02z_pw_drv.o(.rev16_text), (4 bytes).
    Removing mg32x02z_pw_drv.o(.revsh_text), (4 bytes).
    Removing mg32x02z_pw_drv.o(i.PW_BOD1Threshold_Select), (28 bytes).
    Removing mg32x02z_pw_drv.o(i.PW_BOD1Trigger_Select), (24 bytes).
    Removing mg32x02z_pw_drv.o(i.PW_BOD1_Cmd), (40 bytes).
    Removing mg32x02z_pw_drv.o(i.PW_ClearFlag), (12 bytes).
    Removing mg32x02z_pw_drv.o(i.PW_GetAllFlagStatus), (12 bytes).
    Removing mg32x02z_pw_drv.o(i.PW_GetBod1Status), (28 bytes).
    Removing mg32x02z_pw_drv.o(i.PW_GetSingleFlagStatus), (28 bytes).
    Removing mg32x02z_pw_drv.o(i.PW_GetWakeUpMode), (52 bytes).
    Removing mg32x02z_pw_drv.o(i.PW_ITEA_Cmd), (40 bytes).
    Removing mg32x02z_pw_drv.o(i.PW_IT_Config), (36 bytes).
    Removing mg32x02z_pw_drv.o(i.PW_IntVoltageRef), (40 bytes).
    Removing mg32x02z_pw_drv.o(i.PW_OnModeLDO_Select), (28 bytes).
    Removing mg32x02z_pw_drv.o(i.PW_PeriphSleepModeContinuous_Config), (32 bytes).
    Removing mg32x02z_pw_drv.o(i.PW_PeriphStopModeContinuous_Config), (32 bytes).
    Removing mg32x02z_pw_drv.o(i.PW_PeriphStopModeWakeUp_Config), (80 bytes).
    Removing mg32x02z_pw_drv.o(i.PW_StopModeLDO_Select), (28 bytes).
    Removing mg32x02z_pw_drv.o(i.PW_WakeUpDelay_Select), (28 bytes).
    Removing mg32x02z_rst_drv.o(.rev16_text), (4 bytes).
    Removing mg32x02z_rst_drv.o(.revsh_text), (4 bytes).
    Removing mg32x02z_rst_drv.o(i.RST_CRstSource_Config), (34 bytes).
    Removing mg32x02z_rst_drv.o(i.RST_ClearFlag), (8 bytes).
    Removing mg32x02z_rst_drv.o(i.RST_ForceResetPeriph_SW), (188 bytes).
    Removing mg32x02z_rst_drv.o(i.RST_GetAllFlagStatus), (8 bytes).
    Removing mg32x02z_rst_drv.o(i.RST_GetSingleFlagStatus), (24 bytes).
    Removing mg32x02z_rst_drv.o(i.RST_TriggerSystemRst_SW), (40 bytes).
    Removing mg32x02z_rst_drv.o(i.RST_WRstGPIOLock_Config), (34 bytes).
    Removing mg32x02z_rst_drv.o(i.RST_WRstSource_Config), (34 bytes).
    Removing mg32x02z_rst_drv.o(i.RST_WWDTWRstMask_Cmd), (40 bytes).
    Removing mg32x02z_csc_drv.o(.rev16_text), (4 bytes).
    Removing mg32x02z_csc_drv.o(.revsh_text), (4 bytes).
    Removing mg32x02z_csc_drv.o(i.CSC_CK_LS_Select), (28 bytes).
    Removing mg32x02z_csc_drv.o(i.CSC_CK_ST_Select), (28 bytes).
    Removing mg32x02z_csc_drv.o(i.CSC_CK_UT_Divider_Select), (32 bytes).
    Removing mg32x02z_csc_drv.o(i.CSC_GetAllFlagStatus), (12 bytes).
    Removing mg32x02z_csc_drv.o(i.CSC_ICKO_ClockSource_Select), (32 bytes).
    Removing mg32x02z_csc_drv.o(i.CSC_ICKO_Cmd), (40 bytes).
    Removing mg32x02z_csc_drv.o(i.CSC_ICKO_Divider_Select), (32 bytes).
    Removing mg32x02z_csc_drv.o(i.CSC_ITEA_Cmd), (40 bytes).
    Removing mg32x02z_csc_drv.o(i.CSC_IT_Config), (36 bytes).
    Removing mg32x02z_csc_drv.o(i.CSC_MissingClockDetectionDuration_Select), (28 bytes).
    Removing mg32x02z_csc_drv.o(i.CSC_MissingClockDetection_Cmd), (36 bytes).
    Removing mg32x02z_csc_drv.o(i.CSC_PeriphSleepModeClock_Config), (132 bytes).
    Removing mg32x02z_csc_drv.o(i.CSC_PeriphStopModeClock_Config), (44 bytes).
    Removing mg32x02z_csc_drv.o(i.CSC_XOSCGain_Select), (28 bytes).
    Removing mg32x02z_csc_drv.o(i.CSC_XOSC_Cmd), (52 bytes).
    Removing mg32x02z_sys_drv.o(.rev16_text), (4 bytes).
    Removing mg32x02z_sys_drv.o(.revsh_text), (4 bytes).
    Removing mg32x02z_sys_drv.o(i.SYS_GetChipMID), (12 bytes).
    Removing mg32x02z_sys_drv.o(i.SYS_ITEA_Cmd), (24 bytes).
    Removing mg32x02z_sys_drv.o(i.SYS_ReadGeneralReg), (12 bytes).
    Removing mg32x02z_sys_drv.o(i.SYS_WriteGeneralReg), (12 bytes).
    Removing mg32x02z_cfg_drv.o(.rev16_text), (4 bytes).
    Removing mg32x02z_cfg_drv.o(.revsh_text), (4 bytes).
    Removing mg32x02z_cfg_drv.o(i.CFG_GetADC0RefBottom), (16 bytes).
    Removing mg32x02z_cfg_drv.o(i.CFG_GetADC0RefMiddle), (16 bytes).
    Removing mg32x02z_cfg_drv.o(i.CFG_GetADC0RefTop), (16 bytes).
    Removing mg32x02z_cfg_drv.o(i.CFG_GetTempHigValue), (16 bytes).
    Removing mg32x02z_cfg_drv.o(i.CFG_GetTempLowValue), (16 bytes).
    Removing mg32x02z_cfg_drv.o(i.CFG_SetADC0RefBottom), (16 bytes).
    Removing mg32x02z_cfg_drv.o(i.CFG_SetADC0RefMiddle), (16 bytes).
    Removing mg32x02z_cfg_drv.o(i.CFG_SetADC0RefTop), (16 bytes).
    Removing mg32x02z_mem_drv.o(.rev16_text), (4 bytes).
    Removing mg32x02z_mem_drv.o(.revsh_text), (4 bytes).
    Removing mg32x02z_mem_drv.o(i.MEM_APWrite_Cmd), (124 bytes).
    Removing mg32x02z_mem_drv.o(i.MEM_Access_Cmd), (60 bytes).
    Removing mg32x02z_mem_drv.o(i.MEM_ClearFlag), (8 bytes).
    Removing mg32x02z_mem_drv.o(i.MEM_Cmd), (60 bytes).
    Removing mg32x02z_mem_drv.o(i.MEM_ErrorHardFault_Cmd), (60 bytes).
    Removing mg32x02z_mem_drv.o(i.MEM_ErrorReset_Cmd), (60 bytes).
    Removing mg32x02z_mem_drv.o(i.MEM_GetAccessState), (22 bytes).
    Removing mg32x02z_mem_drv.o(i.MEM_GetAllAccessState), (16 bytes).
    Removing mg32x02z_mem_drv.o(i.MEM_GetAllFlagStatus), (8 bytes).
    Removing mg32x02z_mem_drv.o(i.MEM_GetFlagStatus), (22 bytes).
    Removing mg32x02z_mem_drv.o(i.MEM_GetIAPSize), (12 bytes).
    Removing mg32x02z_mem_drv.o(i.MEM_GetISPSize), (12 bytes).
    Removing mg32x02z_mem_drv.o(i.MEM_IAPExecuteCode_Cmd), (120 bytes).
    Removing mg32x02z_mem_drv.o(i.MEM_IAPWrite_Cmd), (120 bytes).
    Removing mg32x02z_mem_drv.o(i.MEM_ISPDRead_Cmd), (120 bytes).
    Removing mg32x02z_mem_drv.o(i.MEM_ISPDWrite_Cmd), (120 bytes).
    Removing mg32x02z_mem_drv.o(i.MEM_ISPRead_Cmd), (124 bytes).
    Removing mg32x02z_mem_drv.o(i.MEM_ISPWrite_Cmd), (124 bytes).
    Removing mg32x02z_mem_drv.o(i.MEM_ITEA_Cmd), (60 bytes).
    Removing mg32x02z_mem_drv.o(i.MEM_IT_Cmd), (60 bytes).
    Removing mg32x02z_mem_drv.o(i.MEM_SetIAPSize), (116 bytes).
    Removing mg32x02z_mem_drv.o(i.MEM_SetIAPSizeLock), (56 bytes).
    Removing mg32x02z_mem_drv.o(i.MEM_SetISPMultiplePageEraseUnProtect), (104 bytes).
    Removing mg32x02z_mem_drv.o(i.MEM_SetISPMultipleProgramUnProtect), (100 bytes).
    Removing mg32x02z_mem_drv.o(i.MEM_SetISPMultipleWriteProtect), (56 bytes).
    Removing mg32x02z_mem_drv.o(i.MEM_SetISPSinglePageEraseUnProtect), (104 bytes).
    Removing mg32x02z_mem_drv.o(i.MEM_SetISPSingleProgramUnProtect), (104 bytes).
    Removing mg32x02z_mem_drv.o(i.MEM_SetMultiplePageEraseUnProtect), (56 bytes).
    Removing mg32x02z_mem_drv.o(i.MEM_SetMultipleProgramUnProtect), (56 bytes).
    Removing mg32x02z_mem_drv.o(i.MEM_SetMultipleWriteProtect), (60 bytes).
    Removing mg32x02z_mem_drv.o(i.MEM_SetSinglePageEraseUnProtect), (56 bytes).
    Removing mg32x02z_mem_drv.o(i.MEM_SetSingleProgramUnProtect), (56 bytes).
    Removing mg32x02z_mem_drv.o(i.MEM_SetWriteMode), (48 bytes).
    Removing mg32x02z_mem_drv.o(i.MEM_SetWriteUnProtect), (168 bytes).
    Removing mg32x02z_mem_drv.o(i.MEM_WriteFlashHold_Cmd), (60 bytes).
    Removing mg32x02z_gpio_drv.o(.rev16_text), (4 bytes).
    Removing mg32x02z_gpio_drv.o(.revsh_text), (4 bytes).
    Removing mg32x02z_gpio_drv.o(i.GPIO_ClearPortBit), (4 bytes).
    Removing mg32x02z_gpio_drv.o(i.GPIO_PinFunction_Select), (26 bytes).
    Removing mg32x02z_gpio_drv.o(i.GPIO_PinHighSpeedMode_Cmd), (20 bytes).
    Removing mg32x02z_gpio_drv.o(i.GPIO_PinInFilterDivider_Select), (18 bytes).
    Removing mg32x02z_gpio_drv.o(i.GPIO_PinInverse_Cmd), (20 bytes).
    Removing mg32x02z_gpio_drv.o(i.GPIO_PinMode_Select), (20 bytes).
    Removing mg32x02z_gpio_drv.o(i.GPIO_PinOutputDrive_Select), (18 bytes).
    Removing mg32x02z_gpio_drv.o(i.GPIO_PinPUResister_Cmd), (20 bytes).
    Removing mg32x02z_gpio_drv.o(i.GPIO_PortFilterClockSource_Select), (20 bytes).
    Removing mg32x02z_gpio_drv.o(i.GPIO_PortMode_Config), (74 bytes).
    Removing mg32x02z_gpio_drv.o(i.GPIO_ReadPort), (8 bytes).
    Removing mg32x02z_gpio_drv.o(i.GPIO_SetClearPortBit), (12 bytes).
    Removing mg32x02z_gpio_drv.o(i.GPIO_SetPortBit), (4 bytes).
    Removing mg32x02z_gpio_drv.o(i.GPIO_WritePort), (4 bytes).
    Removing mg32x02z_exic_drv.o(.rev16_text), (4 bytes).
    Removing mg32x02z_exic_drv.o(.revsh_text), (4 bytes).
    Removing mg32x02z_exic_drv.o(i.EXIC_ClearPxTriggerEventFlag), (4 bytes).
    Removing mg32x02z_exic_drv.o(i.EXIC_ClearPxTriggerITFlag), (18 bytes).
    Removing mg32x02z_exic_drv.o(i.EXIC_GetITSourceID), (16 bytes).
    Removing mg32x02z_exic_drv.o(i.EXIC_GetPinxTriggerEventSingleFlagStatus), (16 bytes).
    Removing mg32x02z_exic_drv.o(i.EXIC_GetPxAllTriggerEventFlagStatus), (8 bytes).
    Removing mg32x02z_exic_drv.o(i.EXIC_GetPxAllTriggerITFlagStatus), (28 bytes).
    Removing mg32x02z_exic_drv.o(i.EXIC_GetPxTriggerAndITFlagStatus), (32 bytes).
    Removing mg32x02z_exic_drv.o(i.EXIC_GetPxTriggerOrITFlagStatus), (32 bytes).
    Removing mg32x02z_exic_drv.o(i.EXIC_NMITrigger_SW), (20 bytes).
    Removing mg32x02z_exic_drv.o(i.EXIC_NMI_Cmd), (24 bytes).
    Removing mg32x02z_exic_drv.o(i.EXIC_PxTriggerAndMask_Select), (4 bytes).
    Removing mg32x02z_exic_drv.o(i.EXIC_PxTriggerAndUnmatch_Cmd), (38 bytes).
    Removing mg32x02z_exic_drv.o(i.EXIC_PxTriggerITEA_Cmd), (36 bytes).
    Removing mg32x02z_exic_drv.o(i.EXIC_PxTriggerMode_Select), (52 bytes).
    Removing mg32x02z_exic_drv.o(i.EXIC_PxTriggerOrMask_Select), (4 bytes).
    Removing mg32x02z_exic_drv.o(i.EXIC_RXEV_Cmd), (26 bytes).
    Removing mg32x02z_gpl_drv.o(.rev16_text), (4 bytes).
    Removing mg32x02z_gpl_drv.o(.revsh_text), (4 bytes).
    Removing mg32x02z_gpl_drv.o(i.GPL_AfterBitOrderChange_Select), (20 bytes).
    Removing mg32x02z_gpl_drv.o(i.GPL_BeferBitOrderChange_Select), (20 bytes).
    Removing mg32x02z_gpl_drv.o(i.GPL_ByteOrderChange_Cmd), (40 bytes).
    Removing mg32x02z_gpl_drv.o(i.GPL_CRC_Cmd), (40 bytes).
    Removing mg32x02z_gpl_drv.o(i.GPL_CRC_Data_Size_Select), (20 bytes).
    Removing mg32x02z_gpl_drv.o(i.GPL_CRC_Mode_Select), (20 bytes).
    Removing mg32x02z_gpl_drv.o(i.GPL_CRC_SetInitValue), (8 bytes).
    Removing mg32x02z_gpl_drv.o(i.GPL_DataInput), (8 bytes).
    Removing mg32x02z_gpl_drv.o(i.GPL_GetAllFlagStatus), (8 bytes).
    Removing mg32x02z_gpl_drv.o(i.GPL_GetFlagStatus), (22 bytes).
    Removing mg32x02z_gpl_drv.o(i.GPL_GetOutputData), (24 bytes).
    Removing mg32x02z_gpl_drv.o(i.GPL_GetParityCheckByte), (118 bytes).
    Removing mg32x02z_gpl_drv.o(i.GPL_GetParityCheckByte_0), (26 bytes).
    Removing mg32x02z_gpl_drv.o(i.GPL_GetParityCheckByte_1), (26 bytes).
    Removing mg32x02z_gpl_drv.o(i.GPL_GetParityCheckByte_2), (26 bytes).
    Removing mg32x02z_gpl_drv.o(i.GPL_GetParityCheckByte_3), (26 bytes).
    Removing mg32x02z_gpl_drv.o(i.GPL_GetParityCheckHalfWord), (58 bytes).
    Removing mg32x02z_gpl_drv.o(i.GPL_GetParityCheckHalfWord_High), (26 bytes).
    Removing mg32x02z_gpl_drv.o(i.GPL_GetParityCheckHalfWord_Low), (26 bytes).
    Removing mg32x02z_gpl_drv.o(i.GPL_GetParityCheckWord), (26 bytes).
    Removing mg32x02z_gpl_drv.o(i.GPL_Inverse_Cmd), (40 bytes).
    Removing mg32x02z_gpl_drv.o(i.GPL_ParityCheck_Select), (20 bytes).
    Removing mg32x02z_dma_drv.o(.rev16_text), (4 bytes).
    Removing mg32x02z_dma_drv.o(.revsh_text), (4 bytes).
    Removing mg32x02z_dma_drv.o(i.DMA_ClearChannelFlag), (4 bytes).
    Removing mg32x02z_dma_drv.o(i.DMA_DeInit), (60 bytes).
    Removing mg32x02z_dma_drv.o(i.DMA_GetAllFlagStatus), (6 bytes).
    Removing mg32x02z_dma_drv.o(i.DMA_GetCHxUseGPL), (10 bytes).
    Removing mg32x02z_dma_drv.o(i.DMA_GetCurrentDestinationAddress), (6 bytes).
    Removing mg32x02z_dma_drv.o(i.DMA_GetCurrentSourceAddress), (6 bytes).
    Removing mg32x02z_dma_drv.o(i.DMA_GetRemainDataCount), (6 bytes).
    Removing mg32x02z_dma_drv.o(i.DMA_Hold_Cmd), (20 bytes).
    Removing mg32x02z_dma_drv.o(i.DMA_ITEA_Cmd), (16 bytes).
    Removing mg32x02z_dma_drv.o(i.DMA_IT_Config), (20 bytes).
    Removing mg32x02z_dma_drv.o(i.DMA_LastCycle_Cmd), (96 bytes).
    Removing mg32x02z_dma_drv.o(i.DMA_PriorityMode_Select), (20 bytes).
    Removing mg32x02z_dma_drv.o(i.DMA_SetChxSKIP3Mode), (20 bytes).
    Removing mg32x02z_dma_drv.o(i.DMA_SetExtraGPLChannel), (20 bytes).
    Removing mg32x02z_dma_drv.o(i.DMA_SetPrority), (20 bytes).
    Removing mg32x02z_emb_drv.o(.rev16_text), (4 bytes).
    Removing mg32x02z_emb_drv.o(.revsh_text), (4 bytes).
    Removing mg32x02z_emb_drv.o(i.EMB_AddressDataBusMode_Config), (52 bytes).
    Removing mg32x02z_emb_drv.o(i.EMB_GetSingleFlagStatus), (24 bytes).
    Removing mg32x02z_emb_drv.o(i.EMB_IT_Cmd), (32 bytes).
    Removing mg32x02z_emb_drv.o(i.EMB_SendSignalStatus_SW), (52 bytes).
    Removing mg32x02z_emb_drv.o(i.EMB_SignalInverse_Cmd), (52 bytes).
    Removing mg32x02z_emb_drv.o(i.EMB_SignalSWAP_Cmd), (52 bytes).
    Removing mg32x02z_emb_drv.o(i.EMB_SignalSW_Cmd), (52 bytes).
    Removing mg32x02z_emb_drv.o(i.EMB_WriteMode_Select), (32 bytes).
    Removing mg32x02z_apb_drv.o(.rev16_text), (4 bytes).
    Removing mg32x02z_apb_drv.o(.revsh_text), (4 bytes).
    Removing mg32x02z_apb_drv.o(i.APB_BreakSourceChannel0_Select), (16 bytes).
    Removing mg32x02z_apb_drv.o(i.APB_BreakSourceChannel1_Select), (20 bytes).
    Removing mg32x02z_apb_drv.o(i.APB_BreakSourceChannel2_Select), (16 bytes).
    Removing mg32x02z_apb_drv.o(i.APB_ClearFlag), (4 bytes).
    Removing mg32x02z_apb_drv.o(i.APB_GetAllFlagStatus), (6 bytes).
    Removing mg32x02z_apb_drv.o(i.APB_GetOBMxInitState), (20 bytes).
    Removing mg32x02z_apb_drv.o(i.APB_GetOBMxOutputState), (24 bytes).
    Removing mg32x02z_apb_drv.o(i.APB_GetOBMxSwitchState), (24 bytes).
    Removing mg32x02z_apb_drv.o(i.APB_GetSingleFlagStatus), (18 bytes).
    Removing mg32x02z_apb_drv.o(i.APB_IRCLK_Select), (24 bytes).
    Removing mg32x02z_apb_drv.o(i.APB_IRDAT_Select), (26 bytes).
    Removing mg32x02z_apb_drv.o(i.APB_ITEA_Cmd), (16 bytes).
    Removing mg32x02z_apb_drv.o(i.APB_ITR6_Select), (24 bytes).
    Removing mg32x02z_apb_drv.o(i.APB_ITR7_Select), (26 bytes).
    Removing mg32x02z_apb_drv.o(i.APB_IT_Config), (20 bytes).
    Removing mg32x02z_apb_drv.o(i.APB_InverseBKS0_Cmd), (16 bytes).
    Removing mg32x02z_apb_drv.o(i.APB_InverseBKS1_Cmd), (20 bytes).
    Removing mg32x02z_apb_drv.o(i.APB_InverseBKS2_Cmd), (20 bytes).
    Removing mg32x02z_apb_drv.o(i.APB_InverseIRCLK_Cmd), (26 bytes).
    Removing mg32x02z_apb_drv.o(i.APB_InverseIRDAT_Cmd), (26 bytes).
    Removing mg32x02z_apb_drv.o(i.APB_InverseOBMxOutput_Cmd), (20 bytes).
    Removing mg32x02z_apb_drv.o(i.APB_InverseOutputChannel0_Cmd), (16 bytes).
    Removing mg32x02z_apb_drv.o(i.APB_InverseOutputChannel1_Cmd), (20 bytes).
    Removing mg32x02z_apb_drv.o(i.APB_OBMxOpMode_Select), (16 bytes).
    Removing mg32x02z_apb_drv.o(i.APB_OutputChannel0Source_Select), (16 bytes).
    Removing mg32x02z_apb_drv.o(i.APB_OutputChannel1Source_Select), (20 bytes).
    Removing mg32x02z_apb_drv.o(i.APB_OutputFilter_Select), (20 bytes).
    Removing mg32x02z_apb_drv.o(i.APB_SetOBMxInitState), (34 bytes).
    Removing mg32x02z_apb_drv.o(i.APB_TimerX_Cmd), (16 bytes).
    Removing mg32x02z_adc_drv.o(.rev16_text), (4 bytes).
    Removing mg32x02z_adc_drv.o(.revsh_text), (4 bytes).
    Removing mg32x02z_adc_drv.o(i.ADC_AutoOff_Cmd), (20 bytes).
    Removing mg32x02z_adc_drv.o(i.ADC_BaseStructure_Init), (20 bytes).
    Removing mg32x02z_adc_drv.o(i.ADC_Base_Init), (56 bytes).
    Removing mg32x02z_adc_drv.o(i.ADC_ChannelMUX_Select), (24 bytes).
    Removing mg32x02z_adc_drv.o(i.ADC_ClearFlag), (4 bytes).
    Removing mg32x02z_adc_drv.o(i.ADC_ClearSum0Flags), (4 bytes).
    Removing mg32x02z_adc_drv.o(i.ADC_ClearSum1Flags), (4 bytes).
    Removing mg32x02z_adc_drv.o(i.ADC_ClearSum2Flags), (4 bytes).
    Removing mg32x02z_adc_drv.o(i.ADC_ClockSource_Select), (16 bytes).
    Removing mg32x02z_adc_drv.o(i.ADC_Cmd), (16 bytes).
    Removing mg32x02z_adc_drv.o(i.ADC_ContinueMode_Cmd), (24 bytes).
    Removing mg32x02z_adc_drv.o(i.ADC_ConversionMode_Select), (136 bytes).
    Removing mg32x02z_adc_drv.o(i.ADC_DMA_Cmd), (20 bytes).
    Removing mg32x02z_adc_drv.o(i.ADC_DataAlignment_Select), (20 bytes).
    Removing mg32x02z_adc_drv.o(i.ADC_DataOverrunMode_Select), (16 bytes).
    Removing mg32x02z_adc_drv.o(i.ADC_DataResolution_Select), (20 bytes).
    Removing mg32x02z_adc_drv.o(i.ADC_DeInit), (50 bytes).
    Removing mg32x02z_adc_drv.o(i.ADC_ExternalChannel_Select), (6 bytes).
    Removing mg32x02z_adc_drv.o(i.ADC_GetAllFlagStatus), (6 bytes).
    Removing mg32x02z_adc_drv.o(i.ADC_GetDAT0Channel), (10 bytes).
    Removing mg32x02z_adc_drv.o(i.ADC_GetDAT0Data), (10 bytes).
    Removing mg32x02z_adc_drv.o(i.ADC_GetDAT0Flags), (8 bytes).
    Removing mg32x02z_adc_drv.o(i.ADC_GetSingleFlagStatus), (18 bytes).
    Removing mg32x02z_adc_drv.o(i.ADC_GetSum0Data), (8 bytes).
    Removing mg32x02z_adc_drv.o(i.ADC_GetSum0Flags), (6 bytes).
    Removing mg32x02z_adc_drv.o(i.ADC_GetSum1Data), (8 bytes).
    Removing mg32x02z_adc_drv.o(i.ADC_GetSum1Flags), (6 bytes).
    Removing mg32x02z_adc_drv.o(i.ADC_GetSum2Data), (8 bytes).
    Removing mg32x02z_adc_drv.o(i.ADC_GetSum2Flags), (6 bytes).
    Removing mg32x02z_adc_drv.o(i.ADC_HoldConversion_Cmd), (24 bytes).
    Removing mg32x02z_adc_drv.o(i.ADC_ITEA_Cmd), (16 bytes).
    Removing mg32x02z_adc_drv.o(i.ADC_IT_Config), (20 bytes).
    Removing mg32x02z_adc_drv.o(i.ADC_InternalChannel_Select), (6 bytes).
    Removing mg32x02z_adc_drv.o(i.ADC_MainConversionMode_Select), (20 bytes).
    Removing mg32x02z_adc_drv.o(i.ADC_Output_Select), (20 bytes).
    Removing mg32x02z_adc_drv.o(i.ADC_PGAOffsetCalibration_Cmd), (268 bytes).
    Removing mg32x02z_adc_drv.o(i.ADC_PGA_Cmd), (24 bytes).
    Removing mg32x02z_adc_drv.o(i.ADC_ScanLoopChannel_Enable), (20 bytes).
    Removing mg32x02z_adc_drv.o(i.ADC_SetDigitalOffset), (16 bytes).
    Removing mg32x02z_adc_drv.o(i.ADC_SetExtendSampling), (8 bytes).
    Removing mg32x02z_adc_drv.o(i.ADC_SetHigherThreshold), (4 bytes).
    Removing mg32x02z_adc_drv.o(i.ADC_SetInternalClockDivider), (20 bytes).
    Removing mg32x02z_adc_drv.o(i.ADC_SetLimitFunction), (20 bytes).
    Removing mg32x02z_adc_drv.o(i.ADC_SetLowerThreshold), (4 bytes).
    Removing mg32x02z_adc_drv.o(i.ADC_SetOutputCodeFormat), (16 bytes).
    Removing mg32x02z_adc_drv.o(i.ADC_SetPGAGain), (20 bytes).
    Removing mg32x02z_adc_drv.o(i.ADC_SetPGAOffset), (20 bytes).
    Removing mg32x02z_adc_drv.o(i.ADC_SetPLLClockDivider), (20 bytes).
    Removing mg32x02z_adc_drv.o(i.ADC_SetSum0Channel), (16 bytes).
    Removing mg32x02z_adc_drv.o(i.ADC_SetSum0Data), (4 bytes).
    Removing mg32x02z_adc_drv.o(i.ADC_SetSum1Channel), (20 bytes).
    Removing mg32x02z_adc_drv.o(i.ADC_SetSum1Data), (4 bytes).
    Removing mg32x02z_adc_drv.o(i.ADC_SetSum2Channel), (16 bytes).
    Removing mg32x02z_adc_drv.o(i.ADC_SetSum2Data), (4 bytes).
    Removing mg32x02z_adc_drv.o(i.ADC_SetSumNumber), (16 bytes).
    Removing mg32x02z_adc_drv.o(i.ADC_SingleDifferentMode_Select), (20 bytes).
    Removing mg32x02z_adc_drv.o(i.ADC_SoftwareConversion_Cmd), (20 bytes).
    Removing mg32x02z_adc_drv.o(i.ADC_StartCalibration), (600 bytes).
    Removing mg32x02z_adc_drv.o(i.ADC_SumChannelMode_Select), (20 bytes).
    Removing mg32x02z_adc_drv.o(i.ADC_SumOverrunMode_Select), (20 bytes).
    Removing mg32x02z_adc_drv.o(i.ADC_TriggerEdge_Select), (24 bytes).
    Removing mg32x02z_adc_drv.o(i.ADC_TriggerSource_Select), (20 bytes).
    Removing mg32x02z_adc_drv.o(i.ADC_VRMCalibration), (320 bytes).
    Removing mg32x02z_adc_drv.o(i.ADC_WaitDataReadOut), (20 bytes).
    Removing mg32x02z_adc_drv.o(i.ADC_WindowDetectRange_Select), (20 bytes).
    Removing mg32x02z_adc_drv.o(i.ADC_WindowDetect_Cmd), (16 bytes).
    Removing mg32x02z_cmp_drv.o(.rev16_text), (4 bytes).
    Removing mg32x02z_cmp_drv.o(.revsh_text), (4 bytes).
    Removing mg32x02z_cmp_drv.o(i.CMP_ClearFlag), (4 bytes).
    Removing mg32x02z_cmp_drv.o(i.CMP_Cmd), (16 bytes).
    Removing mg32x02z_cmp_drv.o(i.CMP_DeInit), (24 bytes).
    Removing mg32x02z_cmp_drv.o(i.CMP_FilterClockDivider_Select), (20 bytes).
    Removing mg32x02z_cmp_drv.o(i.CMP_FilterClock_Select), (20 bytes).
    Removing mg32x02z_cmp_drv.o(i.CMP_GetAllFlagStatus), (6 bytes).
    Removing mg32x02z_cmp_drv.o(i.CMP_GetOutput), (120 bytes).
    Removing mg32x02z_cmp_drv.o(i.CMP_GetSingleFlagStatus), (18 bytes).
    Removing mg32x02z_cmp_drv.o(i.CMP_ITEA_Cmd), (16 bytes).
    Removing mg32x02z_cmp_drv.o(i.CMP_IT_Config), (20 bytes).
    Removing mg32x02z_cmp_drv.o(i.CMP_IVREF2_Cmd), (16 bytes).
    Removing mg32x02z_cmp_drv.o(i.CMP_IVREF2_Select), (40 bytes).
    Removing mg32x02z_cmp_drv.o(i.CMP_IVREF_Cmd), (16 bytes).
    Removing mg32x02z_cmp_drv.o(i.CMP_IVREF_Select), (40 bytes).
    Removing mg32x02z_cmp_drv.o(i.CMP_InverseOutputPin), (20 bytes).
    Removing mg32x02z_cmp_drv.o(i.CMP_NegativePin_Select), (20 bytes).
    Removing mg32x02z_cmp_drv.o(i.CMP_OutputPolarity_Select), (16 bytes).
    Removing mg32x02z_cmp_drv.o(i.CMP_PositivePin_Select), (16 bytes).
    Removing mg32x02z_cmp_drv.o(i.CMP_Power_Select), (20 bytes).
    Removing mg32x02z_dac_drv.o(.rev16_text), (4 bytes).
    Removing mg32x02z_dac_drv.o(.revsh_text), (4 bytes).
    Removing mg32x02z_dac_drv.o(i.DAC_ClearFlag), (4 bytes).
    Removing mg32x02z_dac_drv.o(i.DAC_Cmd), (16 bytes).
    Removing mg32x02z_dac_drv.o(i.DAC_CurrentMode_Select), (20 bytes).
    Removing mg32x02z_dac_drv.o(i.DAC_DMA_Cmd), (20 bytes).
    Removing mg32x02z_dac_drv.o(i.DAC_DataAlignment_Select), (20 bytes).
    Removing mg32x02z_dac_drv.o(i.DAC_DataResolution_Select), (20 bytes).
    Removing mg32x02z_dac_drv.o(i.DAC_DeInit), (14 bytes).
    Removing mg32x02z_dac_drv.o(i.DAC_GetAllFlagStatus), (6 bytes).
    Removing mg32x02z_dac_drv.o(i.DAC_GetDACState), (20 bytes).
    Removing mg32x02z_dac_drv.o(i.DAC_GetDAT0), (6 bytes).
    Removing mg32x02z_dac_drv.o(i.DAC_GetOutput), (6 bytes).
    Removing mg32x02z_dac_drv.o(i.DAC_GetSingleFlagStatus), (18 bytes).
    Removing mg32x02z_dac_drv.o(i.DAC_ITEA_Cmd), (16 bytes).
    Removing mg32x02z_dac_drv.o(i.DAC_IT_Config), (20 bytes).
    Removing mg32x02z_dac_drv.o(i.DAC_SetDAT0), (4 bytes).
    Removing mg32x02z_dac_drv.o(i.DAC_TriggerEdge_Select), (20 bytes).
    Removing mg32x02z_dac_drv.o(i.DAC_TriggerSource_Select), (16 bytes).
    Removing mg32x02z_tm_drv.o(.rev16_text), (4 bytes).
    Removing mg32x02z_tm_drv.o(.revsh_text), (4 bytes).
    Removing mg32x02z_tm_drv.o(i.TM_AlignmentMode_Select), (20 bytes).
    Removing mg32x02z_tm_drv.o(i.TM_AutoStop_Cmd), (16 bytes).
    Removing mg32x02z_tm_drv.o(i.TM_BreakCH012_Cmd), (20 bytes).
    Removing mg32x02z_tm_drv.o(i.TM_BreakCH3_Cmd), (24 bytes).
    Removing mg32x02z_tm_drv.o(i.TM_BreakMode_Select), (24 bytes).
    Removing mg32x02z_tm_drv.o(i.TM_BreakTrigger_SW), (24 bytes).
    Removing mg32x02z_tm_drv.o(i.TM_CH0Function_Config), (20 bytes).
    Removing mg32x02z_tm_drv.o(i.TM_CH1Function_Config), (24 bytes).
    Removing mg32x02z_tm_drv.o(i.TM_CH2Function_Config), (20 bytes).
    Removing mg32x02z_tm_drv.o(i.TM_CH3Function_Config), (24 bytes).
    Removing mg32x02z_tm_drv.o(i.TM_CKOOutputState_Init), (32 bytes).
    Removing mg32x02z_tm_drv.o(i.TM_ClearFlag), (4 bytes).
    Removing mg32x02z_tm_drv.o(i.TM_ClockOutSource_Select), (20 bytes).
    Removing mg32x02z_tm_drv.o(i.TM_ClockOut_Cmd), (16 bytes).
    Removing mg32x02z_tm_drv.o(i.TM_CounterClock_Select), (20 bytes).
    Removing mg32x02z_tm_drv.o(i.TM_Counter_Cmd), (24 bytes).
    Removing mg32x02z_tm_drv.o(i.TM_Counter_Config), (6 bytes).
    Removing mg32x02z_tm_drv.o(i.TM_Counter_SW), (22 bytes).
    Removing mg32x02z_tm_drv.o(i.TM_DMAChannel_Cmd), (20 bytes).
    Removing mg32x02z_tm_drv.o(i.TM_DMAUpdateMode_Select), (24 bytes).
    Removing mg32x02z_tm_drv.o(i.TM_DeInit), (76 bytes).
    Removing mg32x02z_tm_drv.o(i.TM_ExtTRGI2UEV_Cmd), (20 bytes).
    Removing mg32x02z_tm_drv.o(i.TM_ExtTRGI_Cmd), (20 bytes).
    Removing mg32x02z_tm_drv.o(i.TM_ExternalBreakEvent_Config), (30 bytes).
    Removing mg32x02z_tm_drv.o(i.TM_ExternalClock_Select), (20 bytes).
    Removing mg32x02z_tm_drv.o(i.TM_FallingCaptureIC0_SW), (20 bytes).
    Removing mg32x02z_tm_drv.o(i.TM_FallingCaptureIC1_SW), (20 bytes).
    Removing mg32x02z_tm_drv.o(i.TM_FallingCaptureIC2_SW), (20 bytes).
    Removing mg32x02z_tm_drv.o(i.TM_FallingCaptureIC3_SW), (20 bytes).
    Removing mg32x02z_tm_drv.o(i.TM_ForceUpdate_SW), (20 bytes).
    Removing mg32x02z_tm_drv.o(i.TM_GateCounter_SW), (20 bytes).
    Removing mg32x02z_tm_drv.o(i.TM_GatePrescaler_SW), (20 bytes).
    Removing mg32x02z_tm_drv.o(i.TM_GenerateCF0A_SW), (16 bytes).
    Removing mg32x02z_tm_drv.o(i.TM_GenerateCF0B_SW), (20 bytes).
    Removing mg32x02z_tm_drv.o(i.TM_GenerateCF1A_SW), (20 bytes).
    Removing mg32x02z_tm_drv.o(i.TM_GenerateCF1B_SW), (20 bytes).
    Removing mg32x02z_tm_drv.o(i.TM_GenerateCF2A_SW), (20 bytes).
    Removing mg32x02z_tm_drv.o(i.TM_GenerateCF2B_SW), (20 bytes).
    Removing mg32x02z_tm_drv.o(i.TM_GenerateCF3A_SW), (20 bytes).
    Removing mg32x02z_tm_drv.o(i.TM_GenerateCF3B_SW), (20 bytes).
    Removing mg32x02z_tm_drv.o(i.TM_GetAllFlagStatus), (6 bytes).
    Removing mg32x02z_tm_drv.o(i.TM_GetCC0A), (8 bytes).
    Removing mg32x02z_tm_drv.o(i.TM_GetCC0B), (8 bytes).
    Removing mg32x02z_tm_drv.o(i.TM_GetCC1A), (8 bytes).
    Removing mg32x02z_tm_drv.o(i.TM_GetCC1B), (8 bytes).
    Removing mg32x02z_tm_drv.o(i.TM_GetCC2A), (8 bytes).
    Removing mg32x02z_tm_drv.o(i.TM_GetCC2B), (8 bytes).
    Removing mg32x02z_tm_drv.o(i.TM_GetCC3A), (8 bytes).
    Removing mg32x02z_tm_drv.o(i.TM_GetCC3B), (8 bytes).
    Removing mg32x02z_tm_drv.o(i.TM_GetCounter), (6 bytes).
    Removing mg32x02z_tm_drv.o(i.TM_GetIC0Value), (24 bytes).
    Removing mg32x02z_tm_drv.o(i.TM_GetIC1Value), (24 bytes).
    Removing mg32x02z_tm_drv.o(i.TM_GetIC2Value), (24 bytes).
    Removing mg32x02z_tm_drv.o(i.TM_GetIC3Value), (24 bytes).
    Removing mg32x02z_tm_drv.o(i.TM_GetPrescaler), (6 bytes).
    Removing mg32x02z_tm_drv.o(i.TM_GetSingleFlagStatus), (18 bytes).
    Removing mg32x02z_tm_drv.o(i.TM_IC0OverWritten_Cmd), (16 bytes).
    Removing mg32x02z_tm_drv.o(i.TM_IC1OverWritten_Cmd), (20 bytes).
    Removing mg32x02z_tm_drv.o(i.TM_IC2OverWritten_Cmd), (20 bytes).
    Removing mg32x02z_tm_drv.o(i.TM_IC3OverWritten_Cmd), (20 bytes).
    Removing mg32x02z_tm_drv.o(i.TM_IN0Source_Select), (20 bytes).
    Removing mg32x02z_tm_drv.o(i.TM_IN0TriggerEvent_Select), (20 bytes).
    Removing mg32x02z_tm_drv.o(i.TM_IN1Source_Select), (24 bytes).
    Removing mg32x02z_tm_drv.o(i.TM_IN1TriggerEvent_Select), (24 bytes).
    Removing mg32x02z_tm_drv.o(i.TM_IN2Source_Select), (20 bytes).
    Removing mg32x02z_tm_drv.o(i.TM_IN2TriggerEvent_Select), (24 bytes).
    Removing mg32x02z_tm_drv.o(i.TM_IN3Source_Select), (24 bytes).
    Removing mg32x02z_tm_drv.o(i.TM_IN3TriggerEvent_Select), (24 bytes).
    Removing mg32x02z_tm_drv.o(i.TM_ITEA_Cmd), (16 bytes).
    Removing mg32x02z_tm_drv.o(i.TM_ITRx_Select), (16 bytes).
    Removing mg32x02z_tm_drv.o(i.TM_IT_Config), (20 bytes).
    Removing mg32x02z_tm_drv.o(i.TM_InternalBreakEvent_Config), (30 bytes).
    Removing mg32x02z_tm_drv.o(i.TM_InternalClockSource_Select), (16 bytes).
    Removing mg32x02z_tm_drv.o(i.TM_InverseExtTRGI_Cmd), (20 bytes).
    Removing mg32x02z_tm_drv.o(i.TM_InverseOC0H_Cmd), (24 bytes).
    Removing mg32x02z_tm_drv.o(i.TM_InverseOC0N_Cmd), (20 bytes).
    Removing mg32x02z_tm_drv.o(i.TM_InverseOC0z_Cmd), (20 bytes).
    Removing mg32x02z_tm_drv.o(i.TM_InverseOC1H_Cmd), (24 bytes).
    Removing mg32x02z_tm_drv.o(i.TM_InverseOC1N_Cmd), (24 bytes).
    Removing mg32x02z_tm_drv.o(i.TM_InverseOC1z_Cmd), (24 bytes).
    Removing mg32x02z_tm_drv.o(i.TM_InverseOC2H_Cmd), (22 bytes).
    Removing mg32x02z_tm_drv.o(i.TM_InverseOC2N_Cmd), (24 bytes).
    Removing mg32x02z_tm_drv.o(i.TM_InverseOC2_Cmd), (24 bytes).
    Removing mg32x02z_tm_drv.o(i.TM_InverseOC3H_Cmd), (24 bytes).
    Removing mg32x02z_tm_drv.o(i.TM_InverseOC3_Cmd), (24 bytes).
    Removing mg32x02z_tm_drv.o(i.TM_InverseTRGO_Cmd), (20 bytes).
    Removing mg32x02z_tm_drv.o(i.TM_OC00Output_Cmd), (20 bytes).
    Removing mg32x02z_tm_drv.o(i.TM_OC01Output_Cmd), (24 bytes).
    Removing mg32x02z_tm_drv.o(i.TM_OC02Output_Cmd), (24 bytes).
    Removing mg32x02z_tm_drv.o(i.TM_OC0BreakControl_Select), (24 bytes).
    Removing mg32x02z_tm_drv.o(i.TM_OC0HOutputState_Init), (30 bytes).
    Removing mg32x02z_tm_drv.o(i.TM_OC0NBreakStopState_Init), (24 bytes).
    Removing mg32x02z_tm_drv.o(i.TM_OC0NOutput_Cmd), (20 bytes).
    Removing mg32x02z_tm_drv.o(i.TM_OC0zBreakStopState_Init), (20 bytes).
    Removing mg32x02z_tm_drv.o(i.TM_OC0zOutputState_Init), (30 bytes).
    Removing mg32x02z_tm_drv.o(i.TM_OC0zOutput_Cmd), (62 bytes).
    Removing mg32x02z_tm_drv.o(i.TM_OC10Output_Cmd), (24 bytes).
    Removing mg32x02z_tm_drv.o(i.TM_OC11Output_Cmd), (24 bytes).
    Removing mg32x02z_tm_drv.o(i.TM_OC12Output_Cmd), (24 bytes).
    Removing mg32x02z_tm_drv.o(i.TM_OC1BreakControl_Select), (24 bytes).
    Removing mg32x02z_tm_drv.o(i.TM_OC1HOutputState_Init), (36 bytes).
    Removing mg32x02z_tm_drv.o(i.TM_OC1NBreakStopState_Init), (24 bytes).
    Removing mg32x02z_tm_drv.o(i.TM_OC1NOutput_Cmd), (24 bytes).
    Removing mg32x02z_tm_drv.o(i.TM_OC1zBreakStopState_Init), (24 bytes).
    Removing mg32x02z_tm_drv.o(i.TM_OC1zOutputState_Init), (36 bytes).
    Removing mg32x02z_tm_drv.o(i.TM_OC1zOutput_Cmd), (64 bytes).
    Removing mg32x02z_tm_drv.o(i.TM_OC2BreakControl_Select), (24 bytes).
    Removing mg32x02z_tm_drv.o(i.TM_OC2BreakStopState_Init), (24 bytes).
    Removing mg32x02z_tm_drv.o(i.TM_OC2HOutputState_Init), (36 bytes).
    Removing mg32x02z_tm_drv.o(i.TM_OC2NBreakStopState_Init), (24 bytes).
    Removing mg32x02z_tm_drv.o(i.TM_OC2NOutput_Cmd), (20 bytes).
    Removing mg32x02z_tm_drv.o(i.TM_OC2OutputState_Init), (36 bytes).
    Removing mg32x02z_tm_drv.o(i.TM_OC2Output_Cmd), (20 bytes).
    Removing mg32x02z_tm_drv.o(i.TM_OC3BreakControl_Select), (24 bytes).
    Removing mg32x02z_tm_drv.o(i.TM_OC3BreakStopState_Init), (24 bytes).
    Removing mg32x02z_tm_drv.o(i.TM_OC3HOutputState_Init), (36 bytes).
    Removing mg32x02z_tm_drv.o(i.TM_OC3OutputState_Init), (36 bytes).
    Removing mg32x02z_tm_drv.o(i.TM_OC3Output_Cmd), (24 bytes).
    Removing mg32x02z_tm_drv.o(i.TM_PreloadActive_SW), (24 bytes).
    Removing mg32x02z_tm_drv.o(i.TM_PreloadEventSource_Config), (30 bytes).
    Removing mg32x02z_tm_drv.o(i.TM_PreloadOC0z_Config), (22 bytes).
    Removing mg32x02z_tm_drv.o(i.TM_PreloadOC1z_Config), (22 bytes).
    Removing mg32x02z_tm_drv.o(i.TM_PrescalerClock_Select), (20 bytes).
    Removing mg32x02z_tm_drv.o(i.TM_Prescaler_Cmd), (24 bytes).
    Removing mg32x02z_tm_drv.o(i.TM_Prescaler_Config), (6 bytes).
    Removing mg32x02z_tm_drv.o(i.TM_Prescaler_SW), (22 bytes).
    Removing mg32x02z_tm_drv.o(i.TM_ReloadFromCCxB_Cmd), (20 bytes).
    Removing mg32x02z_tm_drv.o(i.TM_ResetCounter_SW), (20 bytes).
    Removing mg32x02z_tm_drv.o(i.TM_ResetPrescaler_SW), (20 bytes).
    Removing mg32x02z_tm_drv.o(i.TM_RisingCaptureIC0_SW), (16 bytes).
    Removing mg32x02z_tm_drv.o(i.TM_RisingCaptureIC1_SW), (20 bytes).
    Removing mg32x02z_tm_drv.o(i.TM_RisingCaptureIC2_SW), (20 bytes).
    Removing mg32x02z_tm_drv.o(i.TM_RisingCaptureIC3_SW), (20 bytes).
    Removing mg32x02z_tm_drv.o(i.TM_SetCC0A), (6 bytes).
    Removing mg32x02z_tm_drv.o(i.TM_SetCC0B), (6 bytes).
    Removing mg32x02z_tm_drv.o(i.TM_SetCC1A), (6 bytes).
    Removing mg32x02z_tm_drv.o(i.TM_SetCC1B), (6 bytes).
    Removing mg32x02z_tm_drv.o(i.TM_SetCC2A), (6 bytes).
    Removing mg32x02z_tm_drv.o(i.TM_SetCC2B), (6 bytes).
    Removing mg32x02z_tm_drv.o(i.TM_SetCC3A), (6 bytes).
    Removing mg32x02z_tm_drv.o(i.TM_SetCC3B), (6 bytes).
    Removing mg32x02z_tm_drv.o(i.TM_SetCounterDirection), (52 bytes).
    Removing mg32x02z_tm_drv.o(i.TM_SetDeadTime), (14 bytes).
    Removing mg32x02z_tm_drv.o(i.TM_SetDeadZoneClockDivider), (16 bytes).
    Removing mg32x02z_tm_drv.o(i.TM_SetInternalClockDivider), (20 bytes).
    Removing mg32x02z_tm_drv.o(i.TM_SetPrescalerDirection), (56 bytes).
    Removing mg32x02z_tm_drv.o(i.TM_TRGICounter_Select), (16 bytes).
    Removing mg32x02z_tm_drv.o(i.TM_TRGIPrescaler_Select), (20 bytes).
    Removing mg32x02z_tm_drv.o(i.TM_TRGOOut_SW), (16 bytes).
    Removing mg32x02z_tm_drv.o(i.TM_TRGO_Select), (20 bytes).
    Removing mg32x02z_tm_drv.o(i.TM_TimeBaseStruct_Init), (26 bytes).
    Removing mg32x02z_tm_drv.o(i.TM_TimeBase_Init), (112 bytes).
    Removing mg32x02z_tm_drv.o(i.TM_TimerMode_Select), (20 bytes).
    Removing mg32x02z_tm_drv.o(i.TM_Timer_Cmd), (24 bytes).
    Removing mg32x02z_tm_drv.o(i.TM_TriggerSource_Select), (20 bytes).
    Removing mg32x02z_tm_drv.o(i.TM_UEV_Cmd), (24 bytes).
    Removing mg32x02z_tm_drv.o(i.TM_UEV_Config), (20 bytes).
    Removing mg32x02z_iwdt_drv.o(.rev16_text), (4 bytes).
    Removing mg32x02z_iwdt_drv.o(.revsh_text), (4 bytes).
    Removing mg32x02z_iwdt_drv.o(i.IWDT_ClearFlag), (8 bytes).
    Removing mg32x02z_iwdt_drv.o(i.IWDT_Cmd), (42 bytes).
    Removing mg32x02z_iwdt_drv.o(i.IWDT_Divider_Select), (26 bytes).
    Removing mg32x02z_iwdt_drv.o(i.IWDT_GetAllFlagStatus), (8 bytes).
    Removing mg32x02z_iwdt_drv.o(i.IWDT_GetCounter), (8 bytes).
    Removing mg32x02z_iwdt_drv.o(i.IWDT_GetSingleFlagStatus), (24 bytes).
    Removing mg32x02z_iwdt_drv.o(i.IWDT_IT_Config), (34 bytes).
    Removing mg32x02z_iwdt_drv.o(i.IWDT_RefreshCounter), (16 bytes).
    Removing mg32x02z_iwdt_drv.o(i.IWDT_StopModeWakeUpEvent_Config), (34 bytes).
    Removing mg32x02z_wwdt_drv.o(.rev16_text), (4 bytes).
    Removing mg32x02z_wwdt_drv.o(.revsh_text), (4 bytes).
    Removing mg32x02z_wwdt_drv.o(i.WWDT_CLK_Select), (28 bytes).
    Removing mg32x02z_wwdt_drv.o(i.WWDT_ClearFlag), (12 bytes).
    Removing mg32x02z_wwdt_drv.o(i.WWDT_Cmd), (40 bytes).
    Removing mg32x02z_wwdt_drv.o(i.WWDT_DIV_Select), (28 bytes).
    Removing mg32x02z_wwdt_drv.o(i.WWDT_GetAllFlagStatus), (12 bytes).
    Removing mg32x02z_wwdt_drv.o(i.WWDT_GetCounter), (12 bytes).
    Removing mg32x02z_wwdt_drv.o(i.WWDT_GetReloadReg), (12 bytes).
    Removing mg32x02z_wwdt_drv.o(i.WWDT_GetSingleFlagStatus), (28 bytes).
    Removing mg32x02z_wwdt_drv.o(i.WWDT_GetWarningThreshold), (12 bytes).
    Removing mg32x02z_wwdt_drv.o(i.WWDT_GetWindowThreshold), (12 bytes).
    Removing mg32x02z_wwdt_drv.o(i.WWDT_IT_Config), (36 bytes).
    Removing mg32x02z_wwdt_drv.o(i.WWDT_PDIV_Select), (24 bytes).
    Removing mg32x02z_wwdt_drv.o(i.WWDT_RefreshCounter), (16 bytes).
    Removing mg32x02z_wwdt_drv.o(i.WWDT_RstEvent_Config), (36 bytes).
    Removing mg32x02z_wwdt_drv.o(i.WWDT_SetReloadReg), (12 bytes).
    Removing mg32x02z_wwdt_drv.o(i.WWDT_SetWarningThreshold), (12 bytes).
    Removing mg32x02z_wwdt_drv.o(i.WWDT_SetWindowThreshold), (12 bytes).
    Removing mg32x02z_rtc_drv.o(.rev16_text), (4 bytes).
    Removing mg32x02z_rtc_drv.o(.revsh_text), (4 bytes).
    Removing mg32x02z_rtc_drv.o(i.RTC_Alarm_Cmd), (36 bytes).
    Removing mg32x02z_rtc_drv.o(i.RTC_CLK_Select), (28 bytes).
    Removing mg32x02z_rtc_drv.o(i.RTC_ClearFlag), (12 bytes).
    Removing mg32x02z_rtc_drv.o(i.RTC_Cmd), (32 bytes).
    Removing mg32x02z_rtc_drv.o(i.RTC_Divider_Select), (28 bytes).
    Removing mg32x02z_rtc_drv.o(i.RTC_GetAlarmCompareValue), (12 bytes).
    Removing mg32x02z_rtc_drv.o(i.RTC_GetAlarmState), (24 bytes).
    Removing mg32x02z_rtc_drv.o(i.RTC_GetAllFlagStatus), (12 bytes).
    Removing mg32x02z_rtc_drv.o(i.RTC_GetCaptureReg), (12 bytes).
    Removing mg32x02z_rtc_drv.o(i.RTC_GetReladReg), (12 bytes).
    Removing mg32x02z_rtc_drv.o(i.RTC_GetSingleFlagStatus), (24 bytes).
    Removing mg32x02z_rtc_drv.o(i.RTC_ITEA_Cmd), (40 bytes).
    Removing mg32x02z_rtc_drv.o(i.RTC_IT_Config), (32 bytes).
    Removing mg32x02z_rtc_drv.o(i.RTC_InitOutputSignalState_Cmd), (40 bytes).
    Removing mg32x02z_rtc_drv.o(i.RTC_OutputSignal_Select), (24 bytes).
    Removing mg32x02z_rtc_drv.o(i.RTC_PreDivider_Select), (28 bytes).
    Removing mg32x02z_rtc_drv.o(i.RTC_RCR_Mode_Select), (28 bytes).
    Removing mg32x02z_rtc_drv.o(i.RTC_SetAlarmCompareValue), (12 bytes).
    Removing mg32x02z_rtc_drv.o(i.RTC_SetReladReg), (12 bytes).
    Removing mg32x02z_rtc_drv.o(i.RTC_StopModeWakeUpEvent_Config), (36 bytes).
    Removing mg32x02z_rtc_drv.o(i.RTC_TriggerStamp_SW), (12 bytes).
    Removing mg32x02z_rtc_drv.o(i.RTC_TriggerStamp_Select), (28 bytes).
    Removing mg32x02z_i2c_drv.o(.rev16_text), (4 bytes).
    Removing mg32x02z_i2c_drv.o(.revsh_text), (4 bytes).
    Removing mg32x02z_i2c_drv.o(i.I2C_ClearEventFlag), (8 bytes).
    Removing mg32x02z_i2c_drv.o(i.I2C_ClearFlag), (4 bytes).
    Removing mg32x02z_i2c_drv.o(i.I2C_Cmd), (24 bytes).
    Removing mg32x02z_i2c_drv.o(i.I2C_GeneralCallAddress_Cmd), (24 bytes).
    Removing mg32x02z_i2c_drv.o(i.I2C_GetAllFlagStatus), (6 bytes).
    Removing mg32x02z_i2c_drv.o(i.I2C_GetEventCode), (12 bytes).
    Removing mg32x02z_i2c_drv.o(i.I2C_GetEventFlag), (22 bytes).
    Removing mg32x02z_i2c_drv.o(i.I2C_GetFlagStatus), (18 bytes).
    Removing mg32x02z_i2c_drv.o(i.I2C_GetITSource), (10 bytes).
    Removing mg32x02z_i2c_drv.o(i.I2C_GetSlaveAddress), (38 bytes).
    Removing mg32x02z_i2c_drv.o(i.I2C_GetSlaveMatchAddress), (6 bytes).
    Removing mg32x02z_i2c_drv.o(i.I2C_ITEA_Cmd), (24 bytes).
    Removing mg32x02z_i2c_drv.o(i.I2C_IT_Config), (20 bytes).
    Removing mg32x02z_i2c_drv.o(i.I2C_ReceiveSBUF), (8 bytes).
    Removing mg32x02z_i2c_drv.o(i.I2C_SendSBUF), (6 bytes).
    Removing mg32x02z_i2c_drv.o(i.I2C_SetClockDivider), (14 bytes).
    Removing mg32x02z_i2c_drv.o(i.I2C_SetClockPrescaler), (16 bytes).
    Removing mg32x02z_i2c_drv.o(i.I2C_SetClockSource), (14 bytes).
    Removing mg32x02z_i2c_drv.o(i.I2C_SetPreDriveTime), (16 bytes).
    Removing mg32x02z_i2c_drv.o(i.I2C_SetSCLHighTime), (4 bytes).
    Removing mg32x02z_i2c_drv.o(i.I2C_SetSCLLowTime), (4 bytes).
    Removing mg32x02z_i2c_drv.o(i.I2C_SetSlaveAddress), (14 bytes).
    Removing mg32x02z_i2c_drv.o(i.I2C_SlaveAddressDetect_Cmd), (20 bytes).
    Removing mg32x02z_spi_drv.o(.rev16_text), (4 bytes).
    Removing mg32x02z_spi_drv.o(.revsh_text), (4 bytes).
    Removing mg32x02z_spi_drv.o(i.SPI_BidirectionalOutput_Cmd), (80 bytes).
    Removing mg32x02z_spi_drv.o(i.SPI_ClearFlag), (4 bytes).
    Removing mg32x02z_spi_drv.o(i.SPI_ClearRxData), (12 bytes).
    Removing mg32x02z_spi_drv.o(i.SPI_ClearTxData), (12 bytes).
    Removing mg32x02z_spi_drv.o(i.SPI_ClockOutputSingnal_Select), (20 bytes).
    Removing mg32x02z_spi_drv.o(i.SPI_ClockPhase_Select), (20 bytes).
    Removing mg32x02z_spi_drv.o(i.SPI_ClockPolarity_Select), (20 bytes).
    Removing mg32x02z_spi_drv.o(i.SPI_Clock_Select), (20 bytes).
    Removing mg32x02z_spi_drv.o(i.SPI_Cmd), (16 bytes).
    Removing mg32x02z_spi_drv.o(i.SPI_DMAReceive_Cmd), (20 bytes).
    Removing mg32x02z_spi_drv.o(i.SPI_DMASend_Cmd), (20 bytes).
    Removing mg32x02z_spi_drv.o(i.SPI_DataLineOutput_Cmd), (26 bytes).
    Removing mg32x02z_spi_drv.o(i.SPI_DataLine_Select), (20 bytes).
    Removing mg32x02z_spi_drv.o(i.SPI_DataSize_Select), (16 bytes).
    Removing mg32x02z_spi_drv.o(i.SPI_DeInit), (32 bytes).
    Removing mg32x02z_spi_drv.o(i.SPI_Divider_Select), (20 bytes).
    Removing mg32x02z_spi_drv.o(i.SPI_FirstBit_Select), (20 bytes).
    Removing mg32x02z_spi_drv.o(i.SPI_GetAllFlagStatus), (8 bytes).
    Removing mg32x02z_spi_drv.o(i.SPI_GetDataBufferReceivedBytes), (10 bytes).
    Removing mg32x02z_spi_drv.o(i.SPI_GetNSSInputStatust), (18 bytes).
    Removing mg32x02z_spi_drv.o(i.SPI_GetRxData), (6 bytes).
    Removing mg32x02z_spi_drv.o(i.SPI_GetRxShadowBufferLevel), (10 bytes).
    Removing mg32x02z_spi_drv.o(i.SPI_GetSingleFlagStatus), (16 bytes).
    Removing mg32x02z_spi_drv.o(i.SPI_GetTxData), (6 bytes).
    Removing mg32x02z_spi_drv.o(i.SPI_GetTxShadowBufferLevel), (10 bytes).
    Removing mg32x02z_spi_drv.o(i.SPI_ITEA_Cmd), (16 bytes).
    Removing mg32x02z_spi_drv.o(i.SPI_IT_Config), (20 bytes).
    Removing mg32x02z_spi_drv.o(i.SPI_LoopBackMode_Cmd), (20 bytes).
    Removing mg32x02z_spi_drv.o(i.SPI_ModeAndNss_Select), (18 bytes).
    Removing mg32x02z_spi_drv.o(i.SPI_ModfHappenedAction_Select), (20 bytes).
    Removing mg32x02z_spi_drv.o(i.SPI_MosiMisoSignalSwap_Cmd), (20 bytes).
    Removing mg32x02z_spi_drv.o(i.SPI_NSSInputSignal_Select), (20 bytes).
    Removing mg32x02z_spi_drv.o(i.SPI_NSSOutputStatusControl_SW), (16 bytes).
    Removing mg32x02z_spi_drv.o(i.SPI_NssInputInverse_Cmd), (20 bytes).
    Removing mg32x02z_spi_drv.o(i.SPI_NssInputOutputSoftwareControl_Cmd), (20 bytes).
    Removing mg32x02z_spi_drv.o(i.SPI_NssOutputInverse_Cmd), (20 bytes).
    Removing mg32x02z_spi_drv.o(i.SPI_PreDivider_Select), (20 bytes).
    Removing mg32x02z_spi_drv.o(i.SPI_Prescaler_Select), (16 bytes).
    Removing mg32x02z_spi_drv.o(i.SPI_SendCopyMode_Cmd), (12 bytes).
    Removing mg32x02z_spi_drv.o(i.SPI_SetDataBufferReceivedBytes), (16 bytes).
    Removing mg32x02z_spi_drv.o(i.SPI_SetTxData), (42 bytes).
    Removing mg32x02z_spi_drv.o(i.SPI_SingleMasterModeNssPulse_Cmd), (14 bytes).
    Removing mg32x02z_spi_drv.o(i.SPI_SlaveModeReceivedThreshold_Select), (16 bytes).
    Removing mg32x02z_spi_drv.o(i.SPI_TransferBidirection_Select), (80 bytes).
    Removing mg32x02z_urt_drv.o(.rev16_text), (4 bytes).
    Removing mg32x02z_urt_drv.o(.revsh_text), (4 bytes).
    Removing mg32x02z_urt_drv.o(i.URT_AutoCalibration_Cmd), (14 bytes).
    Removing mg32x02z_urt_drv.o(i.URT_AutoEnterMuteMode_Select), (6 bytes).
    Removing mg32x02z_urt_drv.o(i.URT_AutoExitMuteMode_Select), (6 bytes).
    Removing mg32x02z_urt_drv.o(i.URT_BaudRateGeneratorClock_Select), (12 bytes).
    Removing mg32x02z_urt_drv.o(i.URT_BaudRateGeneratorMode_Select), (14 bytes).
    Removing mg32x02z_urt_drv.o(i.URT_BreakDisableDMA_Cmd), (16 bytes).
    Removing mg32x02z_urt_drv.o(i.URT_BreakTimeoutDetect_Config), (50 bytes).
    Removing mg32x02z_urt_drv.o(i.URT_CLKSignalSource_Select), (12 bytes).
    Removing mg32x02z_urt_drv.o(i.URT_CLKSignal_Cmd), (14 bytes).
    Removing mg32x02z_urt_drv.o(i.URT_CPHAMode_Select), (12 bytes).
    Removing mg32x02z_urt_drv.o(i.URT_CPOLMode_Select), (12 bytes).
    Removing mg32x02z_urt_drv.o(i.URT_CTSInverse_Cmd), (14 bytes).
    Removing mg32x02z_urt_drv.o(i.URT_CTS_Cmd), (12 bytes).
    Removing mg32x02z_urt_drv.o(i.URT_CalibrationCompleteDataHold_Cmd), (14 bytes).
    Removing mg32x02z_urt_drv.o(i.URT_CalibrationMode_Select), (12 bytes).
    Removing mg32x02z_urt_drv.o(i.URT_CalibrationTimeoutDetect_Config), (48 bytes).
    Removing mg32x02z_urt_drv.o(i.URT_Calibration_SW), (12 bytes).
    Removing mg32x02z_urt_drv.o(i.URT_ClearRXData), (10 bytes).
    Removing mg32x02z_urt_drv.o(i.URT_ClearRxHoldFlag), (6 bytes).
    Removing mg32x02z_urt_drv.o(i.URT_ClearTXData), (10 bytes).
    Removing mg32x02z_urt_drv.o(i.URT_CtrlBROSignalStatus_SW), (20 bytes).
    Removing mg32x02z_urt_drv.o(i.URT_CtrlCLKSignalStatus_SW), (20 bytes).
    Removing mg32x02z_urt_drv.o(i.URT_CtrlNSS_SW), (16 bytes).
    Removing mg32x02z_urt_drv.o(i.URT_CtrlRTS_SW), (14 bytes).
    Removing mg32x02z_urt_drv.o(i.URT_CtrlTMOSignalStatus_SW), (20 bytes).
    Removing mg32x02z_urt_drv.o(i.URT_DEGaurdTime_Select), (14 bytes).
    Removing mg32x02z_urt_drv.o(i.URT_DEInverse_Cmd), (16 bytes).
    Removing mg32x02z_urt_drv.o(i.URT_DE_Cmd), (16 bytes).
    Removing mg32x02z_urt_drv.o(i.URT_ExtraBreakBit_Select), (12 bytes).
    Removing mg32x02z_urt_drv.o(i.URT_GetBaudRateGeneratorCount), (8 bytes).
    Removing mg32x02z_urt_drv.o(i.URT_GetBaudRateGeneratorCountReload), (8 bytes).
    Removing mg32x02z_urt_drv.o(i.URT_GetBaudRateGeneratorPre), (8 bytes).
    Removing mg32x02z_urt_drv.o(i.URT_GetBaudRateGeneratorPreReload), (8 bytes).
    Removing mg32x02z_urt_drv.o(i.URT_GetBreakBusyFlag), (18 bytes).
    Removing mg32x02z_urt_drv.o(i.URT_GetCTSLineStatus), (20 bytes).
    Removing mg32x02z_urt_drv.o(i.URT_GetCaptureData), (8 bytes).
    Removing mg32x02z_urt_drv.o(i.URT_GetCaptureStatusBit), (16 bytes).
    Removing mg32x02z_urt_drv.o(i.URT_GetITAllFlagStatus), (14 bytes).
    Removing mg32x02z_urt_drv.o(i.URT_GetITStatus), (6 bytes).
    Removing mg32x02z_urt_drv.o(i.URT_GetIrDaBusyFlag), (18 bytes).
    Removing mg32x02z_urt_drv.o(i.URT_GetRXData), (6 bytes).
    Removing mg32x02z_urt_drv.o(i.URT_GetRXDataRegLevel), (12 bytes).
    Removing mg32x02z_urt_drv.o(i.URT_GetRXShadowBufferLevel), (10 bytes).
    Removing mg32x02z_urt_drv.o(i.URT_GetRXShiftBufferData), (8 bytes).
    Removing mg32x02z_urt_drv.o(i.URT_GetRXShiftBufferStatusBit), (16 bytes).
    Removing mg32x02z_urt_drv.o(i.URT_GetRxBusyFlag), (18 bytes).
    Removing mg32x02z_urt_drv.o(i.URT_GetRxDifferentFlag), (18 bytes).
    Removing mg32x02z_urt_drv.o(i.URT_GetRxHoldFlag), (18 bytes).
    Removing mg32x02z_urt_drv.o(i.URT_GetRxNoiseFlag), (18 bytes).
    Removing mg32x02z_urt_drv.o(i.URT_GetTXDataRegLevel), (12 bytes).
    Removing mg32x02z_urt_drv.o(i.URT_GetTXShadowBufferLevel), (10 bytes).
    Removing mg32x02z_urt_drv.o(i.URT_GetTXShiftBufferData), (8 bytes).
    Removing mg32x02z_urt_drv.o(i.URT_GetTimeoutTimerCounter), (8 bytes).
    Removing mg32x02z_urt_drv.o(i.URT_GetTimeoutTimerReload), (8 bytes).
    Removing mg32x02z_urt_drv.o(i.URT_GlobalAddress_Cmd), (14 bytes).
    Removing mg32x02z_urt_drv.o(i.URT_HalfDuplexMode_Cmd), (14 bytes).
    Removing mg32x02z_urt_drv.o(i.URT_IdleDetect_Select), (4 bytes).
    Removing mg32x02z_urt_drv.o(i.URT_IdleTimeoutDetect_Config), (32 bytes).
    Removing mg32x02z_urt_drv.o(i.URT_IrDA_Cmd), (12 bytes).
    Removing mg32x02z_urt_drv.o(i.URT_IrDA_Config), (18 bytes).
    Removing mg32x02z_urt_drv.o(i.URT_LoopBackMode_Cmd), (16 bytes).
    Removing mg32x02z_urt_drv.o(i.URT_Mute_Cmd), (12 bytes).
    Removing mg32x02z_urt_drv.o(i.URT_NoiseDataSkip_Cmd), (16 bytes).
    Removing mg32x02z_urt_drv.o(i.URT_NssInverse_Cmd), (16 bytes).
    Removing mg32x02z_urt_drv.o(i.URT_NssSW_Cmd), (16 bytes).
    Removing mg32x02z_urt_drv.o(i.URT_RTSInverse_Cmd), (14 bytes).
    Removing mg32x02z_urt_drv.o(i.URT_RTS_Cmd), (14 bytes).
    Removing mg32x02z_urt_drv.o(i.URT_RXDMA_Cmd), (76 bytes).
    Removing mg32x02z_urt_drv.o(i.URT_RXInverse_Cmd), (16 bytes).
    Removing mg32x02z_urt_drv.o(i.URT_RXParityError_Config), (28 bytes).
    Removing mg32x02z_urt_drv.o(i.URT_RXTimeoutDetect_Config), (32 bytes).
    Removing mg32x02z_urt_drv.o(i.URT_RxTxSwap_Cmd), (16 bytes).
    Removing mg32x02z_urt_drv.o(i.URT_SendAddress), (14 bytes).
    Removing mg32x02z_urt_drv.o(i.URT_SendBreak), (16 bytes).
    Removing mg32x02z_urt_drv.o(i.URT_SetSlaveAddress), (6 bytes).
    Removing mg32x02z_urt_drv.o(i.URT_SetSlaveAddressMask), (6 bytes).
    Removing mg32x02z_urt_drv.o(i.URT_SetTimeoutTimerCompare), (6 bytes).
    Removing mg32x02z_urt_drv.o(i.URT_SetTimeoutTimerCounter), (6 bytes).
    Removing mg32x02z_urt_drv.o(i.URT_TXDMA_Cmd), (72 bytes).
    Removing mg32x02z_urt_drv.o(i.URT_TXErrorDetectMode_Select), (12 bytes).
    Removing mg32x02z_urt_drv.o(i.URT_TXErrorResnedTime_Select), (14 bytes).
    Removing mg32x02z_urt_drv.o(i.URT_TXHalt_Cmd), (14 bytes).
    Removing mg32x02z_urt_drv.o(i.URT_TXInverse_Cmd), (16 bytes).
    Removing mg32x02z_urt_drv.o(i.URT_TimeoutMode_Select), (12 bytes).
    Removing mg32x02z_urt_drv.o(i.URT_TimeoutTimerClockSource_Select), (14 bytes).
    Removing mg32x02z_urt_drv.o(i.URT_TimeroutTimer_Cmd), (12 bytes).
    Removing mg32x02z_urt_drv.o(i.URT_TriggerTimeoutTimerRst_SW), (10 bytes).
    Removing mg32x02z_cm0_drv.o(.rev16_text), (4 bytes).
    Removing mg32x02z_cm0_drv.o(.revsh_text), (4 bytes).
    Removing mg32x02z_cm0_drv.o(i.CM0_GetSysTickCurrentValue), (12 bytes).
    Removing mg32x02z_cm0_drv.o(i.CM0_SysTickClockSource_Select), (36 bytes).
    Removing mg32x02z_cm0_drv.o(i.CM0_SysTickIT_Cmd), (36 bytes).
    Removing mg32x02z_cm0_drv.o(i.CM0_SysTick_Cmd), (36 bytes).
    Removing mg32x02z__irqhandler.o(.rev16_text), (4 bytes).
    Removing mg32x02z__irqhandler.o(.revsh_text), (4 bytes).
    Removing mg32x02z_wwdt_irq.o(.rev16_text), (4 bytes).
    Removing mg32x02z_wwdt_irq.o(.revsh_text), (4 bytes).
    Removing mg32x02z_wwdt_irq.o(i.WWDT_IRQ), (52 bytes).
    Removing mg32x02z_iwdt_irq.o(.rev16_text), (4 bytes).
    Removing mg32x02z_iwdt_irq.o(.revsh_text), (4 bytes).
    Removing mg32x02z_iwdt_irq.o(i.IWDT_IRQ), (78 bytes).
    Removing mg32x02z_pw_irq.o(.rev16_text), (4 bytes).
    Removing mg32x02z_pw_irq.o(.revsh_text), (4 bytes).
    Removing mg32x02z_pw_irq.o(i.PW_IRQ), (66 bytes).
    Removing mg32x02z_rtc_irq.o(.rev16_text), (4 bytes).
    Removing mg32x02z_rtc_irq.o(.revsh_text), (4 bytes).
    Removing mg32x02z_rtc_irq.o(i.RTC_IRQ), (84 bytes).
    Removing mg32x02z_csc_irq.o(.rev16_text), (4 bytes).
    Removing mg32x02z_csc_irq.o(.revsh_text), (4 bytes).
    Removing mg32x02z_csc_irq.o(i.CSC_IRQ), (110 bytes).
    Removing mg32x02z_apb_irq.o(.rev16_text), (4 bytes).
    Removing mg32x02z_apb_irq.o(.revsh_text), (4 bytes).
    Removing mg32x02z_apb_irq.o(i.APB_IRQ), (30 bytes).
    Removing mg32x02z_mem_irq.o(.rev16_text), (4 bytes).
    Removing mg32x02z_mem_irq.o(.revsh_text), (4 bytes).
    Removing mg32x02z_mem_irq.o(i.MEM_IRQ), (2 bytes).
    Removing mg32x02z_exic_irq.o(.rev16_text), (4 bytes).
    Removing mg32x02z_exic_irq.o(.revsh_text), (4 bytes).
    Removing mg32x02z_exic_irq.o(i.EXINT0_IRQ), (56 bytes).
    Removing mg32x02z_exic_irq.o(i.EXINT1_IRQ), (56 bytes).
    Removing mg32x02z_exic_irq.o(i.EXINT2_IRQ), (56 bytes).
    Removing mg32x02z_exic_irq.o(i.EXINT3_IRQ), (56 bytes).
    Removing mg32x02z_cmp_irq.o(.rev16_text), (4 bytes).
    Removing mg32x02z_cmp_irq.o(.revsh_text), (4 bytes).
    Removing mg32x02z_cmp_irq.o(i.CMP_IRQ), (204 bytes).
    Removing mg32x02z_dma_irq.o(.rev16_text), (4 bytes).
    Removing mg32x02z_dma_irq.o(.revsh_text), (4 bytes).
    Removing mg32x02z_dma_irq.o(i.DMA_IRQ), (252 bytes).
    Removing mg32x02z_adc_irq.o(.rev16_text), (4 bytes).
    Removing mg32x02z_adc_irq.o(.revsh_text), (4 bytes).
    Removing mg32x02z_adc_irq.o(i.ADC_IRQ), (286 bytes).
    Removing mg32x02z_dac_irq.o(.rev16_text), (4 bytes).
    Removing mg32x02z_dac_irq.o(.revsh_text), (4 bytes).
    Removing mg32x02z_dac_irq.o(i.DAC_IRQ), (48 bytes).
    Removing mg32x02z_tm00_irq.o(.rev16_text), (4 bytes).
    Removing mg32x02z_tm00_irq.o(.revsh_text), (4 bytes).
    Removing mg32x02z_tm00_irq.o(i.TM00_IRQ), (100 bytes).
    Removing mg32x02z_tm01_irq.o(.rev16_text), (4 bytes).
    Removing mg32x02z_tm01_irq.o(.revsh_text), (4 bytes).
    Removing mg32x02z_tm01_irq.o(i.TM01_IRQ), (88 bytes).
    Removing mg32x02z_tm10_irq.o(.rev16_text), (4 bytes).
    Removing mg32x02z_tm10_irq.o(.revsh_text), (4 bytes).
    Removing mg32x02z_tm10_irq.o(i.TM10_IRQ), (100 bytes).
    Removing mg32x02z_tm16_irq.o(.rev16_text), (4 bytes).
    Removing mg32x02z_tm16_irq.o(.revsh_text), (4 bytes).
    Removing mg32x02z_tm16_irq.o(i.TM16_IRQ), (108 bytes).
    Removing mg32x02z_tm20_irq.o(.rev16_text), (4 bytes).
    Removing mg32x02z_tm20_irq.o(.revsh_text), (4 bytes).
    Removing mg32x02z_tm20_irq.o(i.TM20_IRQ), (204 bytes).
    Removing mg32x02z_tm26_irq.o(.rev16_text), (4 bytes).
    Removing mg32x02z_tm26_irq.o(.revsh_text), (4 bytes).
    Removing mg32x02z_tm26_irq.o(i.TM26_IRQ), (196 bytes).
    Removing mg32x02z_tm36_irq.o(.rev16_text), (4 bytes).
    Removing mg32x02z_tm36_irq.o(.revsh_text), (4 bytes).
    Removing mg32x02z_tm36_irq.o(i.TM36_IRQ), (284 bytes).
    Removing mg32x02z_urt0_irq.o(.rev16_text), (4 bytes).
    Removing mg32x02z_urt0_irq.o(.revsh_text), (4 bytes).
    Removing mg32x02z_urt0_irq.o(i.URT0_IRQ), (480 bytes).
    Removing mg32x02z_urt1_irq.o(.rev16_text), (4 bytes).
    Removing mg32x02z_urt1_irq.o(.revsh_text), (4 bytes).
    Removing mg32x02z_urt1_irq.o(i.URT1_IRQ), (448 bytes).
    Removing mg32x02z_urt2_irq.o(.rev16_text), (4 bytes).
    Removing mg32x02z_urt2_irq.o(.revsh_text), (4 bytes).
    Removing mg32x02z_urt2_irq.o(i.URT2_IRQ), (448 bytes).
    Removing mg32x02z_urt3_irq.o(.rev16_text), (4 bytes).
    Removing mg32x02z_urt3_irq.o(.revsh_text), (4 bytes).
    Removing mg32x02z_urt3_irq.o(i.URT3_IRQ), (448 bytes).
    Removing mg32x02z_spi_irq.o(.rev16_text), (4 bytes).
    Removing mg32x02z_spi_irq.o(.revsh_text), (4 bytes).
    Removing mg32x02z_spi_irq.o(i.SPI0_IRQ), (124 bytes).
    Removing mg32x02z_i2c_irq.o(.rev16_text), (4 bytes).
    Removing mg32x02z_i2c_irq.o(.revsh_text), (4 bytes).
    Removing mg32x02z_i2c_irq.o(i.I2C0_IRQ), (28 bytes).
    Removing mg32x02z_i2c_irq.o(i.I2C1_IRQ), (28 bytes).
    Removing mg32x02z_i2c_irq.o(i.I2C_ByteMode_Event_Handler), (138 bytes).
    Removing mg32x02z_i2c_irq.o(i.I2C_Timeout_Handler), (26 bytes).
    Removing mg32x02z_i2c_irq.o(i.I2C_WakeUp_Handler), (2 bytes).
    Removing startup_mg32x02z.o(HEAP), (512 bytes).
    Removing system_mg32x02z.o(.rev16_text), (4 bytes).
    Removing system_mg32x02z.o(.revsh_text), (4 bytes).
    Removing system_mg32x02z.o(i.SystemCoreClockUpdate), (16 bytes).
    Removing dadd.o(.text), (356 bytes).
    Removing dmul.o(.text), (208 bytes).
    Removing ddiv.o(.text), (240 bytes).
    Removing dfixul.o(.text), (64 bytes).
    Removing cdrcmple.o(.text), (40 bytes).
    Removing depilogue.o(.text), (190 bytes).
    Removing mg32x02z_adc_drv.o(i.__ARM_common_switch8), (28 bytes).
    Removing depilogue.o(i.__ARM_clz), (46 bytes).

813 unused section(s) (total 24194 bytes) removed from the image.

==============================================================================

Image Symbol Table

    Local Symbols

    Symbol Name                              Value     Ov Type        Size  Object(Section)

    RESET                                    0x00000000   Section      192  startup_mg32x02z.o(RESET)
    ../clib/microlib/division.c              0x00000000   Number         0  uldiv.o ABSOLUTE
    ../clib/microlib/division.c              0x00000000   Number         0  uidiv.o ABSOLUTE
    ../clib/microlib/division.c              0x00000000   Number         0  idiv.o ABSOLUTE
    ../clib/microlib/init/entry.s            0x00000000   Number         0  entry10a.o ABSOLUTE
    ../clib/microlib/init/entry.s            0x00000000   Number         0  entry9a.o ABSOLUTE
    ../clib/microlib/init/entry.s            0x00000000   Number         0  entry7b.o ABSOLUTE
    ../clib/microlib/init/entry.s            0x00000000   Number         0  entry7a.o ABSOLUTE
    ../clib/microlib/init/entry.s            0x00000000   Number         0  entry5.o ABSOLUTE
    ../clib/microlib/init/entry.s            0x00000000   Number         0  entry11b.o ABSOLUTE
    ../clib/microlib/init/entry.s            0x00000000   Number         0  entry11a.o ABSOLUTE
    ../clib/microlib/init/entry.s            0x00000000   Number         0  entry10b.o ABSOLUTE
    ../clib/microlib/init/entry.s            0x00000000   Number         0  entry9b.o ABSOLUTE
    ../clib/microlib/init/entry.s            0x00000000   Number         0  entry2.o ABSOLUTE
    ../clib/microlib/init/entry.s            0x00000000   Number         0  entry8b.o ABSOLUTE
    ../clib/microlib/init/entry.s            0x00000000   Number         0  entry8a.o ABSOLUTE
    ../clib/microlib/init/entry.s            0x00000000   Number         0  entry.o ABSOLUTE
    ../clib/microlib/longlong.c              0x00000000   Number         0  llsshr.o ABSOLUTE
    ../clib/microlib/longlong.c              0x00000000   Number         0  llushr.o ABSOLUTE
    ../clib/microlib/longlong.c              0x00000000   Number         0  llshl.o ABSOLUTE
    ../clib/microlib/printf/printf.c         0x00000000   Number         0  printf1.o ABSOLUTE
    ../clib/microlib/printf/printf.c         0x00000000   Number         0  printfa.o ABSOLUTE
    ../clib/microlib/printf/printf.c         0x00000000   Number         0  printf8.o ABSOLUTE
    ../clib/microlib/printf/printf.c         0x00000000   Number         0  printf7.o ABSOLUTE
    ../clib/microlib/printf/printf.c         0x00000000   Number         0  printf6.o ABSOLUTE
    ../clib/microlib/printf/printf.c         0x00000000   Number         0  printf0.o ABSOLUTE
    ../clib/microlib/printf/printf.c         0x00000000   Number         0  printf5.o ABSOLUTE
    ../clib/microlib/printf/printf.c         0x00000000   Number         0  printf4.o ABSOLUTE
    ../clib/microlib/printf/printf.c         0x00000000   Number         0  printf3.o ABSOLUTE
    ../clib/microlib/printf/printf.c         0x00000000   Number         0  printf2.o ABSOLUTE
    ../clib/microlib/printf/printf.c         0x00000000   Number         0  printfb.o ABSOLUTE
    ../clib/microlib/printf/stubs.s          0x00000000   Number         0  stubs.o ABSOLUTE
    ../clib/microlib/stdio/streams.c         0x00000000   Number         0  stdout.o ABSOLUTE
    ../clib/microlib/stubs.s                 0x00000000   Number         0  iusefp.o ABSOLUTE
    ../fplib/microlib/fpadd.c                0x00000000   Number         0  dadd.o ABSOLUTE
    ../fplib/microlib/fpdiv.c                0x00000000   Number         0  ddiv.o ABSOLUTE
    ../fplib/microlib/fpepilogue.c           0x00000000   Number         0  depilogue.o ABSOLUTE
    ../fplib/microlib/fpfix.c                0x00000000   Number         0  dfixul.o ABSOLUTE
    ../fplib/microlib/fpmul.c                0x00000000   Number         0  dmul.o ABSOLUTE
    Drivers\Source\MG32x02z_ADC_DRV.c        0x00000000   Number         0  mg32x02z_adc_drv.o ABSOLUTE
    Drivers\Source\MG32x02z_APB_DRV.c        0x00000000   Number         0  mg32x02z_apb_drv.o ABSOLUTE
    Drivers\Source\MG32x02z_CFG_DRV.c        0x00000000   Number         0  mg32x02z_cfg_drv.o ABSOLUTE
    Drivers\Source\MG32x02z_CM0_DRV.c        0x00000000   Number         0  mg32x02z_cm0_drv.o ABSOLUTE
    Drivers\Source\MG32x02z_CMP_DRV.c        0x00000000   Number         0  mg32x02z_cmp_drv.o ABSOLUTE
    Drivers\Source\MG32x02z_CSC_DRV.c        0x00000000   Number         0  mg32x02z_csc_drv.o ABSOLUTE
    Drivers\Source\MG32x02z_DAC_DRV.c        0x00000000   Number         0  mg32x02z_dac_drv.o ABSOLUTE
    Drivers\Source\MG32x02z_DMA_DRV.c        0x00000000   Number         0  mg32x02z_dma_drv.o ABSOLUTE
    Drivers\Source\MG32x02z_EMB_DRV.c        0x00000000   Number         0  mg32x02z_emb_drv.o ABSOLUTE
    Drivers\Source\MG32x02z_EXIC_DRV.c       0x00000000   Number         0  mg32x02z_exic_drv.o ABSOLUTE
    Drivers\Source\MG32x02z_GPIO_DRV.c       0x00000000   Number         0  mg32x02z_gpio_drv.o ABSOLUTE
    Drivers\Source\MG32x02z_GPL_DRV.c        0x00000000   Number         0  mg32x02z_gpl_drv.o ABSOLUTE
    Drivers\Source\MG32x02z_I2C_DRV.c        0x00000000   Number         0  mg32x02z_i2c_drv.o ABSOLUTE
    Drivers\Source\MG32x02z_IWDT_DRV.c       0x00000000   Number         0  mg32x02z_iwdt_drv.o ABSOLUTE
    Drivers\Source\MG32x02z_MEM_DRV.c        0x00000000   Number         0  mg32x02z_mem_drv.o ABSOLUTE
    Drivers\Source\MG32x02z_PW_DRV.c         0x00000000   Number         0  mg32x02z_pw_drv.o ABSOLUTE
    Drivers\Source\MG32x02z_RST_DRV.c        0x00000000   Number         0  mg32x02z_rst_drv.o ABSOLUTE
    Drivers\Source\MG32x02z_RTC_DRV.c        0x00000000   Number         0  mg32x02z_rtc_drv.o ABSOLUTE
    Drivers\Source\MG32x02z_SPI_DRV.c        0x00000000   Number         0  mg32x02z_spi_drv.o ABSOLUTE
    Drivers\Source\MG32x02z_SYS_DRV.c        0x00000000   Number         0  mg32x02z_sys_drv.o ABSOLUTE
    Drivers\Source\MG32x02z_TM_DRV.c         0x00000000   Number         0  mg32x02z_tm_drv.o ABSOLUTE
    Drivers\Source\MG32x02z_URT_DRV.c        0x00000000   Number         0  mg32x02z_urt_drv.o ABSOLUTE
    Drivers\Source\MG32x02z_WWDT_DRV.c       0x00000000   Number         0  mg32x02z_wwdt_drv.o ABSOLUTE
    Drivers\Source\MG32x02z__Common_DRV.c    0x00000000   Number         0  mg32x02z__common_drv.o ABSOLUTE
    Drivers\\Source\\MG32x02z_ADC_DRV.c      0x00000000   Number         0  mg32x02z_adc_drv.o ABSOLUTE
    Drivers\\Source\\MG32x02z_APB_DRV.c      0x00000000   Number         0  mg32x02z_apb_drv.o ABSOLUTE
    Drivers\\Source\\MG32x02z_CFG_DRV.c      0x00000000   Number         0  mg32x02z_cfg_drv.o ABSOLUTE
    Drivers\\Source\\MG32x02z_CM0_DRV.c      0x00000000   Number         0  mg32x02z_cm0_drv.o ABSOLUTE
    Drivers\\Source\\MG32x02z_CMP_DRV.c      0x00000000   Number         0  mg32x02z_cmp_drv.o ABSOLUTE
    Drivers\\Source\\MG32x02z_CSC_DRV.c      0x00000000   Number         0  mg32x02z_csc_drv.o ABSOLUTE
    Drivers\\Source\\MG32x02z_DAC_DRV.c      0x00000000   Number         0  mg32x02z_dac_drv.o ABSOLUTE
    Drivers\\Source\\MG32x02z_DMA_DRV.c      0x00000000   Number         0  mg32x02z_dma_drv.o ABSOLUTE
    Drivers\\Source\\MG32x02z_EMB_DRV.c      0x00000000   Number         0  mg32x02z_emb_drv.o ABSOLUTE
    Drivers\\Source\\MG32x02z_EXIC_DRV.c     0x00000000   Number         0  mg32x02z_exic_drv.o ABSOLUTE
    Drivers\\Source\\MG32x02z_GPIO_DRV.c     0x00000000   Number         0  mg32x02z_gpio_drv.o ABSOLUTE
    Drivers\\Source\\MG32x02z_GPL_DRV.c      0x00000000   Number         0  mg32x02z_gpl_drv.o ABSOLUTE
    Drivers\\Source\\MG32x02z_I2C_DRV.c      0x00000000   Number         0  mg32x02z_i2c_drv.o ABSOLUTE
    Drivers\\Source\\MG32x02z_IWDT_DRV.c     0x00000000   Number         0  mg32x02z_iwdt_drv.o ABSOLUTE
    Drivers\\Source\\MG32x02z_MEM_DRV.c      0x00000000   Number         0  mg32x02z_mem_drv.o ABSOLUTE
    Drivers\\Source\\MG32x02z_PW_DRV.c       0x00000000   Number         0  mg32x02z_pw_drv.o ABSOLUTE
    Drivers\\Source\\MG32x02z_RST_DRV.c      0x00000000   Number         0  mg32x02z_rst_drv.o ABSOLUTE
    Drivers\\Source\\MG32x02z_RTC_DRV.c      0x00000000   Number         0  mg32x02z_rtc_drv.o ABSOLUTE
    Drivers\\Source\\MG32x02z_SPI_DRV.c      0x00000000   Number         0  mg32x02z_spi_drv.o ABSOLUTE
    Drivers\\Source\\MG32x02z_SYS_DRV.c      0x00000000   Number         0  mg32x02z_sys_drv.o ABSOLUTE
    Drivers\\Source\\MG32x02z_TM_DRV.c       0x00000000   Number         0  mg32x02z_tm_drv.o ABSOLUTE
    Drivers\\Source\\MG32x02z_URT_DRV.c      0x00000000   Number         0  mg32x02z_urt_drv.o ABSOLUTE
    Drivers\\Source\\MG32x02z_WWDT_DRV.c     0x00000000   Number         0  mg32x02z_wwdt_drv.o ABSOLUTE
    Drivers\\Source\\MG32x02z__Common_DRV.c  0x00000000   Number         0  mg32x02z__common_drv.o ABSOLUTE
    RTE\MG32x02z_Device\MG32F02A132\startup_MG32x02z.s 0x00000000   Number         0  startup_mg32x02z.o ABSOLUTE
    RTE\MG32x02z_Device\MG32F02A132\system_MG32x02z.c 0x00000000   Number         0  system_mg32x02z.o ABSOLUTE
    RTE\\MG32x02z_Device\\MG32F02A132\\system_MG32x02z.c 0x00000000   Number         0  system_mg32x02z.o ABSOLUTE
    User\Source\main.c                       0x00000000   Number         0  main.o ABSOLUTE
    User\System\Source\MG32x02z_ADC_IRQ.c    0x00000000   Number         0  mg32x02z_adc_irq.o ABSOLUTE
    User\System\Source\MG32x02z_APB_IRQ.c    0x00000000   Number         0  mg32x02z_apb_irq.o ABSOLUTE
    User\System\Source\MG32x02z_CMP_IRQ.c    0x00000000   Number         0  mg32x02z_cmp_irq.o ABSOLUTE
    User\System\Source\MG32x02z_CSC_IRQ.c    0x00000000   Number         0  mg32x02z_csc_irq.o ABSOLUTE
    User\System\Source\MG32x02z_DAC_IRQ.c    0x00000000   Number         0  mg32x02z_dac_irq.o ABSOLUTE
    User\System\Source\MG32x02z_DMA_IRQ.c    0x00000000   Number         0  mg32x02z_dma_irq.o ABSOLUTE
    User\System\Source\MG32x02z_EXIC_IRQ.c   0x00000000   Number         0  mg32x02z_exic_irq.o ABSOLUTE
    User\System\Source\MG32x02z_I2C_IRQ.c    0x00000000   Number         0  mg32x02z_i2c_irq.o ABSOLUTE
    User\System\Source\MG32x02z_IWDT_IRQ.c   0x00000000   Number         0  mg32x02z_iwdt_irq.o ABSOLUTE
    User\System\Source\MG32x02z_MEM_IRQ.c    0x00000000   Number         0  mg32x02z_mem_irq.o ABSOLUTE
    User\System\Source\MG32x02z_PW_IRQ.c     0x00000000   Number         0  mg32x02z_pw_irq.o ABSOLUTE
    User\System\Source\MG32x02z_RTC_IRQ.c    0x00000000   Number         0  mg32x02z_rtc_irq.o ABSOLUTE
    User\System\Source\MG32x02z_SPI_IRQ.c    0x00000000   Number         0  mg32x02z_spi_irq.o ABSOLUTE
    User\System\Source\MG32x02z_TM00_IRQ.c   0x00000000   Number         0  mg32x02z_tm00_irq.o ABSOLUTE
    User\System\Source\MG32x02z_TM01_IRQ.c   0x00000000   Number         0  mg32x02z_tm01_irq.o ABSOLUTE
    User\System\Source\MG32x02z_TM10_IRQ.c   0x00000000   Number         0  mg32x02z_tm10_irq.o ABSOLUTE
    User\System\Source\MG32x02z_TM16_IRQ.c   0x00000000   Number         0  mg32x02z_tm16_irq.o ABSOLUTE
    User\System\Source\MG32x02z_TM20_IRQ.c   0x00000000   Number         0  mg32x02z_tm20_irq.o ABSOLUTE
    User\System\Source\MG32x02z_TM26_IRQ.c   0x00000000   Number         0  mg32x02z_tm26_irq.o ABSOLUTE
    User\System\Source\MG32x02z_TM36_IRQ.c   0x00000000   Number         0  mg32x02z_tm36_irq.o ABSOLUTE
    User\System\Source\MG32x02z_URT0_IRQ.c   0x00000000   Number         0  mg32x02z_urt0_irq.o ABSOLUTE
    User\System\Source\MG32x02z_URT1_IRQ.c   0x00000000   Number         0  mg32x02z_urt1_irq.o ABSOLUTE
    User\System\Source\MG32x02z_URT2_IRQ.c   0x00000000   Number         0  mg32x02z_urt2_irq.o ABSOLUTE
    User\System\Source\MG32x02z_URT3_IRQ.c   0x00000000   Number         0  mg32x02z_urt3_irq.o ABSOLUTE
    User\System\Source\MG32x02z_WWDT_IRQ.c   0x00000000   Number         0  mg32x02z_wwdt_irq.o ABSOLUTE
    User\System\Source\MG32x02z__IRQHandler.c 0x00000000   Number         0  mg32x02z__irqhandler.o ABSOLUTE
    User\\Source\\main.c                     0x00000000   Number         0  main.o ABSOLUTE
    User\\System\\Source\\MG32x02z_ADC_IRQ.c 0x00000000   Number         0  mg32x02z_adc_irq.o ABSOLUTE
    User\\System\\Source\\MG32x02z_APB_IRQ.c 0x00000000   Number         0  mg32x02z_apb_irq.o ABSOLUTE
    User\\System\\Source\\MG32x02z_CMP_IRQ.c 0x00000000   Number         0  mg32x02z_cmp_irq.o ABSOLUTE
    User\\System\\Source\\MG32x02z_CSC_IRQ.c 0x00000000   Number         0  mg32x02z_csc_irq.o ABSOLUTE
    User\\System\\Source\\MG32x02z_DAC_IRQ.c 0x00000000   Number         0  mg32x02z_dac_irq.o ABSOLUTE
    User\\System\\Source\\MG32x02z_DMA_IRQ.c 0x00000000   Number         0  mg32x02z_dma_irq.o ABSOLUTE
    User\\System\\Source\\MG32x02z_EXIC_IRQ.c 0x00000000   Number         0  mg32x02z_exic_irq.o ABSOLUTE
    User\\System\\Source\\MG32x02z_I2C_IRQ.c 0x00000000   Number         0  mg32x02z_i2c_irq.o ABSOLUTE
    User\\System\\Source\\MG32x02z_IWDT_IRQ.c 0x00000000   Number         0  mg32x02z_iwdt_irq.o ABSOLUTE
    User\\System\\Source\\MG32x02z_MEM_IRQ.c 0x00000000   Number         0  mg32x02z_mem_irq.o ABSOLUTE
    User\\System\\Source\\MG32x02z_PW_IRQ.c  0x00000000   Number         0  mg32x02z_pw_irq.o ABSOLUTE
    User\\System\\Source\\MG32x02z_RTC_IRQ.c 0x00000000   Number         0  mg32x02z_rtc_irq.o ABSOLUTE
    User\\System\\Source\\MG32x02z_SPI_IRQ.c 0x00000000   Number         0  mg32x02z_spi_irq.o ABSOLUTE
    User\\System\\Source\\MG32x02z_TM00_IRQ.c 0x00000000   Number         0  mg32x02z_tm00_irq.o ABSOLUTE
    User\\System\\Source\\MG32x02z_TM01_IRQ.c 0x00000000   Number         0  mg32x02z_tm01_irq.o ABSOLUTE
    User\\System\\Source\\MG32x02z_TM10_IRQ.c 0x00000000   Number         0  mg32x02z_tm10_irq.o ABSOLUTE
    User\\System\\Source\\MG32x02z_TM16_IRQ.c 0x00000000   Number         0  mg32x02z_tm16_irq.o ABSOLUTE
    User\\System\\Source\\MG32x02z_TM20_IRQ.c 0x00000000   Number         0  mg32x02z_tm20_irq.o ABSOLUTE
    User\\System\\Source\\MG32x02z_TM26_IRQ.c 0x00000000   Number         0  mg32x02z_tm26_irq.o ABSOLUTE
    User\\System\\Source\\MG32x02z_TM36_IRQ.c 0x00000000   Number         0  mg32x02z_tm36_irq.o ABSOLUTE
    User\\System\\Source\\MG32x02z_URT0_IRQ.c 0x00000000   Number         0  mg32x02z_urt0_irq.o ABSOLUTE
    User\\System\\Source\\MG32x02z_URT1_IRQ.c 0x00000000   Number         0  mg32x02z_urt1_irq.o ABSOLUTE
    User\\System\\Source\\MG32x02z_URT2_IRQ.c 0x00000000   Number         0  mg32x02z_urt2_irq.o ABSOLUTE
    User\\System\\Source\\MG32x02z_URT3_IRQ.c 0x00000000   Number         0  mg32x02z_urt3_irq.o ABSOLUTE
    User\\System\\Source\\MG32x02z_WWDT_IRQ.c 0x00000000   Number         0  mg32x02z_wwdt_irq.o ABSOLUTE
    User\\System\\Source\\MG32x02z__IRQHandler.c 0x00000000   Number         0  mg32x02z__irqhandler.o ABSOLUTE
    cdrcmple.s                               0x00000000   Number         0  cdrcmple.o ABSOLUTE
    dc.s                                     0x00000000   Number         0  dc.o ABSOLUTE
    handlers.s                               0x00000000   Number         0  handlers.o ABSOLUTE
    init.s                                   0x00000000   Number         0  init.o ABSOLUTE
    .ARM.Collect$$$$00000000                 0x000000c0   Section        0  entry.o(.ARM.Collect$$$$00000000)
    .ARM.Collect$$$$00000001                 0x000000c0   Section        4  entry2.o(.ARM.Collect$$$$00000001)
    .ARM.Collect$$$$00000004                 0x000000c4   Section        4  entry5.o(.ARM.Collect$$$$00000004)
    .ARM.Collect$$$$00000008                 0x000000c8   Section        0  entry7b.o(.ARM.Collect$$$$00000008)
    .ARM.Collect$$$$0000000A                 0x000000c8   Section        0  entry8b.o(.ARM.Collect$$$$0000000A)
    .ARM.Collect$$$$0000000B                 0x000000c8   Section        8  entry9a.o(.ARM.Collect$$$$0000000B)
    .ARM.Collect$$$$0000000D                 0x000000d0   Section        0  entry10a.o(.ARM.Collect$$$$0000000D)
    .ARM.Collect$$$$0000000F                 0x000000d0   Section        0  entry11a.o(.ARM.Collect$$$$0000000F)
    .ARM.Collect$$$$00002712                 0x000000d0   Section        4  entry2.o(.ARM.Collect$$$$00002712)
    __lit__00000000                          0x000000d0   Data           4  entry2.o(.ARM.Collect$$$$00002712)
    .text                                    0x000000d4   Section       36  startup_mg32x02z.o(.text)
    .text                                    0x000000f8   Section        0  uldiv.o(.text)
    .text                                    0x00000158   Section       36  init.o(.text)
    .text                                    0x0000017c   Section        0  llshl.o(.text)
    .text                                    0x0000019c   Section        0  llushr.o(.text)
    i.CSC_CK_AHB_Divider_Select              0x000001c0   Section        0  mg32x02z_csc_drv.o(i.CSC_CK_AHB_Divider_Select)
    i.CSC_CK_APB_Divider_Select              0x000001dc   Section        0  mg32x02z_csc_drv.o(i.CSC_CK_APB_Divider_Select)
    i.CSC_CK_HS_Select                       0x000001f8   Section        0  mg32x02z_csc_drv.o(i.CSC_CK_HS_Select)
    i.CSC_CK_MAIN_Select                     0x00000218   Section        0  mg32x02z_csc_drv.o(i.CSC_CK_MAIN_Select)
    i.CSC_ClearFlag                          0x00000238   Section        0  mg32x02z_csc_drv.o(i.CSC_ClearFlag)
    i.CSC_GetSingleFlagStatus                0x00000244   Section        0  mg32x02z_csc_drv.o(i.CSC_GetSingleFlagStatus)
    i.CSC_IHRCO_Cmd                          0x00000260   Section        0  mg32x02z_csc_drv.o(i.CSC_IHRCO_Cmd)
    i.CSC_IHRCO_Select                       0x00000284   Section        0  mg32x02z_csc_drv.o(i.CSC_IHRCO_Select)
    i.CSC_Init                               0x000002a8   Section        0  main.o(i.CSC_Init)
    i.CSC_PLL_Cmd                            0x00000334   Section        0  mg32x02z_csc_drv.o(i.CSC_PLL_Cmd)
    i.CSC_PLL_Config                         0x00000358   Section        0  mg32x02z_csc_drv.o(i.CSC_PLL_Config)
    i.CSC_PeriphOnModeClock_Config           0x00000388   Section        0  mg32x02z_csc_drv.o(i.CSC_PeriphOnModeClock_Config)
    i.CSC_PeriphProcessClockSource_Config    0x00000430   Section        0  mg32x02z_csc_drv.o(i.CSC_PeriphProcessClockSource_Config)
    i.DMA_AutoIncreaseDestinationAddress     0x000004cc   Section        0  mg32x02z_dma_drv.o(i.DMA_AutoIncreaseDestinationAddress)
    i.DMA_AutoIncreaseSourceAddress          0x000004e0   Section        0  mg32x02z_dma_drv.o(i.DMA_AutoIncreaseSourceAddress)
    i.DMA_BaseInitStructure_Init             0x000004f0   Section        0  mg32x02z_dma_drv.o(i.DMA_BaseInitStructure_Init)
    i.DMA_Base_Init                          0x00000524   Section        0  mg32x02z_dma_drv.o(i.DMA_Base_Init)
    i.DMA_Channel_Cmd                        0x0000058e   Section        0  mg32x02z_dma_drv.o(i.DMA_Channel_Cmd)
    i.DMA_ClearFlag                          0x0000059e   Section        0  mg32x02z_dma_drv.o(i.DMA_ClearFlag)
    i.DMA_Cmd                                0x000005a4   Section        0  mg32x02z_dma_drv.o(i.DMA_Cmd)
    i.DMA_Destination_Select                 0x000005bc   Section        0  mg32x02z_dma_drv.o(i.DMA_Destination_Select)
    i.DMA_GetSingleFlagStatus                0x000005cc   Section        0  mg32x02z_dma_drv.o(i.DMA_GetSingleFlagStatus)
    i.DMA_Init                               0x000005e0   Section        0  main.o(i.DMA_Init)
    i.DMA_LoopMode_Cmd                       0x0000064c   Section        0  mg32x02z_dma_drv.o(i.DMA_LoopMode_Cmd)
    i.DMA_SetBurstSize                       0x00000660   Section        0  mg32x02z_dma_drv.o(i.DMA_SetBurstSize)
    i.DMA_SetDestinationAddress              0x00000674   Section        0  mg32x02z_dma_drv.o(i.DMA_SetDestinationAddress)
    i.DMA_SetExtTriggerMode                  0x00000678   Section        0  mg32x02z_dma_drv.o(i.DMA_SetExtTriggerMode)
    i.DMA_SetExtTriggerPin                   0x00000688   Section        0  mg32x02z_dma_drv.o(i.DMA_SetExtTriggerPin)
    i.DMA_SetSourceAddress                   0x00000698   Section        0  mg32x02z_dma_drv.o(i.DMA_SetSourceAddress)
    i.DMA_SetTransferDataNumber              0x0000069c   Section        0  mg32x02z_dma_drv.o(i.DMA_SetTransferDataNumber)
    i.DMA_Source_Select                      0x000006a0   Section        0  mg32x02z_dma_drv.o(i.DMA_Source_Select)
    i.DMA_StartRequest                       0x000006b0   Section        0  mg32x02z_dma_drv.o(i.DMA_StartRequest)
    i.GPIO_PinMode_Config                    0x000006bc   Section        0  mg32x02z_gpio_drv.o(i.GPIO_PinMode_Config)
    i.GPL_CRC_Check                          0x000006e4   Section        0  main.o(i.GPL_CRC_Check)
    i.GPL_CRC_Config                         0x000017c4   Section        0  main.o(i.GPL_CRC_Config)
    i.GPL_DMA_Cmd                            0x00001804   Section        0  mg32x02z_gpl_drv.o(i.GPL_DMA_Cmd)
    i.MEM_SetFlashWaitState                  0x0000182c   Section        0  mg32x02z_mem_drv.o(i.MEM_SetFlashWaitState)
    i.ProtectModuleReg                       0x00001858   Section        0  mg32x02z__common_drv.o(i.ProtectModuleReg)
    i.Sample_URT0_Init                       0x0000186c   Section        0  main.o(i.Sample_URT0_Init)
    i.SystemInit                             0x000019d0   Section        0  system_mg32x02z.o(i.SystemInit)
    i.URT_BaudRateGenerator_Cmd              0x000019e0   Section        0  mg32x02z_urt_drv.o(i.URT_BaudRateGenerator_Cmd)
    i.URT_BaudRateGenerator_Config           0x000019f0   Section        0  mg32x02z_urt_drv.o(i.URT_BaudRateGenerator_Config)
    i.URT_ClearITFlag                        0x00001a14   Section        0  mg32x02z_urt_drv.o(i.URT_ClearITFlag)
    i.URT_Cmd                                0x00001a1e   Section        0  mg32x02z_urt_drv.o(i.URT_Cmd)
    i.URT_DataCharacter_Config               0x00001a2a   Section        0  mg32x02z_urt_drv.o(i.URT_DataCharacter_Config)
    i.URT_DataLine_Select                    0x00001a6a   Section        0  mg32x02z_urt_drv.o(i.URT_DataLine_Select)
    i.URT_GetITSingleFlagStatus              0x00001a78   Section        0  mg32x02z_urt_drv.o(i.URT_GetITSingleFlagStatus)
    i.URT_ITEA_Cmd                           0x00001a98   Section        0  mg32x02z_urt_drv.o(i.URT_ITEA_Cmd)
    i.URT_IT_Cmd                             0x00001aa4   Section        0  mg32x02z_urt_drv.o(i.URT_IT_Cmd)
    i.URT_IdlehandleMode_Select              0x00001ab4   Section        0  mg32x02z_urt_drv.o(i.URT_IdlehandleMode_Select)
    i.URT_Mode_Select                        0x00001ac2   Section        0  mg32x02z_urt_drv.o(i.URT_Mode_Select)
    i.URT_RXClockSource_Select               0x00001ae8   Section        0  mg32x02z_urt_drv.o(i.URT_RXClockSource_Select)
    i.URT_RXOverSamplingMode_Select          0x00001af6   Section        0  mg32x02z_urt_drv.o(i.URT_RXOverSamplingMode_Select)
    i.URT_RXOverSamplingSampleNumber_Select  0x00001b02   Section        0  mg32x02z_urt_drv.o(i.URT_RXOverSamplingSampleNumber_Select)
    i.URT_RXShadowBufferThreshold_Select     0x00001b12   Section        0  mg32x02z_urt_drv.o(i.URT_RXShadowBufferThreshold_Select)
    i.URT_RX_Cmd                             0x00001b20   Section        0  mg32x02z_urt_drv.o(i.URT_RX_Cmd)
    i.URT_SetTXData                          0x00001b2e   Section        0  mg32x02z_urt_drv.o(i.URT_SetTXData)
    i.URT_TXClockSource_Select               0x00001b60   Section        0  mg32x02z_urt_drv.o(i.URT_TXClockSource_Select)
    i.URT_TXGaudTime_Select                  0x00001b6e   Section        0  mg32x02z_urt_drv.o(i.URT_TXGaudTime_Select)
    i.URT_TXOverSamplingSampleNumber_Select  0x00001b72   Section        0  mg32x02z_urt_drv.o(i.URT_TXOverSamplingSampleNumber_Select)
    i.URT_TX_Cmd                             0x00001b82   Section        0  mg32x02z_urt_drv.o(i.URT_TX_Cmd)
    i.UnProtectModuleReg                     0x00001b90   Section        0  mg32x02z__common_drv.o(i.UnProtectModuleReg)
    i.__0printf$8                            0x00001ba8   Section        0  printf8.o(i.__0printf$8)
    i.__scatterload_copy                     0x00001bc8   Section       14  handlers.o(i.__scatterload_copy)
    i.__scatterload_null                     0x00001bd6   Section        2  handlers.o(i.__scatterload_null)
    i.__scatterload_zeroinit                 0x00001bd8   Section       14  handlers.o(i.__scatterload_zeroinit)
    i._printf_core                           0x00001be8   Section        0  printf8.o(i._printf_core)
    _printf_core                             0x00001be9   Thumb Code  1020  printf8.o(i._printf_core)
    i._printf_post_padding                   0x00002010   Section        0  printf8.o(i._printf_post_padding)
    _printf_post_padding                     0x00002011   Thumb Code    32  printf8.o(i._printf_post_padding)
    i._printf_pre_padding                    0x00002030   Section        0  printf8.o(i._printf_pre_padding)
    _printf_pre_padding                      0x00002031   Thumb Code    44  printf8.o(i._printf_pre_padding)
    i.fputc                                  0x0000205c   Section        0  main.o(i.fputc)
    i.main                                   0x0000208c   Section        0  main.o(i.main)
    .conststring                             0x000020c4   Section     1113  main.o(.conststring)
    .data                                    0x20000000   Section        9  main.o(.data)
    .data                                    0x2000000c   Section        4  system_mg32x02z.o(.data)
    .data                                    0x20000010   Section        4  stdout.o(.data)
    STACK                                    0x20000018   Section     1024  startup_mg32x02z.o(STACK)

    Global Symbols

    Symbol Name                              Value     Ov Type        Size  Object(Section)

    BuildAttributes$$THM_ISAv3M$S$PE$A:L22$X:L11$S22$IEEE1$IW$USESV6$~STKCKD$USESV7$~SHL$OSPACE$ROPI$EBA8$MICROLIB$REQ8$PRES8$EABIv2 0x00000000   Number         0  anon$$obj.o ABSOLUTE
    __ARM_use_no_argv                        0x00000000   Number         0  main.o ABSOLUTE
    __Vectors                                0x00000000   Data           4  startup_mg32x02z.o(RESET)
    _printf_a                                0x00000000   Number         0  stubs.o ABSOLUTE
    _printf_c                                0x00000000   Number         0  stubs.o ABSOLUTE
    _printf_charcount                        0x00000000   Number         0  stubs.o ABSOLUTE
    _printf_d                                0x00000000   Number         0  stubs.o ABSOLUTE
    _printf_e                                0x00000000   Number         0  stubs.o ABSOLUTE
    _printf_f                                0x00000000   Number         0  stubs.o ABSOLUTE
    _printf_flags                            0x00000000   Number         0  stubs.o ABSOLUTE
    _printf_fp_dec                           0x00000000   Number         0  stubs.o ABSOLUTE
    _printf_fp_hex                           0x00000000   Number         0  stubs.o ABSOLUTE
    _printf_g                                0x00000000   Number         0  stubs.o ABSOLUTE
    _printf_i                                0x00000000   Number         0  stubs.o ABSOLUTE
    _printf_int_dec                          0x00000000   Number         0  stubs.o ABSOLUTE
    _printf_l                                0x00000000   Number         0  stubs.o ABSOLUTE
    _printf_lc                               0x00000000   Number         0  stubs.o ABSOLUTE
    _printf_ll                               0x00000000   Number         0  stubs.o ABSOLUTE
    _printf_lld                              0x00000000   Number         0  stubs.o ABSOLUTE
    _printf_lli                              0x00000000   Number         0  stubs.o ABSOLUTE
    _printf_llo                              0x00000000   Number         0  stubs.o ABSOLUTE
    _printf_llu                              0x00000000   Number         0  stubs.o ABSOLUTE
    _printf_llx                              0x00000000   Number         0  stubs.o ABSOLUTE
    _printf_longlong_dec                     0x00000000   Number         0  stubs.o ABSOLUTE
    _printf_longlong_hex                     0x00000000   Number         0  stubs.o ABSOLUTE
    _printf_longlong_oct                     0x00000000   Number         0  stubs.o ABSOLUTE
    _printf_ls                               0x00000000   Number         0  stubs.o ABSOLUTE
    _printf_mbtowc                           0x00000000   Number         0  stubs.o ABSOLUTE
    _printf_n                                0x00000000   Number         0  stubs.o ABSOLUTE
    _printf_o                                0x00000000   Number         0  stubs.o ABSOLUTE
    _printf_p                                0x00000000   Number         0  stubs.o ABSOLUTE
    _printf_percent                          0x00000000   Number         0  stubs.o ABSOLUTE
    _printf_pre_padding                      0x00000000   Number         0  stubs.o ABSOLUTE
    _printf_return_value                     0x00000000   Number         0  stubs.o ABSOLUTE
    _printf_s                                0x00000000   Number         0  stubs.o ABSOLUTE
    _printf_sizespec                         0x00000000   Number         0  stubs.o ABSOLUTE
    _printf_str                              0x00000000   Number         0  stubs.o ABSOLUTE
    _printf_truncate_signed                  0x00000000   Number         0  stubs.o ABSOLUTE
    _printf_truncate_unsigned                0x00000000   Number         0  stubs.o ABSOLUTE
    _printf_u                                0x00000000   Number         0  stubs.o ABSOLUTE
    _printf_wc                               0x00000000   Number         0  stubs.o ABSOLUTE
    _printf_wctomb                           0x00000000   Number         0  stubs.o ABSOLUTE
    _printf_widthprec                        0x00000000   Number         0  stubs.o ABSOLUTE
    _printf_x                                0x00000000   Number         0  stubs.o ABSOLUTE
    __cpp_initialize__aeabi_                  - Undefined Weak Reference
    __cxa_finalize                            - Undefined Weak Reference
    __decompress                              - Undefined Weak Reference
    _clock_init                               - Undefined Weak Reference
    _microlib_exit                            - Undefined Weak Reference
    __Vectors_End                            0x000000c0   Data           0  startup_mg32x02z.o(RESET)
    __Vectors_Size                           0x000000c0   Number         0  startup_mg32x02z.o ABSOLUTE
    __main                                   0x000000c1   Thumb Code     0  entry.o(.ARM.Collect$$$$00000000)
    _main_stk                                0x000000c1   Thumb Code     0  entry2.o(.ARM.Collect$$$$00000001)
    _main_scatterload                        0x000000c5   Thumb Code     0  entry5.o(.ARM.Collect$$$$00000004)
    __main_after_scatterload                 0x000000c9   Thumb Code     0  entry5.o(.ARM.Collect$$$$00000004)
    _main_clock                              0x000000c9   Thumb Code     0  entry7b.o(.ARM.Collect$$$$00000008)
    _main_cpp_init                           0x000000c9   Thumb Code     0  entry8b.o(.ARM.Collect$$$$0000000A)
    _main_init                               0x000000c9   Thumb Code     0  entry9a.o(.ARM.Collect$$$$0000000B)
    __rt_final_cpp                           0x000000d1   Thumb Code     0  entry10a.o(.ARM.Collect$$$$0000000D)
    __rt_final_exit                          0x000000d1   Thumb Code     0  entry11a.o(.ARM.Collect$$$$0000000F)
    MG32x02z_IEC60730_MANAGER                0x000000d5   Thumb Code     0  startup_mg32x02z.o(.text)
    ReInitial_Stack                          0x000000d5   Thumb Code     6  startup_mg32x02z.o(.text)
    Reset_Handler                            0x000000db   Thumb Code     8  startup_mg32x02z.o(.text)
    NMI_Handler                              0x000000e3   Thumb Code     2  startup_mg32x02z.o(.text)
    HardFault_Handler                        0x000000e5   Thumb Code     2  startup_mg32x02z.o(.text)
    SVC_Handler                              0x000000e7   Thumb Code     2  startup_mg32x02z.o(.text)
    PendSV_Handler                           0x000000e9   Thumb Code     2  startup_mg32x02z.o(.text)
    SysTick_Handler                          0x000000eb   Thumb Code     2  startup_mg32x02z.o(.text)
    ADC_IRQHandler                           0x000000ed   Thumb Code     0  startup_mg32x02z.o(.text)
    COMP_IRQHandler                          0x000000ed   Thumb Code     0  startup_mg32x02z.o(.text)
    DAC_IRQHandler                           0x000000ed   Thumb Code     0  startup_mg32x02z.o(.text)
    DMA_IRQHandler                           0x000000ed   Thumb Code     0  startup_mg32x02z.o(.text)
    EXINT0_IRQHandler                        0x000000ed   Thumb Code     0  startup_mg32x02z.o(.text)
    EXINT1_IRQHandler                        0x000000ed   Thumb Code     0  startup_mg32x02z.o(.text)
    EXINT2_IRQHandler                        0x000000ed   Thumb Code     0  startup_mg32x02z.o(.text)
    EXINT3_IRQHandler                        0x000000ed   Thumb Code     0  startup_mg32x02z.o(.text)
    I2C0_IRQHandler                          0x000000ed   Thumb Code     0  startup_mg32x02z.o(.text)
    I2Cx_IRQHandler                          0x000000ed   Thumb Code     0  startup_mg32x02z.o(.text)
    SPI0_IRQHandler                          0x000000ed   Thumb Code     0  startup_mg32x02z.o(.text)
    SYS_IRQHandler                           0x000000ed   Thumb Code     0  startup_mg32x02z.o(.text)
    TM0x_IRQHandler                          0x000000ed   Thumb Code     0  startup_mg32x02z.o(.text)
    TM10_IRQHandler                          0x000000ed   Thumb Code     0  startup_mg32x02z.o(.text)
    TM1x_IRQHandler                          0x000000ed   Thumb Code     0  startup_mg32x02z.o(.text)
    TM20_IRQHandler                          0x000000ed   Thumb Code     0  startup_mg32x02z.o(.text)
    TM2x_IRQHandler                          0x000000ed   Thumb Code     0  startup_mg32x02z.o(.text)
    TM3x_IRQHandler                          0x000000ed   Thumb Code     0  startup_mg32x02z.o(.text)
    URT0_IRQHandler                          0x000000ed   Thumb Code     0  startup_mg32x02z.o(.text)
    URT123_IRQHandler                        0x000000ed   Thumb Code     0  startup_mg32x02z.o(.text)
    WWDT_IRQHandler                          0x000000ed   Thumb Code     0  startup_mg32x02z.o(.text)
    __aeabi_uldivmod                         0x000000f9   Thumb Code    96  uldiv.o(.text)
    __scatterload                            0x00000159   Thumb Code    28  init.o(.text)
    __scatterload_rt2                        0x00000159   Thumb Code     0  init.o(.text)
    __aeabi_llsl                             0x0000017d   Thumb Code    32  llshl.o(.text)
    _ll_shift_l                              0x0000017d   Thumb Code     0  llshl.o(.text)
    __aeabi_llsr                             0x0000019d   Thumb Code    34  llushr.o(.text)
    _ll_ushift_r                             0x0000019d   Thumb Code     0  llushr.o(.text)
    CSC_CK_AHB_Divider_Select                0x000001c1   Thumb Code    22  mg32x02z_csc_drv.o(i.CSC_CK_AHB_Divider_Select)
    CSC_CK_APB_Divider_Select                0x000001dd   Thumb Code    22  mg32x02z_csc_drv.o(i.CSC_CK_APB_Divider_Select)
    CSC_CK_HS_Select                         0x000001f9   Thumb Code    26  mg32x02z_csc_drv.o(i.CSC_CK_HS_Select)
    CSC_CK_MAIN_Select                       0x00000219   Thumb Code    26  mg32x02z_csc_drv.o(i.CSC_CK_MAIN_Select)
    CSC_ClearFlag                            0x00000239   Thumb Code     6  mg32x02z_csc_drv.o(i.CSC_ClearFlag)
    CSC_GetSingleFlagStatus                  0x00000245   Thumb Code    22  mg32x02z_csc_drv.o(i.CSC_GetSingleFlagStatus)
    CSC_IHRCO_Cmd                            0x00000261   Thumb Code    30  mg32x02z_csc_drv.o(i.CSC_IHRCO_Cmd)
    CSC_IHRCO_Select                         0x00000285   Thumb Code    30  mg32x02z_csc_drv.o(i.CSC_IHRCO_Select)
    CSC_Init                                 0x000002a9   Thumb Code   132  main.o(i.CSC_Init)
    CSC_PLL_Cmd                              0x00000335   Thumb Code    32  mg32x02z_csc_drv.o(i.CSC_PLL_Cmd)
    CSC_PLL_Config                           0x00000359   Thumb Code    42  mg32x02z_csc_drv.o(i.CSC_PLL_Config)
    CSC_PeriphOnModeClock_Config             0x00000389   Thumb Code   164  mg32x02z_csc_drv.o(i.CSC_PeriphOnModeClock_Config)
    CSC_PeriphProcessClockSource_Config      0x00000431   Thumb Code   150  mg32x02z_csc_drv.o(i.CSC_PeriphProcessClockSource_Config)
    DMA_AutoIncreaseDestinationAddress       0x000004cd   Thumb Code    20  mg32x02z_dma_drv.o(i.DMA_AutoIncreaseDestinationAddress)
    DMA_AutoIncreaseSourceAddress            0x000004e1   Thumb Code    16  mg32x02z_dma_drv.o(i.DMA_AutoIncreaseSourceAddress)
    DMA_BaseInitStructure_Init               0x000004f1   Thumb Code    44  mg32x02z_dma_drv.o(i.DMA_BaseInitStructure_Init)
    DMA_Base_Init                            0x00000525   Thumb Code   106  mg32x02z_dma_drv.o(i.DMA_Base_Init)
    DMA_Channel_Cmd                          0x0000058f   Thumb Code    16  mg32x02z_dma_drv.o(i.DMA_Channel_Cmd)
    DMA_ClearFlag                            0x0000059f   Thumb Code     4  mg32x02z_dma_drv.o(i.DMA_ClearFlag)
    DMA_Cmd                                  0x000005a5   Thumb Code    20  mg32x02z_dma_drv.o(i.DMA_Cmd)
    DMA_Destination_Select                   0x000005bd   Thumb Code    16  mg32x02z_dma_drv.o(i.DMA_Destination_Select)
    DMA_GetSingleFlagStatus                  0x000005cd   Thumb Code    18  mg32x02z_dma_drv.o(i.DMA_GetSingleFlagStatus)
    DMA_Init                                 0x000005e1   Thumb Code    94  main.o(i.DMA_Init)
    DMA_LoopMode_Cmd                         0x0000064d   Thumb Code    20  mg32x02z_dma_drv.o(i.DMA_LoopMode_Cmd)
    DMA_SetBurstSize                         0x00000661   Thumb Code    20  mg32x02z_dma_drv.o(i.DMA_SetBurstSize)
    DMA_SetDestinationAddress                0x00000675   Thumb Code     4  mg32x02z_dma_drv.o(i.DMA_SetDestinationAddress)
    DMA_SetExtTriggerMode                    0x00000679   Thumb Code    16  mg32x02z_dma_drv.o(i.DMA_SetExtTriggerMode)
    DMA_SetExtTriggerPin                     0x00000689   Thumb Code    16  mg32x02z_dma_drv.o(i.DMA_SetExtTriggerPin)
    DMA_SetSourceAddress                     0x00000699   Thumb Code     4  mg32x02z_dma_drv.o(i.DMA_SetSourceAddress)
    DMA_SetTransferDataNumber                0x0000069d   Thumb Code     4  mg32x02z_dma_drv.o(i.DMA_SetTransferDataNumber)
    DMA_Source_Select                        0x000006a1   Thumb Code    16  mg32x02z_dma_drv.o(i.DMA_Source_Select)
    DMA_StartRequest                         0x000006b1   Thumb Code    12  mg32x02z_dma_drv.o(i.DMA_StartRequest)
    GPIO_PinMode_Config                      0x000006bd   Thumb Code    38  mg32x02z_gpio_drv.o(i.GPIO_PinMode_Config)
    GPL_CRC_Check                            0x000006e5   Thumb Code  3978  main.o(i.GPL_CRC_Check)
    GPL_CRC_Config                           0x000017c5   Thumb Code    64  main.o(i.GPL_CRC_Config)
    GPL_DMA_Cmd                              0x00001805   Thumb Code    40  mg32x02z_gpl_drv.o(i.GPL_DMA_Cmd)
    MEM_SetFlashWaitState                    0x0000182d   Thumb Code    38  mg32x02z_mem_drv.o(i.MEM_SetFlashWaitState)
    ProtectModuleReg                         0x00001859   Thumb Code    20  mg32x02z__common_drv.o(i.ProtectModuleReg)
    Sample_URT0_Init                         0x0000186d   Thumb Code   344  main.o(i.Sample_URT0_Init)
    SystemInit                               0x000019d1   Thumb Code     8  system_mg32x02z.o(i.SystemInit)
    URT_BaudRateGenerator_Cmd                0x000019e1   Thumb Code    16  mg32x02z_urt_drv.o(i.URT_BaudRateGenerator_Cmd)
    URT_BaudRateGenerator_Config             0x000019f1   Thumb Code    32  mg32x02z_urt_drv.o(i.URT_BaudRateGenerator_Config)
    URT_ClearITFlag                          0x00001a15   Thumb Code    10  mg32x02z_urt_drv.o(i.URT_ClearITFlag)
    URT_Cmd                                  0x00001a1f   Thumb Code    12  mg32x02z_urt_drv.o(i.URT_Cmd)
    URT_DataCharacter_Config                 0x00001a2b   Thumb Code    64  mg32x02z_urt_drv.o(i.URT_DataCharacter_Config)
    URT_DataLine_Select                      0x00001a6b   Thumb Code    12  mg32x02z_urt_drv.o(i.URT_DataLine_Select)
    URT_GetITSingleFlagStatus                0x00001a79   Thumb Code    28  mg32x02z_urt_drv.o(i.URT_GetITSingleFlagStatus)
    URT_ITEA_Cmd                             0x00001a99   Thumb Code    12  mg32x02z_urt_drv.o(i.URT_ITEA_Cmd)
    URT_IT_Cmd                               0x00001aa5   Thumb Code    16  mg32x02z_urt_drv.o(i.URT_IT_Cmd)
    URT_IdlehandleMode_Select                0x00001ab5   Thumb Code    14  mg32x02z_urt_drv.o(i.URT_IdlehandleMode_Select)
    URT_Mode_Select                          0x00001ac3   Thumb Code    38  mg32x02z_urt_drv.o(i.URT_Mode_Select)
    URT_RXClockSource_Select                 0x00001ae9   Thumb Code    14  mg32x02z_urt_drv.o(i.URT_RXClockSource_Select)
    URT_RXOverSamplingMode_Select            0x00001af7   Thumb Code    12  mg32x02z_urt_drv.o(i.URT_RXOverSamplingMode_Select)
    URT_RXOverSamplingSampleNumber_Select    0x00001b03   Thumb Code    16  mg32x02z_urt_drv.o(i.URT_RXOverSamplingSampleNumber_Select)
    URT_RXShadowBufferThreshold_Select       0x00001b13   Thumb Code    14  mg32x02z_urt_drv.o(i.URT_RXShadowBufferThreshold_Select)
    URT_RX_Cmd                               0x00001b21   Thumb Code    14  mg32x02z_urt_drv.o(i.URT_RX_Cmd)
    URT_SetTXData                            0x00001b2f   Thumb Code    50  mg32x02z_urt_drv.o(i.URT_SetTXData)
    URT_TXClockSource_Select                 0x00001b61   Thumb Code    14  mg32x02z_urt_drv.o(i.URT_TXClockSource_Select)
    URT_TXGaudTime_Select                    0x00001b6f   Thumb Code     4  mg32x02z_urt_drv.o(i.URT_TXGaudTime_Select)
    URT_TXOverSamplingSampleNumber_Select    0x00001b73   Thumb Code    16  mg32x02z_urt_drv.o(i.URT_TXOverSamplingSampleNumber_Select)
    URT_TX_Cmd                               0x00001b83   Thumb Code    14  mg32x02z_urt_drv.o(i.URT_TX_Cmd)
    UnProtectModuleReg                       0x00001b91   Thumb Code    18  mg32x02z__common_drv.o(i.UnProtectModuleReg)
    __0printf$8                              0x00001ba9   Thumb Code    24  printf8.o(i.__0printf$8)
    __1printf$8                              0x00001ba9   Thumb Code     0  printf8.o(i.__0printf$8)
    __2printf                                0x00001ba9   Thumb Code     0  printf8.o(i.__0printf$8)
    __scatterload_copy                       0x00001bc9   Thumb Code    14  handlers.o(i.__scatterload_copy)
    __scatterload_null                       0x00001bd7   Thumb Code     2  handlers.o(i.__scatterload_null)
    __scatterload_zeroinit                   0x00001bd9   Thumb Code    14  handlers.o(i.__scatterload_zeroinit)
    fputc                                    0x0000205d   Thumb Code    48  main.o(i.fputc)
    main                                     0x0000208d   Thumb Code    42  main.o(i.main)
    Region$$Table$$Base                      0x00002520   Number         0  anon$$obj.o(Region$$Table)
    Region$$Table$$Limit                     0x00002540   Number         0  anon$$obj.o(Region$$Table)
    DataPattern                              0x20000000   Data           9  main.o(.data)
    SystemCoreClock                          0x2000000c   Data           4  system_mg32x02z.o(.data)
    __stdout                                 0x20000010   Data           4  stdout.o(.data)
    __initial_sp                             0x20000418   Data           0  startup_mg32x02z.o(STACK)



==============================================================================

Memory Map of the image

  Image Entry point : 0x000000c1

  Load Region LR_IROM1 (Base: 0x00000000, Size: 0x00002554, Max: 0x00020000, ABSOLUTE)

    Execution Region ER_IROM1 (Exec base: 0x00000000, Load base: 0x00000000, Size: 0x00002540, Max: 0x00020000, ABSOLUTE)

    Exec Addr    Load Addr    Size         Type   Attr      Idx    E Section Name        Object

    0x00000000   0x00000000   0x000000c0   Data   RO         5520    RESET               startup_mg32x02z.o
    0x000000c0   0x000000c0   0x00000000   Code   RO         5554  * .ARM.Collect$$$$00000000  mc_p.l(entry.o)
    0x000000c0   0x000000c0   0x00000004   Code   RO         5822    .ARM.Collect$$$$00000001  mc_p.l(entry2.o)
    0x000000c4   0x000000c4   0x00000004   Code   RO         5825    .ARM.Collect$$$$00000004  mc_p.l(entry5.o)
    0x000000c8   0x000000c8   0x00000000   Code   RO         5827    .ARM.Collect$$$$00000008  mc_p.l(entry7b.o)
    0x000000c8   0x000000c8   0x00000000   Code   RO         5829    .ARM.Collect$$$$0000000A  mc_p.l(entry8b.o)
    0x000000c8   0x000000c8   0x00000008   Code   RO         5830    .ARM.Collect$$$$0000000B  mc_p.l(entry9a.o)
    0x000000d0   0x000000d0   0x00000000   Code   RO         5832    .ARM.Collect$$$$0000000D  mc_p.l(entry10a.o)
    0x000000d0   0x000000d0   0x00000000   Code   RO         5834    .ARM.Collect$$$$0000000F  mc_p.l(entry11a.o)
    0x000000d0   0x000000d0   0x00000004   Code   RO         5823    .ARM.Collect$$$$00002712  mc_p.l(entry2.o)
    0x000000d4   0x000000d4   0x00000024   Code   RO         5521    .text               startup_mg32x02z.o
    0x000000f8   0x000000f8   0x00000060   Code   RO         5837    .text               mc_p.l(uldiv.o)
    0x00000158   0x00000158   0x00000024   Code   RO         5850    .text               mc_p.l(init.o)
    0x0000017c   0x0000017c   0x00000020   Code   RO         5852    .text               mc_p.l(llshl.o)
    0x0000019c   0x0000019c   0x00000022   Code   RO         5854    .text               mc_p.l(llushr.o)
    0x000001be   0x000001be   0x00000002   PAD
    0x000001c0   0x000001c0   0x0000001c   Code   RO          512    i.CSC_CK_AHB_Divider_Select  mg32x02z_csc_drv.o
    0x000001dc   0x000001dc   0x0000001c   Code   RO          513    i.CSC_CK_APB_Divider_Select  mg32x02z_csc_drv.o
    0x000001f8   0x000001f8   0x00000020   Code   RO          514    i.CSC_CK_HS_Select  mg32x02z_csc_drv.o
    0x00000218   0x00000218   0x00000020   Code   RO          516    i.CSC_CK_MAIN_Select  mg32x02z_csc_drv.o
    0x00000238   0x00000238   0x0000000c   Code   RO          519    i.CSC_ClearFlag     mg32x02z_csc_drv.o
    0x00000244   0x00000244   0x0000001c   Code   RO          521    i.CSC_GetSingleFlagStatus  mg32x02z_csc_drv.o
    0x00000260   0x00000260   0x00000024   Code   RO          525    i.CSC_IHRCO_Cmd     mg32x02z_csc_drv.o
    0x00000284   0x00000284   0x00000024   Code   RO          526    i.CSC_IHRCO_Select  mg32x02z_csc_drv.o
    0x000002a8   0x000002a8   0x0000008c   Code   RO            3    i.CSC_Init          main.o
    0x00000334   0x00000334   0x00000024   Code   RO          531    i.CSC_PLL_Cmd       mg32x02z_csc_drv.o
    0x00000358   0x00000358   0x00000030   Code   RO          532    i.CSC_PLL_Config    mg32x02z_csc_drv.o
    0x00000388   0x00000388   0x000000a8   Code   RO          533    i.CSC_PeriphOnModeClock_Config  mg32x02z_csc_drv.o
    0x00000430   0x00000430   0x0000009c   Code   RO          534    i.CSC_PeriphProcessClockSource_Config  mg32x02z_csc_drv.o
    0x000004cc   0x000004cc   0x00000014   Code   RO         1384    i.DMA_AutoIncreaseDestinationAddress  mg32x02z_dma_drv.o
    0x000004e0   0x000004e0   0x00000010   Code   RO         1385    i.DMA_AutoIncreaseSourceAddress  mg32x02z_dma_drv.o
    0x000004f0   0x000004f0   0x00000034   Code   RO         1386    i.DMA_BaseInitStructure_Init  mg32x02z_dma_drv.o
    0x00000524   0x00000524   0x0000006a   Code   RO         1387    i.DMA_Base_Init     mg32x02z_dma_drv.o
    0x0000058e   0x0000058e   0x00000010   Code   RO         1388    i.DMA_Channel_Cmd   mg32x02z_dma_drv.o
    0x0000059e   0x0000059e   0x00000004   Code   RO         1390    i.DMA_ClearFlag     mg32x02z_dma_drv.o
    0x000005a2   0x000005a2   0x00000002   PAD
    0x000005a4   0x000005a4   0x00000018   Code   RO         1391    i.DMA_Cmd           mg32x02z_dma_drv.o
    0x000005bc   0x000005bc   0x00000010   Code   RO         1393    i.DMA_Destination_Select  mg32x02z_dma_drv.o
    0x000005cc   0x000005cc   0x00000012   Code   RO         1399    i.DMA_GetSingleFlagStatus  mg32x02z_dma_drv.o
    0x000005de   0x000005de   0x00000002   PAD
    0x000005e0   0x000005e0   0x0000006c   Code   RO            4    i.DMA_Init          main.o
    0x0000064c   0x0000064c   0x00000014   Code   RO         1404    i.DMA_LoopMode_Cmd  mg32x02z_dma_drv.o
    0x00000660   0x00000660   0x00000014   Code   RO         1406    i.DMA_SetBurstSize  mg32x02z_dma_drv.o
    0x00000674   0x00000674   0x00000004   Code   RO         1408    i.DMA_SetDestinationAddress  mg32x02z_dma_drv.o
    0x00000678   0x00000678   0x00000010   Code   RO         1409    i.DMA_SetExtTriggerMode  mg32x02z_dma_drv.o
    0x00000688   0x00000688   0x00000010   Code   RO         1410    i.DMA_SetExtTriggerPin  mg32x02z_dma_drv.o
    0x00000698   0x00000698   0x00000004   Code   RO         1413    i.DMA_SetSourceAddress  mg32x02z_dma_drv.o
    0x0000069c   0x0000069c   0x00000004   Code   RO         1414    i.DMA_SetTransferDataNumber  mg32x02z_dma_drv.o
    0x000006a0   0x000006a0   0x00000010   Code   RO         1415    i.DMA_Source_Select  mg32x02z_dma_drv.o
    0x000006b0   0x000006b0   0x0000000c   Code   RO         1416    i.DMA_StartRequest  mg32x02z_dma_drv.o
    0x000006bc   0x000006bc   0x00000026   Code   RO         1023    i.GPIO_PinMode_Config  mg32x02z_gpio_drv.o
    0x000006e2   0x000006e2   0x00000002   PAD
    0x000006e4   0x000006e4   0x000010e0   Code   RO            5    i.GPL_CRC_Check     main.o
    0x000017c4   0x000017c4   0x00000040   Code   RO            6    i.GPL_CRC_Config    main.o
    0x00001804   0x00001804   0x00000028   Code   RO         1239    i.GPL_DMA_Cmd       mg32x02z_gpl_drv.o
    0x0000182c   0x0000182c   0x0000002c   Code   RO          808    i.MEM_SetFlashWaitState  mg32x02z_mem_drv.o
    0x00001858   0x00001858   0x00000014   Code   RO          249    i.ProtectModuleReg  mg32x02z__common_drv.o
    0x0000186c   0x0000186c   0x00000164   Code   RO            7    i.Sample_URT0_Init  main.o
    0x000019d0   0x000019d0   0x00000010   Code   RO         5528    i.SystemInit        system_mg32x02z.o
    0x000019e0   0x000019e0   0x00000010   Code   RO         4242    i.URT_BaudRateGenerator_Cmd  mg32x02z_urt_drv.o
    0x000019f0   0x000019f0   0x00000024   Code   RO         4243    i.URT_BaudRateGenerator_Config  mg32x02z_urt_drv.o
    0x00001a14   0x00001a14   0x0000000a   Code   RO         4256    i.URT_ClearITFlag   mg32x02z_urt_drv.o
    0x00001a1e   0x00001a1e   0x0000000c   Code   RO         4260    i.URT_Cmd           mg32x02z_urt_drv.o
    0x00001a2a   0x00001a2a   0x00000040   Code   RO         4269    i.URT_DataCharacter_Config  mg32x02z_urt_drv.o
    0x00001a6a   0x00001a6a   0x0000000c   Code   RO         4270    i.URT_DataLine_Select  mg32x02z_urt_drv.o
    0x00001a76   0x00001a76   0x00000002   PAD
    0x00001a78   0x00001a78   0x00000020   Code   RO         4281    i.URT_GetITSingleFlagStatus  mg32x02z_urt_drv.o
    0x00001a98   0x00001a98   0x0000000c   Code   RO         4300    i.URT_ITEA_Cmd      mg32x02z_urt_drv.o
    0x00001aa4   0x00001aa4   0x00000010   Code   RO         4301    i.URT_IT_Cmd        mg32x02z_urt_drv.o
    0x00001ab4   0x00001ab4   0x0000000e   Code   RO         4304    i.URT_IdlehandleMode_Select  mg32x02z_urt_drv.o
    0x00001ac2   0x00001ac2   0x00000026   Code   RO         4308    i.URT_Mode_Select   mg32x02z_urt_drv.o
    0x00001ae8   0x00001ae8   0x0000000e   Code   RO         4315    i.URT_RXClockSource_Select  mg32x02z_urt_drv.o
    0x00001af6   0x00001af6   0x0000000c   Code   RO         4318    i.URT_RXOverSamplingMode_Select  mg32x02z_urt_drv.o
    0x00001b02   0x00001b02   0x00000010   Code   RO         4319    i.URT_RXOverSamplingSampleNumber_Select  mg32x02z_urt_drv.o
    0x00001b12   0x00001b12   0x0000000e   Code   RO         4321    i.URT_RXShadowBufferThreshold_Select  mg32x02z_urt_drv.o
    0x00001b20   0x00001b20   0x0000000e   Code   RO         4323    i.URT_RX_Cmd        mg32x02z_urt_drv.o
    0x00001b2e   0x00001b2e   0x00000032   Code   RO         4329    i.URT_SetTXData     mg32x02z_urt_drv.o
    0x00001b60   0x00001b60   0x0000000e   Code   RO         4332    i.URT_TXClockSource_Select  mg32x02z_urt_drv.o
    0x00001b6e   0x00001b6e   0x00000004   Code   RO         4336    i.URT_TXGaudTime_Select  mg32x02z_urt_drv.o
    0x00001b72   0x00001b72   0x00000010   Code   RO         4339    i.URT_TXOverSamplingSampleNumber_Select  mg32x02z_urt_drv.o
    0x00001b82   0x00001b82   0x0000000e   Code   RO         4340    i.URT_TX_Cmd        mg32x02z_urt_drv.o
    0x00001b90   0x00001b90   0x00000018   Code   RO          252    i.UnProtectModuleReg  mg32x02z__common_drv.o
    0x00001ba8   0x00001ba8   0x00000020   Code   RO         5768    i.__0printf$8       mc_p.l(printf8.o)
    0x00001bc8   0x00001bc8   0x0000000e   Code   RO         5864    i.__scatterload_copy  mc_p.l(handlers.o)
    0x00001bd6   0x00001bd6   0x00000002   Code   RO         5865    i.__scatterload_null  mc_p.l(handlers.o)
    0x00001bd8   0x00001bd8   0x0000000e   Code   RO         5866    i.__scatterload_zeroinit  mc_p.l(handlers.o)
    0x00001be6   0x00001be6   0x00000002   PAD
    0x00001be8   0x00001be8   0x00000428   Code   RO         5775    i._printf_core      mc_p.l(printf8.o)
    0x00002010   0x00002010   0x00000020   Code   RO         5776    i._printf_post_padding  mc_p.l(printf8.o)
    0x00002030   0x00002030   0x0000002c   Code   RO         5777    i._printf_pre_padding  mc_p.l(printf8.o)
    0x0000205c   0x0000205c   0x00000030   Code   RO            9    i.fputc             main.o
    0x0000208c   0x0000208c   0x00000038   Code   RO           10    i.main              main.o
    0x000020c4   0x000020c4   0x00000459   Data   RO           11    .conststring        main.o
    0x0000251d   0x0000251d   0x00000003   PAD
    0x00002520   0x00002520   0x00000020   Data   RO         5862    Region$$Table       anon$$obj.o


    Execution Region RW_IRAM1 (Exec base: 0x20000000, Load base: 0x00002540, Size: 0x00000418, Max: 0x00003800, ABSOLUTE)

    Exec Addr    Load Addr    Size         Type   Attr      Idx    E Section Name        Object

    0x20000000   0x00002540   0x00000009   Data   RW           12    .data               main.o
    0x20000009   0x00002549   0x00000003   PAD
    0x2000000c   0x0000254c   0x00000004   Data   RW         5529    .data               system_mg32x02z.o
    0x20000010   0x00002550   0x00000004   Data   RW         5836    .data               mc_p.l(stdout.o)
    0x20000014   0x00002554   0x00000004   PAD
    0x20000018        -       0x00000400   Zero   RW         5518    STACK               startup_mg32x02z.o


==============================================================================

Image component sizes


      Code (inc. data)   RO Data    RW Data    ZI Data      Debug   Object Name

      5092       1914       1113          9          0     192815   main.o
        44          6          0          0          0       1176   mg32x02z__common_drv.o
       640         68          0          0          0       7317   mg32x02z_csc_drv.o
       384         12          0          0          0      13168   mg32x02z_dma_drv.o
        38          0          0          0          0        918   mg32x02z_gpio_drv.o
        40          0          0          0          0        506   mg32x02z_gpl_drv.o
        44          6          0          0          0        568   mg32x02z_mem_drv.o
         0          0          0          0          0       1232   mg32x02z_pw_drv.o
       430          8          0          0          0      12543   mg32x02z_urt_drv.o
        36         10        192          0       1024        720   startup_mg32x02z.o
        16          8          0          4          0        779   system_mg32x02z.o

    ----------------------------------------------------------------------
      6772       2032       1340         16       1024     231742   Object Totals
         0          0         32          0          0          0   (incl. Generated)
         8          0          3          3          0          0   (incl. Padding)

    ----------------------------------------------------------------------

      Code (inc. data)   RO Data    RW Data    ZI Data      Debug   Library Member Name

         0          0          0          0          0          0   entry.o
         0          0          0          0          0          0   entry10a.o
         0          0          0          0          0          0   entry11a.o
         8          4          0          0          0          0   entry2.o
         4          0          0          0          0          0   entry5.o
         0          0          0          0          0          0   entry7b.o
         0          0          0          0          0          0   entry8b.o
         8          4          0          0          0          0   entry9a.o
        30          0          0          0          0          0   handlers.o
        36          8          0          0          0         68   init.o
        32          0          0          0          0         68   llshl.o
        34          0          0          0          0         68   llushr.o
      1172         52          0          0          0        324   printf8.o
         0          0          0          4          0          0   stdout.o
        96          0          0          0          0         84   uldiv.o

    ----------------------------------------------------------------------
      1424         68          0          4          4        612   Library Totals
         4          0          0          0          4          0   (incl. Padding)

    ----------------------------------------------------------------------

      Code (inc. data)   RO Data    RW Data    ZI Data      Debug   Library Name

      1420         68          0          4          0        612   mc_p.l

    ----------------------------------------------------------------------
      1424         68          0          4          4        612   Library Totals

    ----------------------------------------------------------------------

==============================================================================


      Code (inc. data)   RO Data    RW Data    ZI Data      Debug   

      8196       2100       1340         20       1028     229558   Grand Totals
      8196       2100       1340         20       1028     229558   ELF Image Totals
      8196       2100       1340         20          0          0   ROM Totals

==============================================================================

    Total RO  Size (Code + RO Data)                 9536 (   9.31kB)
    Total RW  Size (RW Data + ZI Data)              1048 (   1.02kB)
    Total ROM Size (Code + RO Data + RW Data)       9556 (   9.33kB)

==============================================================================

